:020000040800F2
:1000000000A00020B13901086DE30008E5290108CE
:100010006BE3000869E3000867E3000800000000E4
:1000200000000000000000000000000065E3000880
:1000300063E300080000000061E3000809CF000846
:10004000193A0108193A0108193A0108193A010840
:10005000193A0108193A0108193A0108193A010830
:10006000193A0108193A0108193A0108193A010820
:10007000193A0108714900083FD40008193A0108EB
:10008000193A0108193A0108193A0108193A010800
:10009000CDE30008193A0108193A0108193A010894
:1000A000591101088511010849110108951101082C
:1000B0007911010869110108193A0108193A010872
:1000C000193A0108193A0108193A0108193A0108C0
:1000D000193A0108511301084513010839130108A1
:1000E00019CF0008193A010851E30008193A01082C
:1000F000193A0108193A0108193A0108193A010890
:10010000000000000000000000000000193A010893
:10011000193A0108193A0108193A0108193A01086F
:10012000193A0108193A0108193A0108193A01085F
:10013000193A0108193A0108000000000000000007
:10014000193A0108193A0108193A0108000000009B
:10015000000000000000000000000000000000009F
:100160000000000000000000193A0108193A0108D7
:10017000193A010800000000000000000000000023
:0801800000000000193A01081B
:100188002DE9F04F2DED028B6F4E704B3360AFB001
:100198000023736011F0DEF818B911F0FDF809F0CA
:1001A8007DFB09F035FC6A4B6A4C1A7842F0010273
:1001B8001A70694A4FF47001C2F888100022099237
:1001C8000A92226842F4803222600493236803F47E
:1001D80000330A93099B013309930A9B1BB9099BB6
:1001E800B3F5A04FF2D1236813F4003318BF0123ED
:1001F8000A930A9B012B70D0574F584BFB60636AD8
:10020800B360636ADFF884A1DFF88481DFF8849142
:1002180043F080736362636943F4FC032EAD63614A
:1002280003238DF86A3041F6FF7325F8503D4FF0EF
:100238009040294604F08EFC4FF6FF73504629463D
:10024800ADF8683004F086FC4548294604F082FC85
:100258004448294604F07EFC4348294604F07AFCC9
:100268002946424804F076FC284607F0AFFE1A9B60
:100278003F4AB3FBF2F33F4A3F4913603F4B00222A
:100288001A603F4B5960F02187F823109A603D4F60
:1002980007221A60BB68C8F8003099E80F0085E8A3
:1002A8000F0063691A9843F480236361636943F418
:1002B800802363614FF0200B1023CAF818301BA964
:1002C800CAF818B004F046FC1DA91C9804F042FCBA
:1002D800D8F80030190729D464E02B4B12221A6091
:1002E8006368636063686360636843F48063636042
:1002F800636823F47C136360636843F4E813636002
:10030800236843F0807323602268124B9201FBD567
:100318005A6822F003025A605A6842F002025A6090
:10032800636803F00C03082BFAD165E797F892315C
:10033800012B37D8044B97F893219B6813F080530F
:1003480000F0A7842EE000BF780100201F9100086C
:10035800982F00200010024000ED00E00005FA058B
:1003680000080048000C004800100048001400482D
:1003780040420F00FC1700203F19010038180020E8
:1003880010E000E02C250020002002400004004876
:10039800CC240020F87D0108B54B002283F8932176
:1003A80009F0D2FC64200CF034FCC822B1480021CA
:1003B80015F059FBE369B04A43F00303E361A3690D
:1003C80043F4A123A361636943F4C023636102F189
:1003D800B00C937B506892F80FE003F00701DB083C
:1003E80000EB83038900186A4FF00F0A0EFA01FE2A
:1003F8000AFA01F120EA01011962196A10324EEA7B
:10040800010162451962E4D10023DFF894A20AF1E0
:100418000C020021995401330B2BF6D1FF23974A84
:100428008AF817308AF818308AF819308AF81A309A
:100438008AF81B30924BDFF86CB21360914A039331
:10044800042010705846302215F00DFB14220221AA
:100458008BF800208BF8241001228B49039B8BF822
:10046800182097F805B081F800B0A3F5EE71CAF826
:100478001C108649D8F80080A3F58E730B60844B56
:1004880003EBCB0318F0200F5B78CAF8203018BFB5
:10049800CAF8202000237F4A40F2DC5122F81310CA
:1004A8000133082BF7D113A800211C2215F0DBFA21
:1004B800BBF10E0F03D00BF0EF03082B02D1012381
:1004C8008DF85C3002200CF02FFA18B1408800300B
:1004D80018BF0120C8F340038DF85230C8F38013C9
:1004E8008DF85430C8F340338DF84C30C8F3C0331E
:1004F80000F001008DF84F3018F400638DF85100BA
:1005080007D097F8863103F1FF3EDEF1000343EB95
:100518000E038DF85030C8F300438DF85530336A18
:10052800B7F84801ADF86000003318BF01238DF813
:100538005630C8F300538DF85730B7F84A31ADF844
:100548005A3018F4805FB7F8563118BF4848ADF8EC
:100558005830C8F380438DF85330B7F854311CBF76
:10056800B0F85001ADF86000B3F5FA7FADF85E3031
:1005780084BF0023ADF86030474897F8D63186F835
:100588002430002386F8253043709DF85C3008F04D
:100598000101002BC8F3C0028DF84D108DF84E20D4
:1005A8000CBF0023022301B902B1013309EB83090F
:1005B8004FF0000AD9F810309A1E143303920593AD
:1005C800039A32F8023F03924FF6FF72934200F00B
:1005D80089819DF85100190ADAB2CBB280B1264F51
:1005E800DFF8C4E007EB02177868704508D138894E
:1005F800B0F5806F00F07181B0F5006F00F06D818B
:100608009DF8550090B11001DFF86CE00EEB000783
:100618005EF800E02148864500F05F817868B0F117
:10062800904F03D1B87B062800F057819DF85200FF
:1006380050B1114F07EB02177868B0F1904F03D112
:100648003889102800F049819DF8500050B10A4FB0
:1006580007EB02177868B0F1904F03D138898028EA
:1006680000F03B81022921D19DF84C1022E000BF07
:100678002C250020701800209CA00108442300208D
:100688001C2700202D1200209C090020B4190020EE
:1006980030AE01089C1100209D010020004401405B
:1006A800780100204823002000040048012904D1D3
:1006B8009DF84D10002900F010819DF85600BF49A3
:1006C8004FEA021850B19DF85C0038B9012A05D8E4
:1006D80051F80800BA4FB84208BF04239DF85700E4
:1006E80001EB080730B19DF85C0018B9043A032AF9
:1006F80040F2DC80012B53D19DF85330DFF8D092C3
:100708003BB151F80830B3F1804F04BF032389F897
:100718002730AA4AC9F87C7002EB0801FF2391F838
:100728000DE089F86C3089F86D3048688DF86AE01A
:1007380001F108030989ADF868104FF0000B022198
:100748008DF86B1089F870B01AA90792069389F88A
:1007580028B0C9F82CB0C9F830B0C9F834B0C9F815
:1007680068B089F86EB089F86FB004F0F3F9069BA9
:10077800079A997852F808005A4604F03FF8384624
:1007880011F0AEF98F4B9049C9F880308F4BC9F8FA
:100798008430C9F888B038460A1D10F06FFD9CE017
:1007A800022B49D15FFA8AF21C2101FB02FC884A1C
:1007B800CDF81CC002EB0C09804A89F871A0012110
:1007C80089F8701002EB08014FF0000B91F80DE06A
:1007D800486889F872B001F108020989ADF8681013
:1007E80089F87AB01AA9C9F87C708DF86AE006927F
:1007F8008DF86B3004F0AEF9704B069A53F8080088
:1008080091785A4603F0FAFF384611F069F9704BAF
:10081800DDF81CC06F4AC9F8802003EB0C016E4A52
:10082800C9F884208031C9F888B038460A1D10F00C
:1008380025FD0AF1010A50E0032B35D19DF853300C
:10084800DFF88C81DFF8C4913BB198F826B03846C0
:1008580008214FF6FF7200231AE0BDF85E2098F8D1
:1008680026B0BDF86030B2F5FA7F0BD95B49B1FB11
:10087800F2F23846082192B204F095F9584B49F83B
:100888002B000AE05749B1FBF2F23846012192B237
:1008980004F089F9544B49F82B00C36098F82630C6
:1008A800013388F8263018E0042B16D196F82580F5
:1008B800BDF858204B4B93FBF2F23846BDF85A303E
:1008C800012192B204F06FF996F8253006EB8808FA
:1008D8000133C8F8500186F82530039B059A9342E6
:1008E8007FF46EAE96F8252086F870213F4A404B7B
:1008F80092F800E0AEF117020027022A1F709C460A
:100908001AD8F3693B44D3ED007AF5EE407AF1EE5C
:1009180010FA02D1336A63BB26E0364A07EB0208B5
:100928000FCB88E80F009CF8003010370133C02F38
:100938008CF80030E5D1EDE72F4B13F83E908CF89A
:10094800009003EBCE03D3F804A0BAF1000FE1D076
:100958004F45DFDA274A3B0103EB020853440FCB2C
:10096800013788E80F00F3E7244F3B68DE0451D4D1
:100978001DE0234B234A13F83E00107003EBCE030F
:100988005E68002EF0D000238342EDDAC3EBC3018A
:100998007218DFF87C80D2F8009041F8089001EBDB
:1009A80008079188B9809279BA710133ECE70EF0A3
:1009B800EF03082B144B4DD14FE000BF9CA001085A
:1009C800004001408D450008F801002079460008E4
:1009D80078010020014900086545000800127A00E6
:1009E8009946000840420F00894600089C090020EB
:1009F8006C180020D808002030AE0108CC24002054
:100A08007486010840190020701200203C1800204C
:100A1800411900209CF80020012AC8D9B94B03EBE2
:100A28000212103210339342C1D053ED047AB6EE5D
:100A3800007A67EE877A43ED047A53ED057A67EE1C
:100A4800877A43ED057A53ED037A67EE877A43EDAB
:100A5800037AE7E7BEF10E0F09D11A7842F01002C7
:100A68001A70BEF1180F09D10CF004FC06E01A78D0
:100A780022F010021A70BEF1190FF4E70CF0DEFB39
:100A88003B68A14E58035EBFA04B01221A70049B1D
:100A9800049A1B7843F0040313709D4B1E6063692E
:100AA80043F400336361E36943F48003E361236B38
:100AB80023F020032363236B43F080534FF09048C7
:100AC80043F020032363D8F8243023F0F003C8F858
:100AD8002430D8F8243043F04003C8F82430D8F83C
:100AE800243023F47063C8F82430D8F8243043F451
:100AF8008063C8F824304FF0000902234FF40072D5
:100B080029464FF0030B40468DF86C3004931A9237
:100B18008DF86E908DF86F908DF86DB007F0C4FB6E
:100B28004FF48062294640461A9207F0BDFB3268AE
:100B380022F0010232603168764A0A403260764A11
:100B48003261326842F001023260C6F80890C6F895
:100B58000C90C6F80890B26842F40042B26032685D
:100B68003260726822F0784222F400427260326881
:100B780042F0010232603D68684E4FF0100A05F4F9
:100B88000063524630464946039314F06CFF4FF613
:100B9800FF72049B0E9215F002058DF83D308DF81A
:100BA8003E908DF83F908DF83CB00CD02EA9404671
:100BB80041F880AD07F078FB01250723357086F8EA
:100BC8000190F370B570039B83B12EA9802341F87F
:100BD800803D4FF0904007F067FB042333730723F1
:100BE800F373012375731D44B373EDB2E36A4C4884
:100BF80023F4F873E362E36A43F4D873E362636946
:100C080043F0805343F00203636107F014F91AA814
:100C180007F0E6F8434B1A93434B1B93022D4FF012
:100C2800000314BF1A4680221F924FF480723C4C76
:100C380020924FF4806221922022204622921AA903
:100C48004FF400521C931E9323922493ADF87450D2
:100C580007F0D3F8236843F001032360334CA368FB
:100C680023F04053A360A36843F08053A3600A2095
:100C78000BF0CFFFA36823F08043A360A368A360B1
:100C8800A36843F00043A360A368284A002B51DA05
:100C9800FAE7013A092A3FF685ABD9F8240003930D
:100CA8002946AAF828B028604FF0904003F052FF78
:100CB8004FF09042082191613C200BF0AAFF039B62
:100CC800CAF818B09A4697F893319A45BFF664ABBC
:100CD800174A4FF0904B1021082391617820069114
:100CE8000592ABF8283003930BF088FF059A069914
:100CF800039B11857820CBF818300BF07FFF0AF1A1
:100D0800010AE0E7E008002000580040080E002033
:100D180068110020FFE0CF007A25E000EC150020E4
:100D28000804024040010050FC150020000100505A
:100D3800000400489368AD4923F0405393609368DA
:100D480043F0005393608868A94B034043F4683329
:100D58008B60D168A74B0B4043F40053D360136BEF
:100D6800013D23F00F031D431563002401233219AD
:100D78009178002972D05D1C042B16F804E0D07815
:100D8800DFF874C2EDB20ED803EB43035A00DCF867
:100D980030101F23934021EA03010EFA02F30B439C
:100DA800CCF8303031E0092B0ED8053B06225A43E7
:100DB800DCF834101F23934021EA03010EFA02F3F2
:100DC8000B43CCF8343020E00E2B4FF006010ED840
:100DD800A3F10A024A43DCF838801F23934028EA2B
:100DE80003010EFA02F30B43CCF838300DE00F3B49
:100DF80001FB03F2DCF83C801F23934028EA03013F
:100E08000EFA02F30B43CCF83C30BEF1090F7A4AD4
:100E180011D993699169AEF10A0303EB43034FF0CB
:100E2800070E0EFA03FE21EA0E01916191699840BE
:100E38000843906111E0536951690EF1FF3303EBE8
:100E480043034FF0380E0EFA03FE21EA0E015161FA
:100E5800516903339840084350612B460434102CE1
:100E680085D1654B9A6842F001029A601A4611686A
:100E7800614BC907FBD5DA6822F00202DA60DA684A
:100E880042F00202DA60DA6842F00102DA609A6837
:100E980042F004029A60594AB2F85C319046002B3D
:100EA80040F09487B8F95E21002A40F08F87B8F99E
:100EB8006021002A40F08A873B68514C13F4003FB8
:100EC8001FD0C8200BF0A5FEAE2010F0A4F808B182
:100ED80010F0A6F84B4D84F87101C8200BF099FE6C
:100EE800494BC4F8743100210C22284614F0BBFD8C
:100EF8000223EB700AF08BFB0BF064FE434B0344B8
:100F0800AB6098F86B310393414B42481B68B8F8C3
:100F18006461B3F8563098F863B198F86C5104934B
:100F280000210C22B8F80C9098F80FA014F09BFD43
:100F3800394B069318460021142214F094FD374AC1
:100F4800002111702E4A0592C2F8781110F025F888
:100F5800059A8046002833D0069B314919603149EB
:100F680059603149D960B6F5807F30491961304BF5
:100F780001D1002116E0BB2E01D9012112E0612E1A
:100F880001D902210EE0292E01D903210AE0132EEE
:100F980001D9042106E0092E01D9052102E0002E1D
:100FA800E7D0062119701D4B04211970214B02212D
:100FB800197021490B6843F001030B6059460FE093
:100FC80003200BF06BFF35E24FF0010B0BFA01F039
:100FD80040F2B23303409BB3012940F28D800021D7
:100FE8001648002309290370F9D8EDE700030050DB
:100FF800E010FCFF07C0FFFD000100502C25002079
:10100800780100207C170020B6260020404B4C00B9
:10101800AC11002098230020742000208820002094
:10102800850E0108950D0108150E010890C1793D3E
:1010380000000020040100206C120020C62F0020B0
:1010480010F04D0FC8D00691C2F8783105920FF014
:10105800A4FF059A06990028BED0062168200A46F2
:101068000DEB000303F08CFE9DF86D1001EA0B02F6
:101078009DF86B1001EA0B0101FA0BF343EA8201B8
:101088009DF8692002EA0B030B430BD05BB25B456A
:1010980001D1002202E0022B0FD10122AF4B83F8CD
:1010A8007C2111E00EAB68200C215A4603F068FE43
:1010B8009DF8383013F00F0303D105200BF0EEFE36
:1010C80002E0042BE9D1E4E7A54BA64A1A60A64A38
:1010D8005A60A24A92F87C21002A0CBF6F226E2225
:1010E8001A72A24B04221A70A14B03225A70A14A09
:1010F800136843F002031360042D00F2A380DFE8B5
:1011080005F003BE6B036B000A200BF082FD77200D
:10111800A02101220EAB03F033FE00285CD01E2173
:101128000122772003F0A8FE4FF42F600BF066FD34
:101138004FF0000BABF160010025C9B202221AABD7
:1011480077208DF868508DF8695003F019FE9DF8E6
:1011580069309DF8682043EA0222804B03F5BF718D
:101168002BF801200BF1020BBBF1100FE2D1B3F801
:101178008C2102F00F0E02F47F42A3F88C2101208B
:101188002B462946DFF8D4C121F001056544B5F89E
:101198007E51002D18BF002011F0010F03D0EDB2D1
:1011A8006B40082502E083EA1523FAE713F4004FA1
:1011B80018BF83F4C053013D4FEA4303F6D1013110
:1011C8001029DFD1654942EA0E02A1F88C2118B92D
:1011D800C3F303339E4538D0604D95F88EB1BBF10B
:1011E800000F40F0E98514200BF013FD05F28F1372
:1011F8007620D021012203F0C3FD95F88F31582BBA
:101208003DD105F5C87388211822762003F0B8FD72
:1012180031227620F42103F02FFE012385F88E3148
:10122800554B564A9A60564A5A6045F6D8125A8023
:10123800544ADA60544A1A61544AA3F800B05A6111
:1012480000F0BABD012D13D119E04B4B42F21072D8
:101258001A805A804E4A5A604E4A9A604E4ADA605C
:101268004E4A1A614E4A5A61B8F1000FB4D00325AC
:101278003F4B404A9D70136843F0040313603D4D93
:101288002B689A0702D5364B1B6898473349454A5D
:10129800BAF1000F25D016F0FF0F0AD12B6813F012
:1012A800020F4FF07D0040F2712308BF4FF4FA732C
:1012B80002E04FF47A731846994505DBB9F57A6F61
:1012C800A8BF4FF47A6900E09946431E4B44B3FB2C
:1012D800F0F3013BDBB203FB000081F8AC31106096
:1012E80003E081F8ACA1C2F800902F4B1B68984727
:1012F800DDF80CA02D4E00233370BAF1000F04D096
:10130800AAF10202012A00F25A852EAB4FF0000919
:1013180003F8509D0C204946012203F031FD0028B6
:1013280000F07C859DF86830482B13D1204B214A6A
:101338001A60214A5A604046B8F1000F00F06E85E5
:10134800052333700A4B0322DA702B6843F0080335
:101358002B6033E0484600F061BD00BF78010020F3
:1013680098230020F50E0108D50D0108C62F00208E
:10137800040100206C120020D8060020396B0008F8
:101388003B6B0008C96D00085F6E00083D690008E6
:10139800430D0108850D0108390D0108750D010877
:1013A8003D6B0008082D002074200020C02F00206D
:1013B800B4060020A96E0008D36D0008174B93F8F7
:1013C80058210AB116490A7093F859210AB11549EA
:1013D8000A7093F85A3103B133702B68124913F02D
:1013E800080F25D0BDF91000DFED106A642290FBCC
:1013F800F2F302FB130212B207EE902AB8EEE77A74
:1014080007EE903AF8EEE77AE7EE267AB2EE047A3B
:1014180067EE877AC1ED007A0CE000BF2C2500202A
:1014280088200020C62F0020DC1F00208988883CE7
:1014380000230B60AB4B1A7842F002021A70AA4ADA
:1014480020211185102191610A259846A64EB38A5C
:101458009BB283F02003B382B38A9BB283F010035C
:10146800B38219200BF0D5FB013D19200BF0D1FBFD
:1014780015F0FF05EAD110234FF020099B4DB36109
:10148800C6F818902B681B0709D5994BA6F8289021
:101498001B689847974BC6F8189001221A70964B0C
:1014A8009FED968A1B68964E1B7B00EE103AB8EEAD
:1014B800C00A20EE080A08F0FBF8338807EE903AD5
:1014C800F8EEE77A27EE800A14F0DCFC8D4B9FEDEE
:1014D8008E7A188033888D4E07EE903AF8EEE77AC8
:1014E8008B4BC7EE277A3046FF211A229FED897A67
:1014F800C7EE877A9FED887AC3ED007A874BD3EDE4
:10150800047A874B67EE887A67EE877AC3ED007AAC
:1015180014F0A9FA002232702A68824B012112F0D5
:10152800020F19701FBF717003211970022118BFB3
:10153800B1703046560741BF19784D1C1D70032500
:1015480048BF455412F00A0F0CD01A780421815470
:10155800511CC9B205254554D11C0232D2B21970AA
:101568000621815439688D0641BF1A78551C1D70B3
:10157800072548BF85540A0608D51A7809258554D1
:10158800951C0132D2B21D700A258554664E7579B4
:10159800082D01D00E2D04D11A78571C1F700B2767
:1015A80087541A7811F4803F4FF00C0E00F802E0CF
:1015B80002F101071CBFDFF86CE10232FFB21F70B5
:1015C8001FBF8EF80020514A4FF00E0E02F807E0B8
:1015D8004A0741BF1A78571C1F70102748BF875405
:1015E8001A78571CFFB24FF0120E11F4806F1F705B
:1015F80000F802E00ED096F814E2BEF1000F09D010
:10160800DFF820E102328EF80020404A4FF0130E36
:1016180002F807E01A7811F4007F4FF0140E00F872
:1016280002E002F101071CBFDFF8F8E00232FFB266
:101638001F701FBF8EF80020344A4FF0150E02F8B5
:1016480007E0182D0DD11A7816278754571CFFB2BA
:101658004FF0170E00F807E0D71C0232D2B21F7005
:1016680085540D0341BF1A78511C1970192348BFBE
:101678008354002198222D4814F0F5F90EF017FE36
:101688002B4B2C4A2C491A6000234B800B712B4999
:101698000A60B6F8982190B2294921F8130001335D
:1016A800122BF9D1274F3B68D8045CBFB6F89E01CE
:1016B80008801B0740F1018196F89231062B00F251
:1016C800F680DFE803F0040745748FAFAF0045F2FA
:1016D800F05201E042F6F8221B4B1A800EF084FE0D
:1016E800E4E000BF982F0020000400486C1200209E
:1016F800B4060020CC0600201C21002035FA8E3CC0
:1017080004000020382100200AE81C41751100203F
:10171800EC07002000401C46BD37863574200020A9
:1017280018210020741100202C250020A022002060
:10173800440F0020B6260020940E00208C2F002095
:1017480008250020CC24002044080020CDCCCC3F24
:1017580007EE902A5FED036A814BB8EEE77ADFED7A
:10176800817AE7EE267A42F6F82119800023FCEE0A
:10177800E77A7D4A17EE901A42F823100133122BAC
:10178800F7D17A4A7A4911607A4A402013700BF0EF
:1017980003F9002800F08B8001234FF0070A90F925
:1017A8000000754A8DE808044021744B79E06C4BC1
:1017B80042F6F8221A806D4B714A1A606D4B10225E
:1017C80040201A700BF0E8F8002870D001234FF081
:1017D800000990F900006B4A8DE8080240214FF497
:1017E800E1335EE05E4B42F6F8221A805F4B664AB0
:1017F8001A60604B082240201A700BF0CDF80028C0
:1018080055D001234FF0000C90F900005F4A8DE895
:10181800081040214FF4E1330BF005FA5C4BC3F894
:10182800B00140E04E4ADFF89C91DFF89CC1DFF838
:101838009CE1584D584842F6F82111804D490C2238
:10184800062B0A700FD0002389F800308CF800307E
:101858008EF800301B232B70504B027005221A7033
:101868004FF4E1350CE0002189F800108CF80010E5
:101878008EF8001002702121484A2970484D1370D3
:101888003A4B484A1A6040200BF086F878B1012399
:101898004FF0000E444A90F9000040218DE80840BE
:1018A8002B460BF0C0F9003018BF012028B90820DA
:1018B80007F0C2FF2D4B3D4A1A603B682D4A13F4CE
:1018C800804F1FBF082111702849394818BF086088
:1018D80042F20101194003F0010003F4005581B1FF
:1018E8001F4944F6206EA1F800E025B108211170C7
:1018F8001E49304D0D6020B10C2111701B492E4836
:10190800086011781806A1F10401517040F19C801B
:101918000025DFF8BCA0DFF8BC902848DFF8B8B095
:10192800C4F8B491294615228AF80150CAF804501F
:10193800CAF8085014F097F8A9F105032846CBF81F
:10194800003005F0EBFD1E4B02201B68CAF80C3076
:101958000BF022F8002841D1802007F06DFF6BE0E2
:10196800440800200000B0C4DC2E0020F400002051
:10197800D12701083C230020DD280108A0860100AA
:10198800197A000835280108017A00084D7B0008FB
:1019980078010020821500200315002083150020FF
:1019A80090D003001D7900082D7A0008312801081D
:1019B8000528010821280108112801083003002002
:1019C800F024002004150020811500208015002037
:1019D800000800201C2700202008002045799AF8DC
:1019E8000130CB490C2202FB03125278AA4204D0E0
:1019F8000133DBB2042BF4D900238AF80130DBF879
:101A080000309AF801201B7890F90000002B4FF065
:101A18000C0303FB021314BF0325012500225B7886
:101A28000095019202210BF0FEF8BA4B18600028CD
:101A380092D0012005F072FDB74B1868B74B00F53E
:101A4800C5721A6005F018FEB54AB64B1360B64A5F
:101A5800DFF83093803313603B680025D90389F899
:101A6800005040F1BB800DF035FEDFF81CC3DFF8F5
:101A78001CB3CDF814C040F22A334FF0010A1A46BD
:101A880060462946049389F800A013F0ECFFDBF8C0
:101A98001420DFF8FC924FF0904042F40032CBF86B
:101AA8001420026A22F070620262026A42F08072B6
:101AB8000262032140220C928DF8351002220CA9F3
:101AC8008DF8342003928DF836508DF837A006F043
:101AD800EBFBDBF81810039A41F40031CBF818102F
:101AE800B9F8001021F440710904090CA9F8001094
:101AF8001D21C9F82C104846A9F828200EA9A9F8D4
:101B080030506022C9F814A00E92ADF83E501095DE
:101B1800ADF84450ADF84650ADF84850ADF84A50CD
:101B2800ADF83CA006F014FAD9F8182042F00802E3
:101B3800C9F81820D9F8442042F40042C9F84420D2
:101B4800DBF8142042EA0A02CBF81420ABF57D6BCF
:101B5800584606F070F91AA806F042F9049BADF849
:101B680074308023714A1F934FF48073DDF814C0DA
:101B78001A921AA91022209358464FF40053CDF810
:101B88006CC01C9223931E9521952295249506F0EE
:101B980034F9D9F80C3043F40073C9F80C30DBF889
:101BA800003043F00203CBF800300BA80D238DF86A
:101BB8002C308DF82DA08DF82E508DF82FA00FF019
:101BC80071FF29465A4B1A685A4B43F821200131B4
:101BD8002029F7D102F0E0FE02F0DEFE3B685A054C
:101BE80055D5554BD4F8F894C3F8009004200AF062
:101BF800D3FE0421C4F8FC040AF0AAFE4F4B84F873
:101C080000050820C3F800900AF0C6FE4C4B4D4D65
:101C1800186008210AF09CFE002184F801052C2296
:101C2800284613F020FF8E236B704FF07C0BE023C7
:101C38004FF07D0AEB7085F800B085F82BA0424D77
:101C48002C220021284613F00EFF8A236B701020E7
:101C5800A023EB7085F800B085F82BA0C4F8049594
:101C68000AF09AFE1021C4F808050AF071FE84F8FB
:101C78000C052020C4F810950AF08EFE2021C4F827
:101C880014050AF065FE84F8180509F097FB3B680F
:101C98002E4A13F4002318BF012313700AF092FF91
:101CA8002B4B18607379052B02BF2A4B4FF4C8726F
:101CB8001A80294B4FF47A721A80284BC8221A804E
:101CC800274A137843F008031370264A137823F041
:101CD800020313703A6840F6020313406BB1224BBB
:101CE80022491960224B03211970224B01211970D6
:101CF800214900230B8021490B80930341BF204BCE
:101D080004221A71DA7848BF42F0010242E000BFAB
:101D1800547E010878170020AC110020980F00208D
:101D2800B81F002050270020BC1700203444014071
:101D3800187E01080A0E002060120020B812002048
:101D48000413002088120020BD120020042D00205A
:101D58008C0E0020E4200020BE2F0020B82F002089
:101D680070120020C22F002058120020A826002040
:101D7800BC120020FC000020381000203A1000207F
:101D88007C170020090E00204503002000100240A7
:101D98000044014048BFDA70B3683B60244B01221D
:101DA8001A7098F8003063F07F0388F800302FB07D
:101DB800BDEC028BBDE8F08F0425FFF759BABAF1E4
:101DC800010F7FF6FBAA9A46FFF794BA1BB207EEFB
:101DD800903ADFED186AB8F95E31174AF8EEE77AFB
:101DE80007EE103A67EEA67AB8F96031CDED1A7AA7
:101DF80007EE903AB8EEC77AF8EEE77A002127EEB8
:101E0800267A67EEA67A11701AA80C498DED1B7A0E
:101E1800CDED1C7A07F054FCFFF74EB8BAF1010F6C
:101E28007FF6CCAA4FF0000A3070FFF76EBA00BFF9
:101E3800080E002035FA8E3C38000020C815002016
:101E4800864A2DE9F04F1368854C03F59C432033EF
:101E58002DED028B2360A3880133A380814B196881
:101E680089B011F4804F0592019305D110F084FDDB
:101E780010B9237B0133237300277B4BDFF80082E3
:101E88001E78FDB2AE4230D9D8F800307648072D1A
:101E980098BF595D754B88BF29461B689847032D25
:101EA8001ED8D8F8002005F10E0302EB83039988A9
:101EB800DA88A8B14FF47A73401A5843531A90FB42
:101EC800F3F040F6C90300F57A70984205DC40F259
:101ED800EE239842B8BF184601E040F6CA0080B227
:101EE80004EB45050137E881C7E70F23277B84F812
:101EF8003230032594F83330B7FBF5F505EB45058B
:101F08007D1B029394F834300393D8F800A0DFF8CF
:101F180078B1EBB204930025B54255DA5449029BD7
:101F280031F815904FEA450853B910F025FD28B14E
:101F3800039B002B08BF4FF0000901E0DDF8089073
:101F4800BAF81400484503D8BAF8160048450ED226
:101F5800E8B210F0E7FC032D8146DFBF94F832E0C9
:101F68000120A8402EEA0000D8BF84F8320010F003
:101F780003FD18B13F4828F8009021E0049B94F82D
:101F88007E002BF8139028B9022F15D93449012067
:101F980081F87E00BBF80210BBF800000844BBF8CB
:101FA80004100844344980B228F8010000B2032123
:101FB80090FBF1F080B200E048462E4928F8010075
:101FC80001350BF1060BA7E794F83250244BA5F125
:101FD8000F077D427D4184F898503DB19A8811B22F
:101FE8001429CCBF143A00229A800BE083F83350AE
:101FF800B54207DAE8B210F095FC1E4B23F815003D
:102008000135F5E7019B1B68D80405D51B4B1B68F8
:10201800D90701D410F080F9059B1968184B186886
:10202800837A9BB3013B134D027B35F813301AB109
:10203800C3F53B6308339BB21BB2A3F57A73B3F5C0
:102048007A7FA8BF4FF47A7323EAE37307EE903AD6
:102058009FED0C7AF8EEE77A51E000BFA02F002040
:10206800900E0020CC2400203C230020F400002007
:102078009E0E002008250020100F0020701100205F
:102088008C2F002000007A44C60E0020019A1268A6
:10209800120440D5D4F89C20AD4E8A1A002A3ADBA7
:1020A80001F59C422032C6F89C20AA4AC07A55798C
:1020B800A94A32F8152096F8A050013592B292FB41
:1020C800F0F205F00F0086F8A000304480F8A12057
:1020D8001A46A248185C01330244102B92B2F8D178
:1020E80012B292FBF3F31BB2642BA8BF642323EA5A
:1020F800E37307EE903A9FED9A7AF8EEE77AC7EE27
:10210800877A984A9FED987A67EE877AFCEEE77AA5
:1021180017EE903A1380019B944D1B68DFF870828C
:1021280013F4807F7AD0924B994204D9237A13B959
:10213800874B01221A72B4F904E098F80060844BC6
:10214800BEF1140FCCBF4FF0000E4FF0010EC6F3D6
:102158008006BEF1000F03D000279F725F7200E077
:102168000327A07AD4F8B4B0D4F8B8C0B4F904906E
:10217800617AE3882A88032848D8DFE800F0020E4D
:102188001B35BEF1000F02D02A8000222AE0002E63
:1021980040F05D862A80A6723AE09CF8000000EBC9
:1021A8008000814502DC2A8001221BE001206EB3F9
:1021B80000F0DABE3EB1BBF80E206A80AA80BCF8F7
:1021C8000200E88002279CF800A09CF80100504417
:1021D80000EB8000814500F33D86002E00F03A8632
:1021E8002A800222A27213E02A800322A27261725C
:1021F800E3807EB198F8003043F0020388F800309D
:10220800534B00225A7210F087F803E02A80A0721C
:102218006172E38017B138460AF09AFC554EB6F859
:1022280052010FF0D4FE834668B910F0BFFA524B42
:10223800C3F800B0C3F804B0C3F808B04F4B00228D
:102248001A605A609A6098F800305F0736D5019B8B
:102258001B68D80632D54A4B1B78D9062ED4494B71
:102268001B7893B196F8DE31BBF1000F15D17BB125
:10227800454B1A68D4F8BC309B1A002B08DA10F0CA
:102288004BF8334B83F8C0B018E0BBF1000F0DD109
:1022980010200AF05DFC01230EE03BB13A4A1268B7
:1022A8004FF47A7101FB0323C4F8BC3094F8C030B2
:1022B80023B10AF03BFC002384F8C030002396F8D1
:1022C800DCA196F8DD11B6F89A71B6F89CE11846CB
:1022D80035F913208008BA42C4BF60F07F00C0B24D
:1022E80001337245B8BF40F04000042BF0D194F898
:1022F800C130174A834205D192F8C230F92B04D86D
:10230800013300E0002382F8C2301E4A84F8C1007D
:1023180010780F4B1D4F914600283ED13A68D207DE
:1023280009D5BBF1000F38D198F80030DB0734D558
:102338000FF066FE31E098F8002050072DD593F88D
:10234800332052B35B7A43BB21B30FF0E5FF24E09F
:10235800900E0020EC150020FC150020310F002005
:102368000000C842CC11002000C07F44082500208E
:10237800404B4C002C25002000200020D8160020BF
:102388007012002003000020F024002070110020AB
:10239800C22F0020BBF1000FD7D094F8C2307C4A7E
:1023A800DFF81CB2142B40F0928099F800301AF133
:1023B800000A18BF4FF0010A7BB392F8C1305F2BB7
:1023C80012D198F8003003F0040303F0FF0113B1B1
:1023D8000FF0A2FF08E00B20039102920AF0B8FB6D
:1023E800029A039982F8C210BAF1000F15D094F836
:1023F800C1307D2B11D198F8003003F0040303F0AD
:10240800FF0213B10FF088FF07E00B2002920AF0D9
:102418009FFB5F4B029A83F8C22098F8003003F0C4
:10242800040303F0FF01002B51D194F8C130584A3E
:10243800572B16D1574B4FF47A721A80019B1B68A1
:10244800190601D505F07AF9534B1B685A0742BFA4
:10245800524A0A21118013F0080338D1504A1380D8
:1024680035E001980068400716D55A2B14D14D4B1A
:10247800187820B119704C4B01221A7027E092F895
:10248800C33083F0010382F8C3300BB10C2000E0A5
:102498000D200AF05DFB1AE05D2B00F0DE845B2B5B
:1024A80000F0FC845E2B02D1032000F0F8BC562B10
:1024B80003D1029307F048FC029B99F80020002AF8
:1024C80000F002856F2B40F0F9840FF099FD019B15
:1024D8001B68580733D594F8C330A3B198F8003077
:1024E800590710D5B5F90620B6F89A319A420ADD8F
:1024F8003B6813F0010301BF2C4A32211180244AA2
:1025080008BF82F8C3303B68DA030AD5284B1A782B
:102518002AB9244A127812B9244A32211180012298
:102528000CE0204A137853B198F8003003F0040304
:1025380003F0FF011BB91C4B117001221A70DBF864
:10254800009000233B6009F17B0609F1CB0A327841
:10255800737816F8010C9A420BD231460AF086FAC3
:1025680038B116F8022C012303FA02F23B68134330
:102578003B6004365645EAD10E4B1B7813B30E4D1B
:10258800054F2B680D4E13F0020F40F042833AE3DB
:10259800900E0020BE2F00206C120020B82F0020C3
:1025A800481200201121002012210020F8200020CC
:1025B80010210020C32F00207011002034130020A8
:1025C800AC11002009F1CA0609F5897732787378C9
:1025D80016F8010C9A4225D231460AF047FA08B398
:1025E800B37896F804E0C04A96F80390BF480C21E7
:1025F800013B01FB0E4103EB43031344D1F8C82010
:102608009A420FD0C1F8C830002390F8F420C1F8DE
:10261800CC30012303FA0EF322EA030381F8C490B5
:1026280080F8F4300636BE42D0D1B14BDFF8CCB2D8
:102638001E68B04B1B68039394F83330049300234F
:102648000293DBF80030002B00F0D48293F800905E
:10265800B9F1000F00F0CE82DBF8042003998A1A42
:10266800002A0CDB01F5FA720299CBF8042001224A
:102678008A4094F8F41021EA020284F8F420049ABB
:10268800002A00F0B7821BF8042C59780432D2B221
:10269800002940F0718235F91210974A934FB2F829
:1026A800982102F1C800814202DD93F802A015E0EA
:1026B800C83A914203DA9978C1F1000A0EE0029A09
:1026C8000123934097F8F42022EA030387F8F430B3
:1026D800039B03F5FA73CBF804308BE297F8F430D8
:1026E800029A1341DB0700F18582BAF1000FCCBFD3
:1026F800022001200AF04EFA09F1FF33132B00F2F1
:102708007082DFE813F0140021002F0043005C0002
:102718006300CA004001A701D70107026E02430007
:1027280052006300CA0040019A001201770137780D
:102738005744FA2FA8BFFA2727EAE77730463770B9
:102748000AF07AF901200BE077785744642FA8BF84
:10275800642727EAE777304677700AF06DF9022098
:102768003946D4E196F80390D144B9F1640FA8BF73
:102778004FF0640929EAE97986F803903046D7F8DA
:10278800F8100AF00FF903204946C0E17179514465
:102798006429A8BF642121EAE17171710D200AF052
:1027A800B1F9B9F10D0F00F01C8231795144642957
:1027B800A8BF642121EAE17131710E20A7E1B17946
:1027C800514481F30801B1710520A0E1D7F8FC302C
:1027D8001A78022A22D107EE90AAF8EEE77AB2EE2A
:1027E800040A87EE800AD3ED097A30EE270AB5EE9F
:1027F800C00AF1EE10FA09D4DFED427AB4EE670AA6
:10280800F1EE10FAC8BFB0EE670A01E09FED3E0A8C
:1028180083ED090A0F200AF060F90AE0997851441B
:10282800C829A8BFC82121EAE17199700F200AF0D0
:1028380069F9B9F10F0F00F0D481D7F8FC301A7894
:10284800022A20D107EE90AAB8EEE78AB2EE040A6F
:1028580088EE008A93ED080A38EE000AB5EEC00A41
:10286800F1EE10FA09D4DFED277AB4EE670AF1EE3B
:1028780010FAC8BFB0EE670A01E09FED230A83EDA6
:10288800080A12206BE159785144C829A8BFC82109
:1028980021EAE1715970122039E1D7F8FC301A7831
:1028A800022A33D107EE90AAB8EEE70ADFED157ACF
:1028B80093ED0C7A80EE270A30EE070AB5EEC00ACF
:1028C800F1EE10FA07D4B4EE670AF1EE10FAC8BFB9
:1028D800B0EE670A01E09FED0C0A83ED0C0A1020A8
:1028E8000AF0FBF81DE000BF40820108900E0020AE
:1028F800D0110020F02400202C250020580F0020A3
:1029080000007A440000C84200000000197B5144CE
:10291800C829A8BFC82121EAE171197310200AF05B
:10292800F1F8B9F1100F00F05C81D7F8FC301A7893
:10293800022A1ED107EE90AAB8EEE78A5FED0F7A59
:1029480093ED0B0A88EE278A38EE000AB5EEC00A26
:10295800F1EE10FA07D4B4EE670AF1EE10FAC8BF28
:10296800B0EE670A01E01FED180A83ED0B0A132089
:10297800F5E0D97A5144C829A8BFC82121EAE171F4
:10298800D9721320C3E0D7F8FC301A78022A22D172
:1029980007EE90AA1FED260AF8EEE77A87EE800A7E
:1029A800D3ED0F7A30EE270AB5EEC00AF1EE10FA31
:1029B80009D45FED2C7AB4EE670AF1EE10FAC8BFBD
:1029C800B0EE670A01E01FED300A83ED0F0A11200F
:1029D8000AF083F80AE0997D5144C829A8BFC821A4
:1029E80021EAE171997511200AF08CF8B9F1110FFB
:1029F80000F0F780D7F8FC301A78022A20D107EEC9
:102A080090AA1FED410AB8EEE78A88EE008A93ED96
:102A18000E0A38EE000AB5EEC00AF1EE10FA09D433
:102A28005FED487AB4EE670AF1EE10FAC8BFB0EE6F
:102A3800670A01E01FED4C0A83ED0E0A14208EE0B0
:102A4800597D5144C829A8BFC82121EAE1715975A7
:102A580014205CE0D7F8FC301A78022A20D107EE5F
:102A680090AAB8EEE78AB2EE040A88EE008A93EDDF
:102A78000A0A38EE000AB5EEC00AF1EE10FA09D4D7
:102A88005FED607AB4EE670AF1EE10FAC8BFB0EEF7
:102A9800670A01E01FED640A83ED0A0A09205EE077
:102AA800D9785144C829A8BFC82121EAE171D97051
:102AB80009202CE0D7F8FC301A78022A1ED107EE3C
:102AC80090AAB8EEE78A5FED717A93ED0D0A88EE69
:102AD800278A38EE000AB5EEC00AF1EE10FA07D4DC
:102AE800B4EE670AF1EE10FAC8BFB0EE670A01E06B
:102AF8001FED7B0A83ED0D0A0A2030E0597B514413
:102B0800C829A8BFC82121EAE17159730A2009F030
:102B1800F9FF66E0D7F8FC301A78022A22D107EECE
:102B280090AA1FED890AB8EEE78A88EE008A93ED2D
:102B3800100A38EE000AB5EEC00AF1EE10FA09D410
:102B48005FED907AB4EE670AF1EE10FAC8BFB0EE06
:102B5800670A01E01FED940A83ED100A0B2009F0C3
:102B6800BCFF3EE0D97D5144C829A8BFC82121EA4D
:102B7800E171D9750B20CAE7012932D1987835F966
:102B88001230B3F5617F05DB40F633029342A8BFEC
:102B9800134601E04FF46173B9F10C0F21D14FF4E2
:102BA800966292FBF0F0AE4AA3F5617393FBF0F3E3
:102BB800DFB21378BB4214D0042F34BF3B46022344
:102BC8001370A84A09FB0323A74A0633136006F0CB
:102BD800FBFE4846394609F095FF781CC0B209F05B
:102BE800D9FFA249029A0123934091F8F420134394
:102BF80081F8F430029B0133042B02930BF10C0B88
:102C08007FF41FADBBE4019B1B68D8050ED5637A22
:102C180063B13B68990709D5338813F001090AD1D4
:102C28000FF0C4FD012006F0F7FD04E0012006F0D6
:102C3800E2FD012300E000232A6852070CD55BB1AE
:102C4800012006F0D8FD3388980708D40FF0AEFDB0
:102C5800022006F0E1FD02E0022006F0CCFD3388F8
:102C6800834A13F0030F4FF020010CBF91611185C7
:102C78003A6812F00A0F23D02A68D10609D55A07F4
:102C88000AD4042006F0C8FD7A4B1B88A4F800314A
:102C980002E0042006F0AFFD2B689B0606D53388BA
:102CA800580606D4402006F0B7FD02E0402006F0A2
:102CB800A2FD2B68590642BF6E4B1B88A4F802314F
:102CC8003B689A0608D42B681B0540F18C804FF4AA
:102CD800807006F0A1FD8AE0674B1B789F074FD5EF
:102CE800664B1B78042B4BD92B68604F13F4007983
:102CF8000ED03388DC0637D4102006F08DFD202056
:102D080006F079FD5E48011D04F06CFC022327E003
:102D1800348804F01004A4B22CB1102006F06BFD26
:102D2800012487F804912B68580512D5D7F8083183
:102D380054495A89B1F90030002BB8BF5B4293421D
:102D480007DAB1F90230002BB8BF5B429342C0F2F8
:102D580011813388990608D5202006F04CFD002300
:102D680087F80431012400E0002497F80C31B3B946
:102D78000E2009F0EDFE3D4B012283F80C210EE0F8
:102D8800338803F03003002B9DD0102006F033FD6C
:102D9800202006F030FD002384F8043101E0002CE7
:102DA80091D0394B002003F1280603F15004374A2B
:102DB800002122F81010364A596022F81010043207
:102DC800716022F8101000221A609A603260B260B6
:102DD80022606160A26014331436143400287FF432
:102DE80072AF0120E3E74FF4807006F004FD294B31
:102DF8005A79082A1C4601D00E2A02D1402006F032
:102E0800FAFC019B1B685A0540F1C98094F81432FA
:102E180023B998F8003013F0040F02E02B6813F47C
:102E2800002F0BD01C4B00221A703C200DF026FB03
:102E3800002800F0B4800DF071FCF6E708F0BEFA47
:102E480009B0BDEC028BBDE8F04F0DF030BA01209F
:102E5800FFF791B90320FFF78EB901201FE000BFEB
:102E680078230020D42C0020D0110020900E0020C0
:102E7800000400484812002070120020761200203A
:102E8800D811002050120020A00F0020BA2F0020D7
:102E9800181000202C2500204123002002205FFA72
:102EA80080F909F1FF3386F8AC3706F0F7FC06F035
:102EB800AFFD484609F06EFEFFF709BBBAF1000FF7
:102EC80002D07E2B3FF401AB972B05D1364B4FF444
:102ED800C8721A80FFF7FBBAA72B06D1334A1378BA
:102EE80043F004031370FFF7F2BA0022BB2B0792DA
:102EF80001D1022303E0B72B04D14FF6FE73ADF8DE
:102F08001E3009E0BE2B01D1022303E0BD2B1AD1EC
:102F18004FF6FE73ADF81C30DBF80030BDF81C101E
:102F2800B3F858200A44A3F85820BDF81E10B3F887
:102F38005A200A44A3F85A2006F006FF002384F812
:102F4800C230FFF7C4BA792B04D1194AD37823F0D9
:102F5800010306E07A2B7FF4BAAA154AD37843F026
:102F68000103D370FFF7B3BA013301469BB20220C5
:102F7800FFF701B933889B063FF5F7AE202006F02E
:102F88004BFC0C480C4B011D1A685B6843600260DF
:102F980004F028FB094B012483F80441E5E609B055
:102FA800BDEC028BBDE8F08FE420002070120020F9
:102FB8007C170020E011002078120020900E0020DD
:102FC8002DE9F04FC14BB3F90610C14B2DED028B23
:102FD8001F687A8985B0914201930EDBB1F5FA6FCB
:102FE800FC79BDBF8B1A6343A2F5FA64C4F164048B
:102FF800BCBF93FBF4F4643400E06424B54BB64AD8
:10300800B3F898B193F96231126802929BB21546EF
:1030180003930022AD4B33F912E0CBEB0E0303F21E
:10302800F31640F2E63086424FEA420C03D8002BF2
:10303800B8BF5B4201E04FF4FA73022A2ED0029E19
:1030480096F811611EB1B342CCBF9B1B0023A34E5F
:103058006FF0630A642093FBF0F836F818900AFBC7
:10306800083A08F1010836F918600FFA89F8C8EB30
:10307800060606FB0AF696FBF0F699484E4420F839
:103088000C60BE18642036797343964E93FBF6F3B2
:1030980064339BB2634393FBF0F02DE0029890F801
:1030A80012611EB1B342CCBF9B1B0023DFF86092B4
:1030B8006FF06308642093FBF0F008FB003A39F9DD
:1030C80010600130002B39F91000A0EB060000FB5E
:1030D8000AFABDF80C009AFBF8FAC6EB0A0A1AFBC2
:1030E80000FA7F48A0F804A0B879B8BF5B42434310
:1030F8007C4893FBF0F064306B787B4E4FF06408AB
:10310800434393FBF8F3B354784EEB7A434393FB72
:10311800F8F3B3546B7D724E5843754B90FBF8F03F
:10312800022A9854734B0ED1DE4583F802800DDBDA
:10313800684CB4F89A21914214DBB1F5FA6FA8BF34
:103148004FF4FA610FE0DE459C5404DA36F80C308F
:103158005B4226F80C300132032A05F101057FF4A1
:1031680059AFE5E71146DFF8BCE15D4D891A4FF428
:103178007A736FF063075943C2F5FA626423B1FBAF
:10318800F2F191FBF3F23EF8120007FB0211013253
:1031980007B23EF91220D21B514391FBF3F30344CB
:1031A800F380554B1B885F0635D5544B544A1B8812
:1031B8001288DFED547A9B1A1BB208EE103AB8EE6B
:1031C800C88A28EE278AB0EE480A06F071FAF0EEAF
:1031D800408AB0EE480A06F008FAB5F9023006EE61
:1031E800903AB5F90030F8EEE66A07EE903A20EE2C
:1031F800667AF8EEE77AA7EEA87A67EE807ABDEEEF
:10320800C77AE6EEA87A17EE103AFDEEE77A2B8039
:1032180017EE903A6B803C4D2B68980740F1A180DF
:103228003A4B3B4F1A687B6945F20721D31A8B4208
:1032380040F397807A6105F04DF9364BDFF8E89056
:103248001A78032A9846B9F8003022D10A2B2AD9CD
:103258000023282088F8003009F0DBFC05F03AF953
:103268002D4B188805F020F92C4B1A68D37890FB61
:10327800F3F0013008282A4BA8BF082018705379AA
:1032880080B213FB00F33B83137913FB00F07883C0
:1032980009E00A2B07D80323214A88F800300023C5
:1032A80013703B837B8398F800301A4A012B3DD07A
:1032B80002D3022B4CD054E03A8BB9F800309A4232
:1032C8004FDD012388F8003040E000BF08250020CA
:1032D800D01100202C250020AC110020DE17002082
:1032E800501200200CFEFFFFEC1600202E100020CC
:1032F800EF160020E01F00203413002048120020A1
:10330800920F002035FA8E3CCC240020A02F0020FC
:1033180020100020BC1200200416002058120020A3
:10332800FC000020C61700205C120020B9F800102D
:103338007B8B8B4202DD022313700FE09C4B1B8BAF
:103348000133994202DD002313700AE0082006E0E9
:103358007B8BB9F8002001339A42B2DC072009F0D0
:10336800F7FB2D68290575D5924B914F1A68FB69B3
:10337800C3EB020845F2072398456BDDB6F9063022
:10338800FA61A3F57A7B8C4BB4F85201D3F800901C
:103398008A4E99F80A30012B4FF47A7198FBF1F8AC
:1033A80003D040D3022B1FD03FE0854B386A5A7BAD
:1033B800844B33F812204FF0080E92B290FBFEF3C4
:1033C800C01A8318BA843B6240F6E44293FBFEF3CA
:1033D8009BB25343B9F80820C2EB13334B43B9F9F6
:1033E800062093FBF2F31FE0774BB9F808A01B788F
:1033F800C6F800A05A0718D50EF0E9FD20B915F057
:10340800100F18BF4FF0000BB9F906200BFB0BF19A
:10341800322391FBF3F35B445A434FF47A7392FBE4
:10342800F3F3534400E000233360D7E90A0133681B
:10343800664A03FB08F84FF47A7398FBF3F810EB2D
:10344800080041EBE8710023C7E90A010FF0E0FA30
:103458005F4B18605F4E3368DB0427D52F0622D5F3
:103468005D4B1B789D071ED55C4B187804281AD92C
:1034780000225B4BD7180521951C4FF00A0E122A23
:10348800D154E9B287F801E004D0B0EB510F2A46D5
:10349800EFD800E014215A18322002F8010CFF225C
:1034A8005A540F2000E00A2009F052FB4D4D2A68BB
:1034B800002A44D04C4B4D4F1868396881429846D1
:1034C8003DD84B4BDFF8349118785168B0B90122D8
:1034D8001A70B9F80030CB5CD3B1464B1A700FF0B4
:1034E80057FAB9F800309BB92B681B78053B012BBC
:1034F8000ED809F067FB404B186009E000221A70EB
:10350800B9F80030CB5C1BB13A4B1A700FF040FA97
:103518002A68B9F8003052683848D25CFE2A01D1CE
:1035280000230BE0FF2A02D109F000FB07E0D8F8DE
:1035380000500A2111FB02523A6001330380224DE8
:103548002B78580703D52E4B10221A8570E0326865
:10355800D1075CBF43F001032B701F4B1B781F077B
:103568005EBF2B7823F001032B70D60248BF2B785F
:10357800204A44BF23F001032B70224B1B6813F031
:10358800040F02D02049098851B92049098809B196
:10359800980705D41E4B1B88003318BF0123CBB3F3
:1035A800022313702B7823F001032B7037E000BF40
:1035B80020100020A02F00205812002064120020A4
:1035C800EC150020FC150020C22F0020407E0500CD
:1035D800681200207011002070120020761200205E
:1035E800A4230020F8170020F0240020F017002062
:1035F800EC170020902F0020A82E0020F4170020A0
:10360800000400486C120020B82F0020E42000209D
:10361800BE2F00202978C90758BF0223137009F06C
:10362800D1FAAF4B1B68C01A002801DB0FF0B0F9C4
:1036380007F0C4FEAB4B1E789846002E00F0A98018
:10364800A94E3368002B00F0D286306809F071FC6F
:10365800002800F0CC86A44BA44C186809F066FC3E
:10366800092801D03F2850D14FF0000AD4F8009023
:103678009F4D5746B9F1000F05D09E4829684A4624
:1036880012F03EFA10B9AA4607B92F469A4B1035E0
:103698009D42EFD3C7B1D7F800E0DAF800C023683D
:1036A8001EF803501CF80300A8420DD15A1C91497A
:1036B80038B92D2B05D88D4D2A602025CD54885436
:1036C80002E0CD542260EAE723680BB1574511D0D8
:1036D8008A480DF017F9574507D857F8100B0DF021
:1036E80011F909200DF006F9F5E785480DF00AF9FA
:1036F8004FF0000923689945A7D27E4B13F80900BB
:103708000DF0F8F809F10109F4E72368002B40F0FF
:103718005286042840F09486764808F073FC00F03E
:1037280066BED9F80000DFF8E8A109F002FC30B362
:10373800DAF8000009F0FAFBDBF8003093F84810DB
:103748000246002933D124286AD1012283F848206F
:10375800DBF80030DFF8B4A193F84820062AE0D15E
:1037680093F8490001F0F6FB834600287BD03B68BC
:1037780098790DF010F83B68002283F84820614BD7
:1037880093F83530002B40F004864C36982E00F024
:103798002E865D4BF21892F84A100129F5D15B4F3D
:1037A800F3583A605A4ABB4613609146B9E7012973
:1037B80004D14D2814BF00220222C7E7022904D1F0
:1037C8003C2814BF00220322C0E703290CD140285B
:1037D8004FF0000102D983F84810B9E75871197100
:1037E800D97198710422B1E7042906D1997983F82F
:1037F80049004A409A710522A8E70529A8D15879B5
:1038080019798842987906D950409871481C1871DE
:103818000B441A729CE790420CBF0622002295E7DF
:103828002B78580794D4232ADAF800300ED10121D6
:1038380088F800102C4937480B60324902920B6314
:103848000DF060F82E480DF05DF8029A324B1B68B7
:103858001B78934201BF314B314A1A60314B04BF88
:10386800314ADA6074E7DAF8002092F849304C2BD4
:1038780000F0968400F28580332B00F0CC8421D8A8
:10388800292B00F0598409D8252B00F01384272B05
:1038980000F01784232B40F0CF8539E22D2B00F060
:1038A8005C8407D82B2B40F0C7850CF057FF60715C
:1038B80000F06ABD2F2B00F01A85312B00F02C8503
:1038C80000F0BABD3E2B00F0198144D8372B00F028
:1038D800D6842BD8352B00F06F8200F0ADBD00BF29
:1038E800942F0020C32F002094230020B817002015
:1038F8006C840108881700201C8601086AA4010846
:103908006FA4010820100020A0220020141300201A
:10391800181300209FA4010844230020FC9F0020C6
:10392800EFBEADDE00ED00E00400FA05392B00F033
:10393800D5833C2B40F08085DFF84C94D9F800A063
:103948000CF00CFF8AF80000D9F8003018780BF05A
:103958002DFE00F019BD432B00F06E8406D8412BD4
:1039680040F06A854FF0000900F05ABC442B00F083
:1039780007854A2B40F060850CF0FAFEA08100F024
:1039880003BDD02B00F00F8355D8CA2B00F0C080A0
:1039980009D8C82B00F0858000F226834E2B00F052
:1039A8000C8400F049BDCD2B00F0088304D8CC2B43
:1039B80000F02A8200F040BDCE2B00F00883CF2B08
:1039C80040F03A850CF0D4FE6FF4AF6283189BB2D6
:1039D800C62B98BFA4F898010CF0CAFEA4F84401BD
:1039E8000CF0C6FEA4F846010CF0C2FEA4F848018B
:1039F8000CF0BEFEA4F8DA010CF0B0FE84F8EB017E
:103A08000CF0ACFE0CF0AAFE84F8EC010CF0A6FE5B
:103A180084F887010CF0A2FE84F894010CF09EFE55
:103A2800D94BD3F800900CF0A3FE00EB80004000C7
:103A3800A9F8560052E3D62B00F039820AD8D22BC7
:103A480019D0C0F0F882D32B25D0D42B00F03B82BC
:103A580000F0F2BCEF2B41D005D8D82B40F0EC8415
:103A68004FF0000AE6E0F22B00F07582FA2B00F026
:103A7800B78200F0E1BC2B78590700F185840CF07F
:103A88006DFE022884F8AC0740F29382BF4B0022F7
:103A980083F8AC278DE20CF06BFEBD4B188000F06C
:103AA80073BC92F805904FEA5909B9F1120F03D97E
:103AB8000CF0E0FC00F068BC4FF0000ACA4507D2E1
:103AC8000CF056FEB34B23F81A000AF1010AF5E789
:103AD800B14B012283F8342000F056BCDFF8A892DD
:103AE800D9F800A00CF044FEAAF85A00D9F80090C2
:103AF8000CF03EFEA9F8580000F046BC0CF02EFE73
:103B080084F8DE010CF02AFE84F8DD0100F03CBCEC
:103B18009D4B1A681278022A824699466FD1D9F8C5
:103B280000B00CF01BFE07EE900AF8EE677AB2EED2
:103B3800048AC7EE887A0BEB8A0BCBED087AD9F8A2
:103B480000B00CF00BFE07EE900A9FED947AF8EEA9
:103B5800677A0BEB8A0BC7EE877ACBED0B7AD9F82D
:103B680000B00CF0FBFD07EE900A9FED8D7AF8EEA1
:103B7800677A0BEB8A0BC7EE877A0AF1010ABAF16A
:103B8800030FCBED0E7ACAD1BAF1070FD9F800B0FE
:103B98001CD10CF0E3FD07EE900AF8EE677AC7EE49
:103BA800887ACBED117AD9F800B00CF0D7FD07EE82
:103BB800900AF8EE677AC7EE887ACBED127AD9F8D0
:103BC80000B00CF0CBFD8BF84C0012E00CF0C6FDF9
:103BD800D3448BF80100D9F800B00CF0BFFDD344F2
:103BE8008BF80B00D9F800B00CF0B8FDD3448BF873
:103BF80015000AF1010ABAF10A0FC5D1C4E3D9F8D0
:103C080000B00CF0ABFDD3448BF80100D9F800B03C
:103C18000CF0A4FDD3448BF80B00D9F800B00CF0DD
:103C28009DFDD3440AF1010ABAF10A0F8BF8150079
:103C3800E5D1A9E3DFF850919FED598AD9F800B092
:103C48000CF096FD07EE900AF8EE677A0BEB8A0BFC
:103C5800C7EE887ACBED087AD9F800B00CF088FD69
:103C680007EE900AF8EE677A0BEB8A0BC7EE887AB4
:103C7800CBED0B7AD9F800B00CF07AFD07EE900A7C
:103C8800F8EE677A0BEB8A0BC7EE887A0AF1010A1D
:103C9800BAF1030FCBED0E7ACCD1BAF1070FD9F8F0
:103CA80000B01CD10CF064FD07EE900AF8EE677ABC
:103CB800C7EE887ACBED117AD9F800B00CF058FD30
:103CC80007EE900AF8EE677AC7EE887ACBED127A9B
:103CD800D9F800B00CF04CFD8BF84C0012E00CF059
:103CE80047FDD3448BF80100D9F800B00CF040FD33
:103CF800D3448BF80B00D9F800B00CF039FDD3444D
:103D08008BF815000AF1010ABAF10A0FC5D13BE395
:103D18000CF024FD132883463FF6CAAEDFF868A0EE
:103D2800DAF800900CF01AFD00231E4A0C2101FB62
:103D38000322117A814222D10FFA8BFB09EB8B09FE
:103D4800137889F879300CF009FD89F87A000CF0BD
:103D580005FD89F87B000CF001FD134B134A1A602E
:103D680089F87C00124BDAF80000186000217930DD
:103D780008F0A2FE0F4B80F00100187004E3013335
:103D88001B2BD2D194E600BFAC1100202C250020BB
:103D9800900F002008250020201000200000C842B5
:103DA80000007A44AC820108880F002070260020A9
:103DB8008C0F0020030000200CF0D0FC0B2882465A
:103DC8003FF676AECE4BD3F800900CF0C7FC032834
:103DD8003FF66EAE062303FB0A9989F8CE000CF075
:103DE800BDFC89F8C9000CF0B9FC89F8CA000CF0D0
:103DF800B5FC89F8CB000CF0B1FC89F8CC000CF0CC
:103E0800ADFC89F8CD00BFE25379092B7FF650AE9F
:103E1800019BD3F800900CF0A1FC019B89F80000ED
:103E2800D3F800900CF09AFC89F801000CF096FC8D
:103E3800019B64281B68A8BF642018710CF08EFCD5
:103E4800019B64281B68A8BF642058710CF086FC8D
:103E5800019BFF281B68A8BFFF2098710CF07EFC0F
:103E6800019B6428D3F8009028BF642089F80700D4
:103E78000CF074FC019B89F80200D3F800900CF058
:103E88006DFC019B89F80300D3F800900CF070FCDE
:103E98003B68A9F80A005B790A2B40F27582994BB6
:103EA800D3F800900CF05AFC89F808006CE28246BE
:103EB8000CF05EFC944B23F81A000AF1010ABAF1DF
:103EC800080FF5D160E253790F2B7FF4F1AD0CF0B8
:103ED80045FC072881463FF6EBADDFF824A2DAF867
:103EE80000B00CF045FC0E2303FB09F9CB44ABF8FA
:103EF8001901DAF800B00CF03BFCCB44ABF81B011D
:103F0800DAF800B00CF034FCCB44ABF81D01DAF859
:103F180000B00CF023FCCB448BF81F01DAF800B09A
:103F28000CF01CFCCB448BF82001DAF800B00CF044
:103F380015FCCB448BF82101DAF800B00CF00EFC2C
:103F4800CB44DAF800A08BF822010CF01BFCD1441A
:103F5800C9F8230118E20CF001FC0F2881463FF64E
:103F6800A7AD0CF0FBFBC9EBC909A14489F8D40043
:103F78000CF0F4FB89F8D5000CF0F0FB89F8D600BA
:103F88000CF0ECFB89F8D7000CF0E8FB89F8D800B6
:103F98000CF0E4FB89F8D9000CF0E0FB89F8DA00B2
:103FA80009F068F9F0E12B785B0700F1ED810DF07D
:103FB800F3F905F073FC05F02BFDE5E12B785807C4
:103FC80000F1E281514B4FF4C8721A80DCE12B7882
:103FD800590700F1D9814E4A137843F0040328E0C9
:103FE8002B785A07E5D527E20CF0B8FB484B1A782E
:103FF80010B142F0020201E022F002021A700CF045
:10400800ADFB444BDFF82C9118700CF0BBFBC9F8E2
:1040180000000CF0B7FBC9F804000CF0A9FB3E4BFC
:1040280018800CF0A5FB3D4B3D4A1880137843F0EF
:1040380002031370A8E10CF091FB02900CF0A2FBB4
:1040480083460CF09FFB82460CF09CFB81460CF0EB
:104058008FFB0CF08DFB0CF081FB029BA3B9314B5D
:104068001020C3F800B0C3F804A005F0C4FB284A28
:10407800137843F001031370B9F1000F00F0848145
:10408800294BC3F800907FE1102B40F07D81274B2E
:10409800C3F800B0C3F804A0B9F1000F02D0224B56
:1040A800C3F800902148224B0222011D1A7003F028
:1040B80099FA69E1A0600CF065FBA3681843A06059
:1040C80062E10CF055FBA4F85C010CF051FBA4F87C
:1040D8005E010CF04DFBA4F8600155E10CF03EFBCD
:1040E80084F87C010CF03AFB84F880010CF036FB74
:1040F80084F87F010CF032FB84F8810144E100BFB1
:10410800AC110020D01100207A230020E4200020E8
:104118007012002076120020741200207212002003
:10412800D6110020D8110020E8110020E01100204D
:10413800940F0020781200200CF01AFBA4F88201DA
:104148000CF016FBA4F884010CF008FB84F8860137
:104158000CF00EFBA4F8880116E10CF0FFFA84F8C5
:1041680092010CF005FBA4F89C010CF001FBA4F8EB
:1041780098010CF0FDFAA4F89A010CF0EFFADAF8BD
:10418800003084F893015B79082B40F2FD800CF035
:10419800EFFAA4F89E010CF0EBFAA4F8A001F3E002
:1041A8000CF0DCFA84F8D8010CF0D8FA84F8D901BC
:1041B8000CF0DEFAA4F8DA01E6E092F805900323A1
:1041C800B9FBF3F9B9F1120F3FF672ACDFF888A327
:1041D8004FF0000BCB4580F0D7800CF0BFFA8AF87F
:1041E800A2010CF0C5FA40F2ED23984205DD40F635
:1041F800CA039842A8BF184601E040F2EE20A0F298
:10420800EE2019230BF1010B90FBF3F00AF1020ADF
:104218008AF8A101DEE70CF0A1FA84F89401B3E072
:104228000CF09CFA04EB090309F10109B9F1080F34
:1042380083F88A01F4D1A7E00CF090FAC4F808B02A
:1042480060710CF09FFAA3681843A0600CF086FA1E
:1042580084F892010CF08CFAA4F85C010CF088FA4E
:10426800A4F85E010CF084FAA4F860010CF080FA5E
:10427800A4F882010CF07CFAA4F8840184E0537954
:104288004FF0070AB3FBFAF2C2EBC2029A1A12F015
:10429800FF0F7FF40DACB3FBFAFA0AF1FF3A5FFAAD
:1042A8008AFABAF1FF0F6FD00CF058FA5FFA80FB68
:1042B8004FFA8BF008F038FB814600283FF4F8AB42
:1042C80080F800B00CF054FAA9F802000CF046FA95
:1042D80089F804000CF042FA89F805000CF03EFA5F
:1042E80089F807000CF03AFA89F80600D5E7DFF8F4
:1042F800689209F1400A0CF03BFAA9F8A4020CF004
:104308002DFA89F8A6020CF029FA09F1040989F8AE
:10431800A302D145EFD137E00CF020FA1F288146DF
:104328003FF6C6AB3B685B79082B7FF4C1AB0CF05A
:104338001FFA09F1880904EB890900F03F00A9F880
:1043480006000CF015FAB9F80630800100F4FE50AA
:104358001843A9F806000CF001FA000189F80400D6
:104368000CF0FCF999F8043000F00F00184389F8B4
:1043780004000CF0F3F989F805000BF0ABF903E041
:10438800624B012283F8352000200CF033FAFFF746
:10439800EEB95F4B985908F0C3FD18B9322008F000
:1043A80038FCF6E708F026FF05F04EFA594B5A4A52
:1043B800DA60FFF7EAB90C2844D00A284BD1574DE8
:1043C80057480CF09FFA2846232111F082FB08B1C8
:1043D800401B20602368002B60D1504823600021D7
:1043E800302211F040FB98F80030002B2DD14D4BB6
:1043F8001B689B0615D54C4B44491B688A6B9A1A57
:10440800002A0EDB494A1278042A0AD9484A03F5D9
:10441800123303F5F8738B63938A9BB283F02003FE
:104428009382444B9B68002B6BD0434805B0BDEC8E
:10443800028BBDE8F04F18470CF01CF8FFF797B94E
:104448000C2804D13D480CF05DFA3D480DE07F286A
:1044580012D1FFF7FAB80D28B1D07F2809D1013B56
:104468002E4A384823600021D1540CF04BFAFFF74C
:10447800ECB82F2B3FF6E9A8A0F12002D2B25E2AB1
:104488003FF6E3A813B920283FF4DFA85A1C22609E
:10449800224AD0540CF02EFAFFF7D7B85A1EA95C5E
:1044A800202901D1134696E71C4A23600021D154E4
:1044B800254B264DD3F800A0D5F800B0DFF85C9066
:1044C800584611F014FB07463A464846594611F03B
:1044D80017FB1F4A28B919F8073053445B785B0764
:1044E80003D010359542E7D306E0954204D2781CF4
:1044F800EB684844984702E016480CF003FA00239A
:104508006BE705B0BDEC028BBDE8F08F20100020F2
:10451800A022002000ED00E00400FA058817002022
:104528003AB101086C120020A02F0020761200205A
:1045380000040048742000205C10002074A40108C6
:104548006FA401089BA401080C0100206C840108D9
:104558001C8601087FA401082C25002010F80A3CBD
:104568000133DBB20A2B84BF10F8131C044A00F88D
:104578000A3C82BF002322F8113000F80A3C704739
:10458800242F0020354A70B5136C90681944344BB9
:104598001B78D940081A40F68C2398429160D06065
:1045A800516013463BD9127893F945108A42104658
:1045B8000BD1111F082908D893F84610182901D8DB
:1045C800013103E083F8442002E0002183F846101B
:1045D80093F944402149A24219D191F84740B4B116
:1045E8000C310024944206DA1E4D51F8046F25F868
:1045F80014600134F6E70C2805D01A49002421F884
:1046080010400130F7E7184801780131017083F84C
:104618004520002201211A7083F8471070BD92F8D6
:104628004710C9B1A0F2EF2440F2DA518C4208D801
:1046380011780B2905D80B1D0131117042F82300A0
:1046480070BD002283F84720084B03F13002002197
:1046580043F8041F9342FAD170BD00BFA0010020A7
:104668009F010020242F00209C060020AC01002080
:10467800024A136C0133194411647047A0010020E9
:10468800024B53F820301B68196070473C18002013
:10469800064B53F820301A681B89A1F57A715943E3
:1046A8004FF47A7391FBF3F1116070473C180020C6
:1046B800054B98420CBF054A054A138801339BB243
:1046C80013800020704700BF005400406C11002088
:1046D8006E110020F0B5046D8668236823F001038D
:1046E80023608379054613F0020F40790CBF4FF021
:1046F800000E4FF4005E13F0040F14BF4FF48067F0
:10470800002710F0010F14BF04210021830720683F
:1047180020F001002060626822F440524EEA020252
:104728006260226822F4B05323F00C0348BF41F0C2
:1047380008013B430B432360A36895B023F44073FF
:10474800A360684603F042FC284B9C4201D10C9BB5
:104758000EE0274B9C4201D10D9B09E0254B9C4262
:1047680001D10E9B04E0244B9C420CBF0F9B109B75
:104778002268A879170448BF5B00B3FBF6F206FB72
:104788001233B3EB560F236828BF01321E0441BF12
:104798004FF6F073C2F34201134041EA03026B790A
:1047A80092B213F0020FA28100F0010114BF4FF47E
:1047B80000320022DC0748BF42F480322B6D11B171
:1047C80059680A4302E0596821EA02025A609A6865
:1047D80001074CBF42F0080222F008029A601A68EA
:1047E80042F001021A6015B0F0BD00BF0038014068
:1047F8000044004000480040004C00403D4B1B78FE
:10480800012B30B514BF00240324B1B9036A23F087
:10481800010303628169036A21F0F30123F00A03AB
:1048280041F0010142F001021A4341EA0411816199
:104838000262836923F00C031BE004291DD1016A7D
:104848004FF6EF730B4003628169056A120121F488
:1048580073414FF65F7342F0100241F480712B40B0
:1048680092B2134341EA043181610362836923F4FC
:10487800406383618369836130BD0829016A1AD165
:104888004FF6FF630B400362C169036A9BB289B2AA
:1048980023F4206343F4807321F0F30143EA0222F6
:1048A80041F0010192B241EA0411C1610262C26998
:1048B8004FF6F37319E04EF6FF730B400362C369BA
:1048C800056A40F6FF41194045F6FF732B4043F453
:1048D800805343EA023241F4807192B241EA0431D2
:1048E800C1610262C2694FF2FF331340C361C369F9
:1048F800C36130BD9C01002038B510F80E2C50F86B
:10490800043C044652B9012200F80E2C20F80C1C75
:10491800997A18680222BDE838406FE730F80C2C05
:1049280020F80A1C891A89B220F8081C074A10F8CE
:104938000F0C002522F8101004F80E5C1868997AFC
:104948002A46FFF75BFF04F8065C38BD242F0020D9
:10495800044B53F820301BB107289CBF1B68196013
:10496800704700BFC8020020084A13689B050BD592
:10497800074B00211970074908684FF6FE7303407A
:104988000B604FF400735360704700BF0000024093
:10499800C12F0020300002402DE9F047664D2B68FA
:1049A80066490A78581C02F0FF068E460AB103468B
:1049B800F6E72B60687BAB6895F80C80AA7B3746D6
:1049C80039B2202900F09B80DFF880C10CEB81030D
:1049D8003CF82110DC789B78C3F1FF039BB2002BD5
:1049E80065D0C3F1FF0363434FF03C0C1B12B1FBCE
:1049F800FCF9B9F1050F5DD8DFE809F0030B1A29B6
:104A08003A4AE01ADAB24143B1FBFCF01044C0B2B2
:104A180051E0B1FBFCF00CFB101189B2DAB2C1F124
:104A28003C01E31A4B432046B3FBFCFC94442CE0C6
:104A3800B1FBFCF00CFB10115FFA83F8E21A89B2A3
:104A48004A43B2FBFCF24244D2B2204632E0B1FB08
:104A5800FCF90CFB191189B25FFA83F8E01AC1F16D
:104A68003C014843B0FBFCF04044C0B2224621E080
:104A7800B1FBFCF80CFB1811D8B289B2E31A01FBA0
:104A880003F2B2FBFCFC224684445FFA8CF412E089
:104A9800B1FBFCF80CFB181189B2D8B2C1F13C018A
:104AA800E31A4B43B3FBFCF20244D2B203E02246C2
:104AB800204600E044464FEA042C4CEA004C4CEAFD
:104AC800020C172306F117014FF0010808FA03F842
:104AD800C91A18EA0C0F89B2DFF8748014BF4FF0B6
:104AE80011094FF0090913F1FF3308F80190E9D2D1
:104AF80018360137B6B2BFB2114BA04660E7AA73A9
:104B0800AB60104AE98001238EF800300E4985F821
:104B18000C8040F22A336873AE80536000234B62E6
:104B28000B889BB243F001030B80136843F0010329
:104B38001360BDE8F08700BF60100020C12F00207F
:104B48006C10002030000240004401400A0E002092
:104B58004503002073B506460D46002401232A8824
:104B6800A34013421AD0AA78009302F003038DF8E9
:104B78000430EB78022B03D0032B0CBF0323012353
:104B88008DF805303046C2F301136946C2F381023D
:104B98008DF806308DF8072003F086FB0134102CC1
:104BA800DCD102B070BD2DE9F04F734EF57B07469E
:104BB8000C4687B011469A4600686B1C91462246FF
:104BC8004FF0020BF3730CF0E9FA3B897868ADF803
:104BD800043001A98DF806B08DF807B0FFF7BAFFC9
:104BE8000023ADF80A30ADF81230ADF81630702356
:104BF8000193BA7A3C68CDF80CA0012306F110089D
:104C08002D01ADF808304FF48073A844ADF810B00A
:104C1800ADF814300C2A7ED8DFE802F0077D7D7DE0
:104C28000F7D7D7D387D7D7D5E00204601A903F0E6
:104C38008FF9A36943F0080326E0236A4F4823F05D
:104C480010032362236A6168A26922F0807222F449
:104C5800E642844242F4E04206D000F50060844215
:104C680002D043F0300307E023F0E00321F4406171
:104C780043F0300341F480616160A261C4F838A058
:104C88002362A36943F40063A36144E0236A3B48B9
:104C980023F480732362226A6168E369844223F003
:104CA800730343F0700306D000F50060844202D01D
:104CB80042F4407207E022F4606221F4405142F469
:104CC800407241F480516160E361C4F83CA0226203
:104CD800E36943F008031DE0236A284823F480535E
:104CE8002362226A6168E369844223F4E64343F459
:104CF800E04342F4405203D000F50060844201D101
:104D080041F480416160E361C4F840A02262E36934
:104D180043F40063E3613A7B3B681AB15A6C42F48E
:104D280000425A641A8892B242F001021A80BA7A92
:104D38000C2A18D8DFE802F0071717170B171717F0
:104D48000F1717171300721903F134010AE07219CB
:104D580003F1380106E0721903F13C0102E072190F
:104D680003F14001116135444046A5F818906B6184
:104D780007B0BDE8F08F00BF60100020002C014094
:104D8800F8B53A4E3A4C4000C7B24FF42045306867
:104D9800C4F8D050D0F818E01EF4004F05D0AE4645
:104DA800013DBEF1000FF5D116E0D0F804E0314D19
:104DB8000EEA050545F490353D4345604FF420451E
:104DC800C4F8D050D0F818E01EF0020F2DD1AE462E
:104DD800013DBEF1000FF5D1C4F8D0501FE02946BF
:104DE800013D0029F8D081694906F8D5C4F8D050AA
:104DF80020494568294041F0007141F4105141EAC9
:104E08000241394341604FF42041A2B130688569BD
:104E18006D071ED411F1FF31F9D2C4F8D010FFF795
:104E280047FC003018BF0120F8BD4FF420458162CF
:104E3800C4F8D050D7E73068C4F8D0100B46826960
:104E480092060CD41A46013B002AF8D1C4F8D03097
:104E5800E5E7416A03F8011B013AD2B2D3E7C4F887
:104E6800D0302023C3610120F8BD00BF68110020A5
:104E780060100020009800FC400070B5C5B23248B0
:104E8800324B00684FF42044C3F8D040866936049A
:104E980004D52646013C002EF8D113E046682C4C78
:104EA800344044F0807444F490342C4344604FF40C
:104EB8002044C3F8D0408669B60729D42646013C69
:104EC800002EF8D1C3F8D0401CE02146013C00294F
:104ED800F8D081690E06F8D544681D49214041F093
:104EE800007141F48031294341604FF42041C3F8F7
:104EF800D0108469A40711D40C460139002CF8D1CC
:104F0800C3F8D010FFF7D4FB003018BF012070BDE4
:104F18004FF420448162C3F8D040DAE782624FF44C
:104F28002042C3F8D0208169890606D41146013A87
:104F38000029F8D1C3F8D020E4E7C3F8D020202313
:104F4800C361012070BD00BF6811002060100020FF
:104F5800009800FC2DE9F0474D282DED028B044602
:104F680000F05A8600F2B980302800F0BB8651D88C
:104F7800222800F0978423D8032800F0058214D84B
:104F8800012800F0F581022840F0FB8604200BF090
:104F980031FC43200BF0FFFB4C200BF0FCFB4620C0
:104FA8000BF0F9FB4C2000F05DBE042800F0F58101
:104FB800052840F0E6861A200BF01CFC0024FCE1D2
:104FC800282800F0E88515D8242800F0CF85262861
:104FD80040F0D786D94C06200BF00CFCB4F85C01E5
:104FE8000BF00BFCB4F85E010BF007FCB4F86001A1
:104FF80000F0B9BD2C2800F0E1852E2800F05C8671
:105008002A2840F0BE8601200BF0F4FBCB4B5879E0
:1050180000F028BE3D2800F0F8821ED8362800F09F
:1050280032860BD8322800F01786342840F0A9863B
:1050380048200BF0DFFB002500F056BC3A2800F0B2
:10504800BB823B2800F02784382840F09A86042049
:105058000BF0D0FBB94C00F08FBD452800F07E86E0
:1050680027D8402800F00186422840F08A86B34CB1
:1050780010200BF0BFFB60790BF08DFBA0680BF0E4
:10508800C5FB94F892010BF086FBB4F85C010BF0B9
:10509800B4FBB4F85E010BF0B0FBB4F860010BF0A0
:1050A800ACFBB4F882010BF0A8FBB4F8840100F063
:1050B8005ABD492800F0B4824B2800F09E85462846
:1050C80040F05F860D200BF095FB00200BF063FB92
:1050D80000200BF09BFB00F04CBE702800F0F08223
:1050E80000F2DE80692800F0478200F2AF8066286F
:1050F80000F0A18100F29F80642800F07781652884
:1051080040F03F868E4C0B200BF074FB20880BF090
:1051180074FB62688B4B9A420CBF2089608980B20D
:105128000BF06BFB884B1B68C3F3C000C3F3800212
:10513800800040EA4200C3F340021043C3F3401228
:1051480040EAC20003F0100318430BF056FB7F4BF4
:105158001A88E36812F0010F14BF4FF0020C4FF0E9
:10516800000C12F0020F02F0080814BF4FF0040EF2
:105178004FF0000E03F4475912F0040F14BF102724
:10518800002749EA080912F0400F03F4804814BFC9
:105198002026002649EA080912F0100F03F40048F7
:1051A80014BF4FF40075002549EA080912F0200FD2
:1051B80003F4803814BF4FF48060002049EA0809DE
:1051C80012F4807F03F4003814BF4FF4006100210B
:1051D80049EA080912F4007F03F480285C4A49EA86
:1051E800080903F4002849EA0809127803F480182A
:1051F80049EA080903F0007349EA0303C2F380028D
:1052080043EA020343EA0C0343EA0E0E4EEA070799
:1052180046EA070645EA060540EA050041EA0001B4
:1052280014BF4FF400184FF00008002041EA0808A6
:105238000346217CEAE0672800F02581682840F0D1
:10524800A08510200BF0D6FA00248CE16C2800F021
:10525800A68117D86A2800F00B846B2840F0918546
:1052680005200BF0C7FA3B4B18880BF0C6FA3A4BEF
:1052780018880BF0C2FA324B93F8720000F0010064
:1052880000F0F0BC6E282E4D00F09A8100F2CE811D
:1052980006200BF0AFFA686E0BF0B8FA2F4B89E1D5
:1052A800782800F0FD8018D8742800F03E830AD8CA
:1052B800722800F09D83732840F0638508200BF066
:1052C80099FA0124CDE3762800F0F28300F2668390
:1052D8002F200BF08FFA224CD5E2A42800F00F847F
:1052E80014D87B2800F07582A02840F04A850C204D
:1052F8000BF080FA1B4B18680BF088FA1A4B1868E9
:105308000BF084FA194B186800F037BDF12800F04B
:105318000381FE2800F01A84F02840F03285084CFA
:1053280004200BF067FAA36CB3F85A000BF065FA87
:10533800A36CB3F8580000F016BC00BF2C25002061
:1053480064110020005400406C1200203413002027
:10535800C22F0020EA120020EC1200204012002088
:105368007B820108ACF7FF1FB0F7FF1FB4F7FF1FE0
:1053780003200BF03FFA00200BF00DFA20460BF04B
:105388000AFA0C2000F06EBC0BF034FA01200BF086
:1053980002FA0A200BF0FFF9AFE306200BF02AFA15
:1053A80053200BF0F8F950200BF0F5F94B200BF0D7
:1053B800F2F959200BF0EFF9D4E3B04B185D013442
:1053C8000BF0E9F90B2CF8D10024AD4B185D013432
:1053D8000BF0E1F9082CF8D10024AA4B185D013430
:1053E8000BF0D9F9072CF8D100F0C9BC07200BF055
:1053F80001FAE7200BF0CFF9A34B58790BF0CBF962
:1054080000200BF0C8F9042000F0B7BC8B420BD287
:105418009E4A9C5C012202FA04F414EA080F1CBF9D
:105428009A4010430133F1E70BF0F0F9964B93F8EB
:10543800AC0700F017BC12200BF0DCF9944B1B886A
:10544800B3F5806F8CBF082501250024914B33F9F3
:10545800140090FBF5F0013480B20BF0CEF9032C68
:10546800F4D18D4CA08D0BF0C8F9E08D0BF0C5F987
:10547800208E0BF0C2F9608E0BF0BFF9A08E0BF0F6
:10548800BCF9E08E6FE310200BF0B4F90024834BD5
:10549800185D01340BF07FF9102CF8D100F06FBCC7
:1054A80070200BF0A7F900267B4D0E24AB6C7443DB
:1054B80023440136B3F819010BF09FF9AB6C234470
:1054C800B3F81B010BF099F9AB6C2344B3F81D0139
:1054D8000BF093F9AB6C234493F81F010BF05BF9C5
:1054E800AB6C234493F820010BF055F9AB6C2344C3
:1054F80093F821010BF04FF9AB6C234493F8220188
:105508000BF049F9AB6C1C44D4F823010BF07EF97D
:10551800082EC9D100F033BC70205B4C0BF06AF93F
:1055280004F1700594F8D4000BF035F994F8D5001F
:105538000BF031F994F8D6000BF02DF994F8D70058
:105548000BF029F994F8D8000BF025F994F8D90054
:105558000BF021F9073494F8D3000BF01CF9AC4296
:10556800E0D100F00CBC4E4B185D01340BF013F980
:10557800102CF8D100F003BC4A4D2878400000F008
:10558800FE000BF037F900242B789C4280F0F7835B
:10559800454B33F814000BF030F90134F4E7434C71
:1055A80006200BF027F920880BF027F960880BF00C
:1055B80024F93F4B1888D6E204200BF01BF9DBE3F3
:1055C80007200BF017F93B4B1888FF28A8BFFF20CE
:1055D800C0B20BF0E0F8384B186880F3100080B2C6
:1055E8000BF00BF9B5F868000BF007F9264B93F8A8
:1055F8008721324B186822B10A23584380F31000E0
:1056080001E000F30F0080B2ADE21F4C02200BF066
:10561800F1F894F8DE010BF0BEF894F8DD0121E30F
:1056280002200BF0E7F8184B98899CE20B200BF04E
:10563800E1F8EB6E18780BF0AEF8EB6E58780BF0DB
:10564800AAF80026EB6E144C3344013618790BF097
:10565800A2F8032EF6D1E36ED8790BF09CF8E36E2E
:1056680098780BF098F8E36ED8780BF094F8E36E1E
:1056780058890BF0C2F8E36E187AF3E2A4A1010886
:10568800B0A1010885A101082C2500207511002072
:10569800040000203A120020641100209C11002010
:1056A800B01100203C23002008250020C22400203F
:1056B800481200205C1200206812002064120020AA
:1056C800C64C1E200BF096F8A36C1B78022B4FF0EB
:1056D80000056BD1A36C03EB850393ED080AB2EECA
:1056E800048A20EE080A10F0CDFB80F30800C0B24F
:1056F8000BF051F8A36CDFEDBA7A03EB850393ED59
:105708000B0A20EE270A10F0BDFB80F30800C0B298
:105718000BF041F8A36CDFEDB37A03EB850393ED4F
:105728000E0A20EE270A10F0ADFB80F30800C0B285
:1057380001350BF030F8032DCCD1072DA36C23D104
:1057480093ED110A20EE080A10F09CFB80F3080084
:10575800C0B20BF020F8A36C93ED120A20EE080AF1
:1057680010F090FB80F30800C0B20BF014F8A36CA3
:1057780093F84C3000EE103AB8EE400A10F082FB75
:1057880080F30800C0B20BE02B4458780BF003F804
:10579800A36C2B44D87A0AF0FEFFA36C2B44587DE7
:1057A80001350AF0F8FF0A2DC7D1E8E2A36C2B44B3
:1057B80058780AF0F0FFA36C2B44D87A0AF0EBFF74
:1057C800A36C2B440135587D0AF0E5FF0A2DEDD175
:1057D800D5E23C200BF00EF80024804D9FED818A25
:1057E800AB6C03EB840393ED080A20EE080A10F073
:1057F80049FB80B20BF001F8AB6C03EB840393ED2B
:105808000B0A20EE080A10F03DFB80B20AF0F5FF03
:10581800AB6C03EB840393ED0E0A20EE080A10F03C
:1058280031FB013480B20AF0E8FF032CD5D1072CF4
:10583800AB6C16D193ED110A20EE080A10F022FB8A
:1058480080B20AF0DAFFAB6C93ED120A20EE080A78
:1058580010F018FB80B20AF0D0FFAB6C93F84C0044
:105868000BE0234458780AF0C8FFAB6C2344D87A7D
:105878000AF0C3FFAB6C2344587D01340AF0BDFF26
:105888000A2CD4D17BE214F8010F002800F07782AB
:105898000AF081FFF7E701200AF0ACFF4F4B9B6C41
:1058A8001878DFE150200AF0A5FF00254B4B9C6CCF
:1058B8004D4B04EB85040C2194F8792001FB02334D
:1058C800013593F838000AF066FF94F87A000AF078
:1058D80062FF94F87B000AF05EFF94F87C000AF0FF
:1058E8005AFF142DE2D14AE23C4B9C6C062303FB81
:1058F8000544013594F8CE000AF04DFF94F8C9002C
:105908000AF049FF94F8CA000AF045FF94F8CB0062
:105918000AF041FF94F8CC000AF03DFF94F8CD005E
:105928000AF039FF0C2DDFD129E24FF000080126DB
:1059380000272A4B1A7C974227DA11330024FA5C95
:10594800294D0C2305F130016343595C914207D17D
:105958002B44586B10F0CBF882462EB9B14605E0BF
:1059680001341B2CECD10EE080440CE0D1450ADA5E
:105978000C2303FB04535B6B13F809000AF00BFFBD
:1059880009F10109F2E70137D3E7002E00F0F781AA
:105998005FFA88F00AF02EFF0026C9E70F4D287C31
:1059A8000AF028FF00242B7C9C4280F0E8810F4BF2
:1059B800E65C00210C480C2200F1300702FB01F3E1
:1059C800DA5DB24205D1034493F838000AF0E3FEE9
:1059D80002E001311B29EDD10134E4E76411002014
:1059E8000000C84200007A447C820108751100203A
:1059F800CF4C16200AF0FEFEB4F898010AF0FDFE1E
:105A0800B4F844010AF0F9FEB4F846010AF0F5FECC
:105A1800B4F848010AF0F1FEB4F8DA010AF0EDFE34
:105A280094F8EB010AF0B7FE00200AF0B4FE94F8EF
:105A3800EC010AF0B0FE94F887010AF0ACFE94F885
:105A480094010AF0A8FE00200AF0A5FEB94B9B6C51
:105A58000A20B3F9563093FBF0F080B20AF0CDFE7D
:105A68008AE0E0B201340AF096FE092CF9D186E109
:105A780010200AF0BFFEB04BB04C187800F00200BE
:105A88000AF089FEAE4B18780AF085FE20680AF005
:105A9800BDFE60680AF0BAFEAA4B18880AF0ADFE8F
:105AA800A94B18880AF0A9FEA24BB3F870005AE077
:105AB8000AF054FE074612200AF09CFE9D4C17B9C6
:105AC800666FA56F06E0102F13BF0025E66FD4F8A8
:105AD80080502E4638460AF05EFE30460AF096FEA2
:105AE80028460AF093FED4F884000AF08FFE0020BE
:105AF8000AF083FE00200AF080FE0020B2E08D4DFF
:105B080095F8880080000130C0B20AF073FE95F85D
:105B180088000AF040FE00242E4696F888309C4201
:105B280080F02D81894D285D0AF035FE05F11003BE
:105B3800185D0AF030FE05F120033035185D0AF0D3
:105B48002AFE285D0AF027FE0134E6E708200AF05D
:105B580051FE00200AF051FE00200AF04EFE0020FF
:105B68000AF04BFE00200AF048FE08E104200AF083
:105B780041FE6F4B986800E194F87C010AF00BFE37
:105B880094F880010AF007FE94F87F010AF003FEFA
:105B980094F8810166E0664C07200AF02BFEB4F801
:105BA80082010AF02AFEB4F884010AF026FE94F86D
:105BB80086010AF0F0FDB4F88801D4E75C4C0C20AB
:105BC8000AF018FE94F892010AF0E5FDB4F89C0179
:105BD8000AF013FEB4F898010AF00FFEB4F89A011F
:105BE8000AF00BFE94F893010AF0D5FDB4F89E0173
:105BF8000AF003FEB4F8A001B5E74D4C04200AF002
:105C0800F9FD94F8D8010AF0C6FD94F8D9010AF014
:105C1800C2FDB4F8DA01A6E74D4C4E4D207800EBF2
:105C28004000C0B20AF0E6FD002623789E4205F146
:105C3800020580F0A48015F8020C0AF0ACFD15F8F6
:105C4800010C00EB800000EB800000F2EE2080B237
:105C58000AF0D3FD0136E8E701200AF0CBFD344B0A
:105C680093F894010AF097FD89E008200AF0C2FD34
:105C780000242F4B2344013493F88A010AF08BFD4A
:105C8800082CF6D17BE02B4B294C93F8C900C0EBCC
:105C9800C000C0B20AF0AEFD04F1200594F8F2018C
:105CA80000232D4AD25C90426DD00C33302BF8D1B2
:105CB8000834AC42F2D162E040201D4C0AF09AFD53
:105CC80004F14005B4F8A4020AF097FD94F8A6027E
:105CD8000AF061FD043494F8A3020AF05CFDAC42BA
:105CE800F0D14CE0E020124C0AF084FD04F180056C
:105CF800B4F8260200F03F000AF07FFDB4F826024F
:105D0800C0F386100AF079FD94F8240200090AF01D
:105D180042FD94F8240200F00F000AF03CFD043420
:105D280094F821020AF037FDAC42E1D127E000BF28
:105D38002C25002064110020701200207812002009
:105D4800761200207412002072120020ED1100203B
:105D58003C230020CE2600204823002013200AF0F0
:105D680049FD0024154B185D01340AF014FD0B2C75
:105D7800F8D100200AF04AFD00200AF047FD012072
:105D880018E0002016E00AF006FDB4F8F4010AF065
:105D980034FD94F8F6010AF0FEFC94F8F7010AF0D5
:105DA800FAFC94F8F9010AF0F6FC94F8F8010AF004
:105DB800F2FC7DE7BDEC028BBDE8F087A4A10108E9
:105DC8002DE9F047CB4CCC4F237886B00646002B04
:105DD80000F0EB813A686368D31A7C2B40F2E581C6
:105DE800237A6260013323724FF0000808F124001F
:105DF800C04DC0B205F0D2FA05F10A0333F91830E4
:105E080007EE903ABD4B1B88B8EEE77A07EE903A5A
:105E1800F8EEE77A08F10108C7EE277A9FEDB87A1D
:105E280067EE877AFDEEE77ACDED037ABDF90C00CF
:105E380005F0A2FAB8F1030FD8D1302005F0AEFA78
:105E4800B5F9100005F098FA05F0A0FA2B7A9A0730
:105E58002CD16A6841F288339A4218D9102005F08B
:105E68009DFA4FF06408686990FBF8F000B205F0FD
:105E780083FA212005F092FA686990FBF8F308FB91
:105E880013000028B8BF404200B205F075FA14208C
:105E980005F084FAB4F9180005F06EFA1C2005F034
:105EA8007DFA002005F068FA05F070FA237ADFF829
:105EB80044825B0740F05681022005F06FFAD8F85B
:105EC8001C00DFF854926423323090FBF3F000B2E8
:105ED80005F052FA0320B8F9265005F05FFA894B0D
:105EE8001B7813F0040F4FF0050A95FBFAF5ADB2D5
:105EF8000BD030460CF06BF828B9D9F8003013F005
:105F0800100F18BF002528B205E0D8F82830988966
:105F1800B0FBFAF000B205F02FFAD9F800309E076E
:105F280065D5DFF8F891E68D99F80030A28D714DAE
:105F380036014FF06408B6B208FB02325B00B2FBD0
:105F4800F3F346EA0326B6B2C3F303231E4306203F
:105F580005F024FA30B205F00FFAE38D99F8001035
:105F680001339BB293FBF1F201FB1233E385236B00
:105F78009B7B012B05D1392005F010FAB5F92C00CF
:105F880019E0AD8D6E233A205D43152605F006FA1B
:105F980095FBF6F5AEB2B6FBF8F528B205F0ECF9CC
:105FA80008FB15653B2005F0F9F9A8B2451D0A2044
:105FB80095FBF0F000B205F0DFF9282005F0EEF9C6
:105FC800636B0A2093FBF0F000B205F0D5F90420CA
:105FD80005F0E4F9A36A9B8913B102F03DFA03E0E6
:105FE800444B986B80F3100000B205F0C5F9E36BE1
:105FF800404E9D0640F1AB8096F8403098071DD57D
:10600800112005F0CBF9B6F842003F4B4FF4F36589
:10601800684390FBF3F000B205F0AEF9192005F0E3
:10602800BDF9B6F842004543642095FBF0F595FBB1
:10603800F0F300FB135000B205F09EF994F84030DD
:10604800B4F8445013F0020F08BF0025012005F0F2
:10605800A5F928B205F090F9092005F09FF900206C
:1060680005F08AF9294B94F846501A88B2F5967FBC
:106078000AD9204B1B7A03F00F03072B04D842F2EE
:106088000F75954228BF1546052005F087F9236B43
:106098005B7B0BB928B21CE0A5F1200307EE903A10
:1060A8009FED1B7AF8EEE77AF6EE006AC7EE877A7C
:1060B800BEEE007AF5EEC07AF1EE10FA58BFB0EEF7
:1060C800667A77EE877AFDEEE77ACDED037ABDF949
:1060D8000C0005F051F994F84020064B910703D4C1
:1060E80093F84720012A1DD1012384F84730094835
:1060F80034E000BF30120020F0240020040000200B
:1061080000007A44C22F0020A0860100FE00002073
:106118006666E63F78120020CC240020FC000020B0
:106128008096184B1B6B5FED026A93ED017AD3EDF5
:10613800027A27EE267A67EEA67ABDEEC77AFDEEDA
:10614800E77A8DED047ACDED057A04A806E0B54A24
:1061580092E8030004AB83E80300184602F022FF2C
:1061680005F014F9237A282B1FD1AF4B00221A729D
:106178003C263B684FF47A70B3FBF0F8172005F023
:106188000DF9B8FBF6F5B5FBF6F006FB105000026A
:1061980000B205F0F1F8182005F000F906FB1580AB
:1061A80000B205F0E9F805F0F1F894F850309E4D8A
:1061B800002B00F0588106F005FD6B6D9B4AC31A51
:1061C8009342064640F2C180002385F85A3085F88C
:1061D8005C30AB8DDAB21B0A85F8762085F877300B
:1061E80085F86C2085F86D30D5F884203B689A1ABC
:1061F800D5F88830D97B4FF47A734B439A420ED343
:106208008B4B1B68C5F8843095F88C30013B012B0B
:106218009FBF102385F85A30022385F85C300A2086
:10622800626B92FBF0F284F87420121284F87520E5
:1062380094F84020A36B93FBF0F384F878301B129A
:1062480084F87930920794F84630774984F8A73073
:1062580003D42D2381F8A83076E0042BD4F8489095
:10626800E76CDFF8DC81734A8CBF3323322381F873
:10627800A8304FF0060C704B99FBF3F097FBF3F343
:1062880008FB009108FB037803EB83030CFB01F187
:1062980003EB830391FBF2FE642502FB1E119B00B6
:1062A80091FBF5F184F8991009120CFB08FC84F8AD
:1062B8009A109CFBF2F143FA81F39BB202FB11C2E4
:1062C80092FBF5F284F89E20121284F89C3084F830
:1062D8009F201B0AB4F8422084F89D30242353439E
:1062E80093FBF5F5B4F8BA3084F8A03000EB8000E1
:1062F8001B0A00EB8000800084F8A1300A22B4F861
:106308004430B3FBF2F303F5FA739BB240FA8EF014
:1063180080B284F8A2301B0A4FEAD97984F8970032
:10632800FF0F000A84F8945084F8A330C5F30725BA
:10633800B4F8BC3084F8969084F8980084F89B7080
:1063480084F8955084F8A930666594F8BE80364D77
:10635800B8F1000F0DD1D5F8C40006F0EAFD012808
:1063680007D90228354F00F0528202F00DFE0123B2
:10637800BB70D4F8C8202C4D002A74D095F8BE7094
:106388003FB1D5F8D03040F6B731F31A8B4219D85F
:1063980069E00123D5F8C40085F8BE3007F0A1FFF5
:1063A800D5F8D43093F9000002238DE8880008213D
:1063B8003A464FF4964306F036FC85F8D870C5F88F
:1063C800C4004EE095F8CC70CFB9D5F8C400C5F834
:1063D800C87085F8BE7007F084FFD5F8D43093F9FB
:1063E800000001238DE8880008213A464FF49643BF
:1063F80006F019FCC5F8C40002F0C6FD31E0013F03
:10640800FFB285F8CC7095F8D81095F8D930CFB987
:106418004A1C013385F8D82085F8D930D5F8C4004E
:106428001DE000BFFC830108301200203F0D03006F
:10643800F024002040420F008096980004000020BD
:10644800806967FF12F8017BC5F8C820781885F8BD
:10645800D8000133D5F8C40085F8D930394606F09C
:106468006BFDC4F8D06094F8DA309D4DF3B1D5F8DF
:10647800DC30DBB1D5F8E030C3B1C5F8E4301B68D7
:10648800984AC5F8E830D5F8EC301344187AFEF786
:1064980061FDD5F8E43098790AF07DF9D5F8EC304B
:1064A8000133092B88BF0023C5F8EC308E4D94F8D2
:1064B800F0202E688A4B002A00F0E381D3F8F420FC
:1064C800002A00F0DE8193F8F830013B012B00F23E
:1064D800D881D4F8F400824F06F02BFDE0B1D7F84C
:1064E800F40006F023FD97F8F930D5F800907E2BDC
:1064F80080460ED102231B2887F8F83009D1D7F837
:10650800F40006F016FD20B90123C7F8FC9087F8BF
:10651800003184F8F980DCE7D7F8FC202B689B1A57
:1065280041F6583293421DD9032387F8F830A8E181
:106538006E4A32F8130010B903464FF40360013372
:10654800B0F5C06FDBB275D01DD9B0F5006F7AD049
:1065580031D9B0F5036F3ED184F80131E36B604F58
:1065680099063FD494F8001194F80131002900F0FD
:106578004B812A68921B012ADAD984F80131002359
:1065880084F800317DE1B0F5007F42D007D8B0F53E
:10659800807F47D0B0F5887F00F08580E6E7B0F5CA
:1065A800806F00F0A780B0F5826F00F0EC80B0F546
:1065B800047FDBD123E0B0F5E26F00F08480B0F512
:1065C800E46F00F08580B0F5E06FCFD184F8013139
:1065D800B4F90A1080E0B0F5046F6DD0B0F5026F21
:1065E800C4D1FBE097F840309A07BBD5B7F8421002
:1065F80024234B431233642193FBF1F1FEE084F82A
:1066080001313B4B364F1B689B07ABD5BB8D0A212D
:10661800F3E084F80131364B314F1B681905A1D5D9
:10662800796BEBE084F80131E36B2D4F5A0799D56C
:106638007969E3E084F801312D4B294F1B681B056C
:1066480090D5B96BDAE0E16B254A84F801318F0601
:1066580088D592F84010880784D5D90711D5D36C0E
:1066680083EAE371002BA1EBE37101EB51014FF0D9
:106678001902B1FBF2F1ACBF41F0004141F04041D9
:106688000EE0936C83EAE371A1EBE371002B01EB5D
:1066980051014FF01902B1FBF2F1B8BF41F080414E
:1066A8004FF4006089E084F80131E36B0C4F5B071D
:1066B8007FF558AF3969A1E0B4F9181084F80131B1
:1066C8006423594379E084F80131B4F90C1003E0EC
:1066D800B4F90E1084F801312C2391FBF3F16CE02E
:1066E80030120020FC830108F0240020B2A5010824
:1066F800CC24002084F8013194F80231624A013335
:10670800DBB2032B88BF012382F8023194F802110F
:1067180042F2107359435D4B1B78D80748BF0131CB
:106728009A0748BF02315F07B4F8043148BF043103
:10673800D80748BF0A319A0748BF14311F0648BF17
:106748002831D80548BF28315A0748BF64311F0788
:1067580048BFC831980548BF01F5C8719A0648BFB7
:1067680001F57A71DF0648BF01F5FA61580648BF9E
:1067780001F57A614FF4806002F0D2FB424B0022AF
:1067880083F80021EEE6E16BDFF8FC8084F8013144
:1067980011F0200717D098F8402012F0020F14BF0C
:1067A8004FF47A71002112F0010F14BF4FF4FA630D
:1067B80000230B4494F84610194402F0B1FB00235F
:1067C80084F80031CEE6324B1B6819067FF5CAAE55
:1067D800394602F0A5FB88F80071C3E684F8013158
:1067E800E36B294F9A067FF5BDAE97F840309B07BB
:1067F8007FF5B8AEB7F844306421594302F090FBF6
:10680800002387F80031ADE684F8013139E0BB7820
:1068180023B1C5F8C06087F80280AAE5D5F8C03072
:10682800F31AB3F57A6FFFF4A4AD0123D5F8C400C9
:10683800BB7006F07BFB0746D5F8C40006F076FB74
:106848007F067FF496AD8A2802D08E280CD090E57A
:10685800EB6B98067FF58DAD95F8BE30002B7FF475
:1068680088AD05F18D0306E095F8BE30002B7FF466
:1068780080AD05F15803C5F8C8302D2385F8CC3014
:1068880077E506B0BDE8F08730120020C22F00205F
:10689800CC24002082B01B4B1B4A8DF807101968C6
:1068A800106860B31268052A29D1184A106810BB0D
:1068B8009DF808109DF8073043EA012314490B801E
:1068C800144B1968144B89B20B445B0019680121F9
:1068D800196013680B441360104A136823F4E043EB
:1068E80023F040039BB283F0300343F4004343F0AA
:1068F8008003136003E01A68521A312AD5D902B00E
:10690800704700BFF0240020A82F00209822002004
:1069180080610040505C00400A300020045C004068
:10692800014B1868C0B270475422002001207047FC
:10693800704770476D4B6E4A9FED6E7AD2ED007AC4
:10694800DFED6D4ADFED6D3A30B51C88B3F90AE02A
:106958001D8A06EE904AB8EEE76AF8EE666ADFED41
:10696800687AB3F9044067EEE67AB7EE004AE6EED5
:10697800077A9FED647A67EE666A9FED637AE6EEC2
:10698800076A27EEA77A07EE904AB3F902409FED0F
:106998005F6AF8EEE77A67EE277A07EE104AB8EEF4
:1069A800C77ADC89E6EE877AB6EE007AFDEEE76A0A
:1069B80087EE866AC3ED066AF8EEE66AD2ED017ADA
:1069C8009A89E6EE874A06EE90EAB3F908E09FED69
:1069D800507A05EE90EAF8EEE66AF8EEE55A66EEC9
:1069E800A46A65EEA45A66EEA46AB3F806E0E6EE79
:1069F800875A65EE875AA5EEA34AF0EE445A04EE8C
:106A080010EAB8EE444A25EE844AB5EE404AF1EE63
:106A180010FA5BD02DB205EE905A24B224EEA45A97
:106A280007EE104AF8EEE55A12B265EE255AB8EEAE
:106A3800C75A65EEA35A64EE854AB0EE007AE4EED2
:106A4800875AB5EE007A65EE875A07EE102AB8EE37
:106A5800C75A9FED307ADFED306AB3F91620E5EEBC
:106A6800075AF8EEE77A9FED2D7A76EEE77ADFEDB2
:106A78002C6AE5EEC77A05EE902AB0EE677ADFED6C
:106A8800297AB3F91420B3F9123067EE277A07EEA2
:106A9800102AC7EE847AF8EEE55AB8EEC77A65EEA2
:106AA800A75A27EE877A65EEA75A27EE237AA5EE2E
:106AB800A67AF0EE476A07EE103AB8EEC77A36EED5
:106AC800877ADFED196AE7EE267A01E0DFED177ABB
:106AD80018B1FDEEE77AC0ED007A31B1FDEEC67A65
:106AE800642217EE903A53430B6030BD0803002030
:106AF800381300200000003700007AC70000003873
:106B0800000000390000803A000080380000A045ED
:106B180000000036000080470000804900008039EE
:106B2800000000300050C3450000803D0000000018
:106B3800704770476C4B6D4A2DE9F04F5E89946839
:106B48004FEA062AB4EB0A0A9C884FEA04481C89D3
:106B58004FF000054FF0000B65EB0B0BA4FB0A6729
:106B680004FB0B77F40944EA476418EB04065C88D5
:106B78004FF000094FEAE7154FEAC438DC8849EBC3
:106B8800050787B0CDE90467A4FB0A6704FB0B7708
:106B9800340A44EA076418EB04064FEA27259C895F
:106BA8004FF0000949EB0507CDE90067AAFB046728
:106BB80004FB0B77F40D44EA472414F5FA664FEA10
:106BC800E75545F10007B6F5FA6F77F10003CDE90F
:106BD8000267964667DAA4FB046704FB05F34FF0E7
:106BE800050C07EB4307DDE90489A6FB0C230CFB26
:106BF80007335F104FEA3206B8EB06084FEA9206F1
:106C080069EB070946EA83769F10DDE90023921BAA
:106C180063EB0703DDE90267CDE90023344A4FF04F
:106C2800FF33964277EB0303CDE9048928DA40F66F
:106C3800AC52A4184FF000035D4104FB05F3A4FB1C
:106C4800044505EB43056FF00602664202FB056644
:106C5800A4FB0223334418EB020649EB0307CDE9F2
:106C680004670B26A4FB062306FB0533DDE9004574
:106C78005B104FEA3202A41A65EB0305CDE9004523
:106C88000AFB0BF3DDE90245AAFB0AAB0BEB430B4E
:106C98004FEADA7242EA4B02A41A4FEAEB7365EB49
:106CA8000305CDE90245DEF80C40009B019DA4FBDD
:106CB800032304FB05334FEA52584FEA635948EA65
:106CC800C328DDE90423B8EB020269EB0303994604
:106CD800D30B43EA494300B1036009B1029B0B603F
:106CE80007B0BDE8F08F00BFF6020020381300207F
:106CF80024FAFFFF07EE900AF8EEE77ADFED0C6A58
:106D08009FED0C0AF5EEC07AF1EE10FAD4BFB1EEA1
:106D1800677AC7EEA67A08B5D8BFC7EE267A27EEF7
:106D2800800A02F0C5FC044B83ED000A08BD00BFD1
:106D38008096184B35FA8E3C6C000020F7B51C4B3A
:106D48001A680AB91C6800E001241A490E7C00225E
:106D5800D0B2A04202F1010207D202AD2F18164D9F
:106D68003544285C07F8040CF2E71A68121B1A600D
:106D78000A7C1D6822440A749DB90320402100F052
:106D88007BFF0E4A136823F4804323F070039BB201
:106D980083F4405343F4004343F080031360054BEE
:106DA8001D74002CCBD09DF8040003B0F0BD00BFCB
:106DB8005422002038130020582200200C5C004088
:106DC8007620F4213122FEF757B81FB50446022178
:106DD8000C2001220DF10703FDF7D2FFC8B39DF87F
:106DE8000730DB0735D50321062202AB0C20FDF75F
:106DF800C7FF0C20092101220DF10703FDF7C0FF91
:106E080038B39DF8073013F00C0F22D19DF80920F4
:106E18009DF8083043EA0223C3EB83339B009DF8B7
:106E28000B2023809DF80A3043EA0223C3EB833307
:106E38009B009DF80D2063809DF80C3043EA0223E7
:106E4800C3EB83339B00A3800C200A210122FEF7A9
:106E580013F804B010BD07B5F7216B46062276205B
:106E6800FDF78EFF9DF800309DF801100B4A1B03BB
:106E780043EA01139DF8021043EA111353609DF889
:106E880003309DF804101B0343EA01139DF8051015
:106E980043EA1113136003B05DF804FB38130020B4
:106EA80007B50A2100220C20FDF7E6FF142005F0A3
:106EB800B0FE0A210F220C20FDF7DEFF0A2005F0A4
:106EC800A8FE01AB102103220C20FDF759FF0A2070
:106ED80005F09FFE0A2100220C20FDF7CDFF0A20B5
:106EE80005F097FE0DF10303022101220C20FDF7A6
:106EF80047FF0DF10303092101220C20FDF740FF94
:106F08000A2101220C20FDF7B7FF03B05DF804FB4E
:106F1800F8B59F4B1B680446187818B1012800F093
:106F28007181EDE2242C9B4D0CD006D80A2C00F080
:106F3800DD800D2C00F0DA804EE12A2C06D02C2CB6
:106F480004D049E16874A874E87457E1924BA97CAD
:106F58006F7C904A002058542FBB19781775472921
:106F680021D1597850291ED19978472907D1D97844
:106F7800472904D11979412901D10121117599783D
:106F8800854A522903D1D1784D2900F0BB829978DE
:106F9800814A472907D1D178532904D11279562A31
:106FA80004BF03222A752A7D7A4E022A3AD0032A80
:106FB8004DD0012A40F08880BA1E072A00F284804A
:106FC800DFE802F004080F131A25822B0AF042FFAB
:106FD800A86179E01B78532B76D1AB695B42AB6132
:106FE80072E00AF037FFE8616EE01B78572B6BD12F
:106FF800EB695B42EB6167E01B78302B674B1A78D3
:107008008CBF42F0020222F002021A705CE00020FB
:107018000AF080FF85F8200056E000200AF07AFF89
:10702800688451E0072F06D0082F4DD101200AF0BF
:1070380071FFF08448E001200AF06CFF41F2184328
:1070480058434FF47A73B0FBF3F0B0843CE0022F5E
:1070580007D0032F0BD100200AF05CFF504B1870AB
:1070680032E000200AF056FF86F828002CE02BD9E1
:107078003A1F921096F828300132D2B2013B02EB47
:107088008303DBB2102B1FD8F91EC2F1010201EBFA
:107098008202D2B2012A0BD0042A11D100205E1E2E
:1070A8000AF038FF3F4B98553F4B00229A5507E0AE
:1070B8005E1E3E4A002093550AF02CFF3C4B985523
:1070C8003C4A136801331360324B2A2C18BFDA7C10
:1070D80007F101074FF000000CBF012254406F7404
:1070E800A8740CBF83F82920DC7487E095F8290080
:1070F800002848D0304B13F8012D30495A708B4284
:10710800F9D1254A234C13785278402B85BF373B59
:107118001B011B01DBB298BF03F0F003402A8CBFB0
:10712800373A303AD2B21344EA7CDBB29A4227D1DA
:1071380021230B702249207D0B68204A0133012846
:107148000B600AD002281DD1722313701D4BA28C2C
:107158001A801D4BE28C1A8014E0672313700F4BC2
:107168001B789F070FD5194BA2691A60E2695A600C
:10717800174B94F820201A70164B628C1A8002E084
:107188003F230B700020002385F8293036E000BF2C
:107198002008002038130020F82400207012002056
:1071A800EC1100201D1200200D120020ED1100200E
:1071B800FD11002064170020440300203003002044
:1071C8007017002072120020D411002078120020BD
:1071D8007612002074120020AB7C95F829000E2B43
:1071E8009FBFAB4A591C9174AA4A98BFD454A84A65
:1071F80018B9D37C5C40D47400E00020003018BF7C
:107208000120F8BDA24B93F82A100022082900F2A9
:107218007781DFE801F0050C101A2B3B5F7B8800B3
:10722800B52C40F06D8183F82B2001224FE0622CB1
:1072380008BF02224BE0032283F82A2083F82C405F
:1072480083F82D4083F82E405AE1042283F82A203F
:1072580093F82D2093F82E1083F82F402244D2B2B1
:1072680083F82D200A4483F82E2049E1052283F86B
:107278002A2093F82D2093F82E101C862244D2B28F
:1072880083F82D200A4483F82E2039E1062283F85A
:107298002A2093F82D2093F82E102244D2B283F896
:1072A8002D200A4483F82E201A8E02EB0424A4B25F
:1072B800B4F5AC7F88BF764A1C8684BF012182F86A
:1072C8002B1000225A86002C40F01A81072283F8DE
:1072D8002A2015E193F82D2093F82E102244D2B2DB
:1072E80083F82D200A4483F82E205A8EB2F5AC7FFD
:1072F8003CBF6749891802F1010238BF81F8344060
:10730800198E92B291425A86E0D9F9E0082283F8A0
:107318002A2093F82D30A34200F0F2805C4B012222
:1073280083F82B200FE05C4D83F82A2015F8012DF7
:107338006A705A4A9542F9D193F82E10544AA142DC
:1073480006D03F232B70564A536801335360D7E069
:10735800544801680131016092F82B0010B13E23B6
:107368002B70CDE02121297092F82F10062941D0E9
:1073780004D8022907D0032923D0F8BD122959D0EF
:10738800302967D0F8BD502129704749946B4C606B
:10739800D46B0C60516C4FF47A7491FBF4F1434C4C
:1073A800218092F88C11424A19B1117841F00201FA
:1073B80002E0117821F002011170012283F88D2179
:1073C80090E05321297092F83910CE0705D592F82C
:1073D8003820D51E6A426A4100E0024602F00101E7
:1073E80083F88C11002A7DD131490A7822F00202F3
:1073F8000A7077E04F21297092F83F10CC0705D525
:1074080092F83E20D11E4A424A4100E0024602F06C
:10741800010183F88C1122B925490A7822F0020269
:107428000A70244A93F863101170234AB3F8601065
:10743800118057E0562129702049946C0C8042F243
:107448001074D16C91FBF4F11D4C2180012182F85C
:107458008E1147E04921297092F83810194A1029ED
:1074680088BF10211170184914780022A24235D221
:10747800164D0E7A5655164D4E7A5655154DCE7AEE
:107488005655154D11F80C6F56550132EEE700BFF1
:1074980038130020F8240020440300203003002083
:1074A80000080020701700207812002074120020B5
:1074B8007012002076120020FE00002072120020B8
:1074C800D4110020EC1100206C130020ED110020D5
:1074D800FD1100200D1200201D1200200D490A6820
:1074E80001320A6093F88D310B4A93B192F88E31CC
:1074F8007BB1002182F88D1182F88E111846F8BDF3
:107508000020F8BD1279432A7FF441AD02222A7582
:107518003DE5F8BD64170020381300200449054BE9
:107528000968187000225A6199611A77704700BF7C
:10753800F02400200008002010B5121A07EE902A47
:107548005B1A2DED028BF8EEE78A07EE903A184B9E
:10755800059CB8EEE78AD3ED007A28EE278A28EE54
:10756800080AA8EEA80A0EF033FFDFED127A049B92
:1075780020EE270AF0EE480ABCEEC00A83ED000AA6
:10758800B1EE680A0EF080FDDFED0B7A9FED0B7A05
:10759800E0EE077ABDEC028BFDEEE77A17EE903A43
:1075A800002BBCBF03F50C43A033236010BD00BF04
:1075B8006C0000202C7D8E3F00A00C46A00CB3452B
:1075C80044F25063984203DDA0F50C40A0387047A0
:1075D800034B9842BCBF00F50C40A030704700BF79
:1075E800B0B9FFFF73B51A4C036823600B6863607A
:1075F800184D0068184EFFF77DFB184B009395E86F
:10760800030094E80C000196FFF796FF144B3268CC
:107618001A606868636813491B1A07EE903A124BA0
:10762800286893ED007A23681B1A0B600F4BF8EE5D
:10763800E77A1A600E4B67EE877A1B68FDEEE77AE9
:10764800DA880C4BC1ED017A1A8002B070BD00BF18
:10765800D421002078120020E0210020DC21002025
:107668001C220020E42100206C00002014220020AD
:10767800980F0020102200204279DFED2A5A2A4B69
:107688009FED2A5A07EE902AF8EE677AC27BC7EE7A
:10769800A57AB2EE047AC3ED007A07EE902AF8EEE6
:1076A800677A234ADA60C7EEA57AC3ED017A817951
:1076B800204B07EE901AF8EE677A017CDA60C7EE85
:1076C800877AC3ED007A07EE901A817E06EE101ACB
:1076D800F8EE677AB8EE466AC7EEA57A86EE056ACE
:1076E800C3ED017A83ED026AC179134B06EE901A55
:1076F800417CDA60F8EE666AC6EE876A07EE101A11
:10770800C17EC3ED006A07EE901AB8EE477AF8EE2C
:10771800677A87EE257AC7EE857A83ED017AC3ED1D
:10772800027A70470000C842EC21002000007A4429
:107738000000FA44FC2100202022002010B50C4C47
:1077480023789B0713D50B4B1B78042B0FD90A4AB8
:107758000A4B106852685A601860FFF7CBFA084B5A
:107768001A88084B1A80237843F00103237010BD50
:10777800701200207612002078120020D811002004
:1077880048120020302200201C4B1B681B0307B541
:1077980030D51B4A1B4BD2ED007A1B788DF8003090
:1077A800B2EE047A67EE877A174B9FED187A1B784A
:1077B8008DF80130FCEEE77A0A2017EE903AD2ED08
:1077C800017A8DF8023067EE877A6946FCEEE77A2F
:1077D80017EE903AD2ED027A8DF80330FCEEE77A94
:1077E80017EE903A8DF80430094B1B788DF8053068
:1077F80001F006F803B05DF804FB00BFCC240020BC
:10780800E0240020BC240020DC24002000007A446E
:10781800C0240020054A137883F001031370044A3A
:1078280000231360034A1360AEE700BFC0240020A2
:10783800D8240020D424002010B5214A18B9136890
:1078480002221A8210BD1F48146800230380217881
:1078580011F07F0102460DD1637A990644BF0221D7
:10786800017013F0400F037814BF43F0010323F0B5
:10787800010315E0012921D002291ED1637913F0F3
:10788800800F03F00F034FEA830303F1804303F5EE
:10789800B8431B6806D003F03003102B07D101232F
:1078A800137004E003F44053B3F5805FF6E7064B2A
:1078B8001B681B699847034810BD184610BD00BFD8
:1078C80034220020C8140020C41F002010B5064C24
:1078D80018B9236801221A8210BD044B1B689B68E3
:1078E800984720680C3010BD34220020C41F0020A7
:1078F80010B5064C18B9236801221A8210BD044B32
:107908001B681B68984720680A3010BD3422002085
:10791800C41F002003788B4283BF034B03EB410154
:1079280048880020704700BFC814002070B50022A6
:107938001346244914180C44A47E83EA042308241B
:1079480013F4004F4FEA430318BF83F4815304F143
:10795800FF3418BF83F0010314F0FF049BB2EFD18A
:107968000132192AE5D100F1190200F11A050A4479
:107978000D44967EAA7E02EB062292B29A421FD14D
:10798800104B93F83B50E2B2AA4216D2431C03EBC9
:107998004203DBB2CA1801330B44927E9B7E03EB91
:1079A80002239BB24FF4AF6253431B13064A03F5FD
:1079B800487322F814300134E5E7012381F83C309C
:1079C80070BD00BFC8140020CA14002003788B4281
:1079D8000BD9074B1A78074B89001944086C02B178
:1079E800400800F5777080B270470020704700BFEC
:1079F80040230020C814002007299DBF034B03EB38
:107A08008101B1F870000020704700BFC814002041
:107A1800034B03EB4101B1F89000C008704700BF69
:107A2800C814002070B5334C054605F0CBF8D4F8DF
:107A3800B030C4F8B000C31AB3F5FA5FC4F8B43074
:107A480082BF002384F8B83084F8B93094F8B8308D
:107A58002BB9A12D02BF274A012182F8B91094F849
:107A6800B910244A29B1D118EDB201338D7682F8C4
:107A7800B83094F8B85094F8BA30AB4239D11D4BAD
:107A880093F8BB30052B02D0062B03D02CE0002046
:107A9800FFF74CFFE37E1E2B26D100200246C1B221
:107AA8006B1E994219DA21448B7E0821DBB283EAE6
:107AB8000206F60744BF83F01803C3F3460301F137
:107AC800FF3154BF5B0843F0800311F0FF01C2F39C
:107AD8004702ECD101301A46E1E723449B7E9A42E3
:107AE80002D10320FFF722FF002384F8B93084F87D
:107AF800B83070BDC814002010B5044605F062F80F
:107B08000F4BD3F8BC20C3F8BC00821A41F288316D
:107B18008A42C3F8C02084BF002283F8C42093F8A7
:107B2800C420074913440F2AE4B218BF013283F86E
:107B3800C54012BF81F8C420012381F8D53010BD9B
:107B4800C814002010B5044605F03CF80F4BD3F8D4
:107B5800D820C3F8D800821A41F288318A42C3F883
:107B6800DC2084BF002283F8E02093F8E020074956
:107B78001344142A18BF013283F8E14012BF81F878
:107B8800E020012381F8F63010BD00BFC8140020A2
:107B98002DE9F843324F3D682A8A2E7AB2B9042E6D
:107BA80014D1304C30482378012B0BD12F4B196856
:107BB8002F4B89B20B445B0019681A60302303808D
:107BC800227048E010230380072644E0AC8AAB69A2
:107BD800A24294BF04260226944228BF14461FFAE4
:107BE80084F840469847214A13689BB203F1005332
:107BF80003F540535B0004F1010E1B689BB203F1CF
:107C0800005303F540534FEA6E0E5B0000217145A7
:107C180000F1020009D010F8019C10F802CC4CEADF
:107C2800092C23F821C00131F1E71268104B92B2F8
:107C380013445B001A681C602B8AC8EB03032B8271
:107C48006B8A9844084BA5F8128030221A80094B99
:107C58004FF440521A803B681E72BDE8F88300BF9B
:107C680034220020C42F0020BE1F0020505C00409A
:107C780002300020BC1F00200E4B0F4A1B689BB22D
:107C880003EBC00002443E294FEA420209D94B09DE
:107C9800C80604BF03F1FF339BB29B0243F40043C1
:107CA80004E04B08C90748BF01339B021168136001
:107CB800704700BF505C00400630002010B5454BAF
:107CC8001A68107810F07F0004D1537A23F020034B
:107CD800537210BD02287AD15388002B78D11379BA
:107CE800002B75D1537923F08000840004F1804182
:107CF80001F5B84113F0800F096814BF01F0300195
:107D080001F44051032862D8002960D0927A002AF1
:107D18005DD004F1804404F5B8441906226825D5DD
:107D280002F03002102A4CD103F07F039B0003F1CC
:107D3800804303F5B8431A68510641BF196840F6F5
:107D48000F720A4042F4004244BF42F0C0021A6077
:107D58001A6822F4E04222F0400292B282F0300225
:107D680042F4004242F080021A602AE002F44052D3
:107D7800B2F5805F25D128B9174B93F82C10FFF77F
:107D88007BFF11E09B0003F1804303F5B8431A68B9
:107D9800520441BF196840F60F720A4042F440424B
:107DA80044BF42F080021A60236823F4804323F022
:107DB80070039BB283F4405343F4004343F08003C1
:107DC8002360064B1B685B699847002010BD0220A2
:107DD80010BD00BF34220020A8000020C41F0020CE
:107DE800002303604360836083810361436183618F
:107DF800C36103624362836270478A68036810B58F
:107E08000C6A14430A6914434A6914438A6914437F
:107E1800CA6914434A6A14438A6A23F4FF4323F065
:107E280070032243134303608B8943600B688360AC
:107E38004B68C36010BD02684FF6FE7313400360C1
:107E48000023036043608360C360294B984201D1DB
:107E5800284A27E0284B984201D1264A2AE0274B96
:107E6800984201D1234A2DE0254B984201D1214A5D
:107E780030E0244B984201D11E4A33E0224B98420D
:107E880004D11C4A536843F470032EE01F4B9842F8
:107E980004D1184A536843F0706326E01C4B98429B
:107EA80004D11C4A536843F00F031EE01A4B984252
:107EB80004D1184A536843F0F00316E0174B984270
:107EC80004D1144A536843F470630EE0144B98428B
:107ED80004D1104A536843F4704306E0114B9842AA
:107EE80004D10C4A536843F470235360704700BFB1
:107EF80008000240000002401C000240300002401E
:107F080044000240580002406C00024080000240D9
:107F180008040240000402401C04024030040240ED
:107F28004404024058040240084BDA68D10709D4D7
:107F3800DA68D20608D4DB6813F0040F14BF0320F4
:107F4800042070470120704702207047002002403B
:107F5800036A23F001030362036A70B54468826907
:107F68000D6822F4803222F0730215438A8923F0C7
:107F7800020313438A881343134A90420FD002F531
:107F8800006290420BD002F54062904207D002F5A1
:107F98008062904203D002F5806290420DD1CA8976
:107FA800CE8823F0080313430A8A24F44074144348
:107FB8004A8A23F00403334314438A684460856182
:107FC8004263036270BD00BF002C0140994A5368A8
:107FD80003F00C03042B2DE9F04105D0082B06D043
:107FE80095490160B3B916E0934B036012E05368FA
:107FF8005468C3F38343991CE30349BFD36A8F4B87
:108008008D4C03F00F0344BF0133B4FBF3F34B4330
:10801800036000E000235168894FC1F303117D5CC0
:108028000168EDB221FA05F444605668C6F30226E9
:10803800BE5D24FA06FEC0F808E05668C6F3C226FC
:10804800BE5DF6B2F440C460D2F82C80C8F30418C0
:1080580008F00F0C07EB4C0C18F0100FBCF810C010
:108068001FFA8CFC07D0BCF1000F04D0B3FBFCFC5A
:10807800C0F810C000E00161D2F82CC0CCF3442C49
:108088000CF00F0807EB48071CF0100F3F8ABFB22F
:1080980004D01FB1B3FBF7F7476100E04161176BEC
:1080A800FF065ABF644F87618161176BBF065ABFCD
:1080B800614FC761C161176B7F065ABF5E4F076288
:1080C8000162176BFF0506D5994204D1AE4202D171
:1080D8004F00476200E04462176BFF0406D59942DF
:1080E80004D1AE4202D14F00876200E08462176B70
:1080F800BF0506D5994204D1AE4202D14F00C762EE
:1081080000E0C462176B7F0506D5994204D1AE42E0
:1081180002D14F00476400E04464176B3F0506D561
:10812800994204D1AE4202D14F00876400E08464D2
:10813800176BBF0406D5994204D1AE4202D14B0059
:10814800C36400E08464156B3A4BAD0701D1046346
:1081580015E01C6B04F00304012C01D101630EE04F
:108168001C6B04F00304022C02D14FF4004305E019
:108178001B6B03F00303032B01D12F4B0363146B19
:108188002C4B14F4403F02D1C0F834E018E01C6BCB
:1081980004F44034B4F5803F01D1416310E01C6B16
:1081A80004F44034B4F5003F02D14FF4004306E034
:1081B8001B6B03F44033B3F5403F01D11E4B4363BF
:1081C800146B1C4B14F4402F02D1C0F838E018E0AF
:1081D8001C6B04F44024B4F5802F01D1816310E0B6
:1081E8001C6B04F44024B4F5002F02D14FF4004373
:1081F80006E01B6B03F44023B3F5402F01D10E4B6F
:108208008363146B0B4B14F4401F02D1C0F83CE09D
:1082180020E01C6B04F44014B4F5801F01D1C16345
:1082280018E01C6B04F44014B4F5001F0AD14FF495
:1082380000430EE00010024000127A0000093D00E1
:10824800080000201B6B03F44013B3F5401F01D155
:10825800134BC363126B134B12F4400F03D1C0F8D6
:1082680040E0BDE8F0811A6B02F44002B2F5800FDD
:1082780002D10164BDE8F0811A6B02F44002B2F544
:10828800000F02D14FF4004306E01B6B03F44003D8
:10829800B3F5400F01D1024B0364BDE8F08100BF84
:1082A80000127A0000100240F0B500230E681C4648
:1082B8000125A54005EA060EAE452BD10F797A1E99
:1082C800012A15D8856803229A4025EA02028260AD
:1082D8004D7982689D4015438560828892B222EA72
:1082E8000E0282808A798588A2402A4392B28280CF
:1082F800032205689A40D2431540056005689F40EF
:108308002F430760C7681740CA7902FA03F547EA9E
:108318000502C2600134102C03F10203C8D1F0BD7C
:1083280038B52DED048B4A4C0368C4F8F8308388BF
:10833800A4F8FC30013A0D46072A42D8DFE802F0DB
:10834800040A101822292F35B4F8F8300B80B4F835
:10835800FA3013E0B4F8FA300B80B4F8F83005E0DE
:10836800B4F8F8305B420B80B4F8FA305B4205E0B1
:10837800B4F8FA305B420B80B4F8F8306B80B4F88C
:10838800FC301DE0B4F8F8305B420B80B4F8FA30EA
:1083980012E0B4F8FA300B80B4F8F8300CE0B4F816
:1083A800F8300B80B4F8FA3005E0B4F8FA305B42E4
:1083B8000B80B4F8F8305B426B80B4F8FC305B4259
:1083C800AB80244B93F83030002B3ED1B5F9003008
:1083D80094ED430AD4ED407A09EE103AB5F902302B
:1083E80008EE103AB8EEC88AB5F90430B8EEC99A62
:1083F80028EE000A08EE903AA7EE890AF8EEE88A15
:10840800D4ED467AA7EEA80A0DF03CFD94ED440A97
:10841800D4ED417A288028EE000AA7EE890AD4ED27
:10842800477AA7EEA80A0DF02DFD94ED450AD4ED84
:10843800427A688028EE000AA7EE890AD4ED487AC5
:10844800A7EEA80A0DF01EFDA880BDEC048B38BD70
:10845800C814002008000020104BDFED117A1B68BB
:108468009A89104B1B6883F31003D31A07EE103A4E
:10847800B8EEC77A27EE277A07EE902AF8EEE77A61
:10848800C7EE277AFDEEE77A17EE900A6428A8BFB0
:10849800642020EAE070C0B2704700BF5812002084
:1084A8000000C84268120020094B1A68137844F685
:1084B800FB7103EB431300FB03135078C0EB003050
:1084C800B3FBF0F39078B3FBF0F080B2704700BFD5
:1084D8005812002008B50A4890F8253100EB4303EC
:1084E8000A22B3F8341189B2A0F83C1100F5A07043
:1084F80004F025FD80B2FFF7D7FF024B188008BDB6
:10850800C81400205C1200202E4B2F4A1B681268EA
:1085180010B51A602D4A1168596051689268DA607E
:108528002B4A996011681961516892689A61294AC1
:1085380059611168D961516892685A62264A19626C
:1085480011881985518859859188D288DA85234AF6
:108558009985118819865188598692889A86204A61
:108568001188D986518819871946928821F83A2F97
:108578001C4A10780022824206DA1B4C34F812405A
:1085880021F8024F0132F6E7184A1288A3F864204E
:10859800174A1288A3F86620164A1188A3F86C10A7
:1085A80051889288A3F87020134AA3F86E101268B5
:1085B8009A66124A1288A3F87220114A5289A3F8BF
:1085C8005E2010BD282D0020A02F00205020002064
:1085D8005C2000206820002050120020901100200C
:1085E8003A1200206C180020B01100200416002058
:1085F800441000209611002044120020CC110020C5
:108608009C1100202DE9F8430E4B93E880030546A2
:108618000E460024B44213DA7B1933F9140008EB30
:10862800050333F9142009EB050333F91430134417
:10863800022293FBF2F3C01A09F02DFA0134E9E79C
:10864800BDE8F883282D002070B5472009F072F99D
:10865800174B1B681B0307D5164B174A5B68106836
:108668001B68C01A09F008FA144E154C154D3078DD
:1086780009F002FA23682868C01A09F00CFA63683E
:108688006868C01A09F007FA0F4B188809F0F4F95E
:108698000E4B188809F0F0F90D4B188809F0ECF921
:1086A800337823742B68A3606B68E36070BD00BFE8
:1086B800942E0020282D0020A02F002076120020C4
:1086C800142D00207812002074120020721200204D
:1086D800D41100207FB5254C254E264D2649274A22
:1086E800274B20B127480088B0F5805F30D230880A
:1086F800ADF8040028781D4D897912788DF80600A8
:108708008DF807108DF808201B788DF8093001A81E
:10871800294606220DF08CF928B30198BDF80830D7
:108728002860AB80532009F005F9208809F0A4F9E6
:10873800A07809F0A1F9E37801932379029301A8BD
:108748006379039309F0FEF80E4B00221A800AE0C1
:10875800308820808979287812781B78A070E17099
:1087680022716371DEE704B070BD00BF901600206F
:108778003413002070120020940E0020C30E002035
:10878800280F0020B42E0020A0F17D03012B70B526
:1087980004460D460A4E05D830687D2104F0CCFB0E
:1087A80084F020043068214604F0C6FB35B12B88DC
:1087B8001C4404EB142404F0FF042C8070BD00BF9B
:1087C800241300200A4A138801331380094A1368C6
:1087D80001331360084A138801339BB2202B01BF71
:1087E80000231380054A138808BF0133138070479C
:1087F800B42E00209C2E0020A02E0020A22E0020A7
:1088080038B53A4B1B78083B012B05460C466BD80C
:10881800452009F08FF8284609F08CF80C2D23D054
:1088280004D80A2D0AD014D835B138BD0E2D4BD036
:108838002ED3FF2D50D038BD206849E0207809F0AC
:1088480079F862796378002A14BF802000201843E1
:1088580000E0207809F06EF8A07809F06BF8E0786D
:1088680009F068F820793BE0B4F9000009F0FAF85B
:10887800A07809F05FF8E07809F05CF8B4F9040032
:1088880009F0F0F8B4F90600BDE8384009F0EAB894
:10889800637820788BB180F0800009F04BF8A468E9
:1088A800E0B209F047F8C4F3072009F043F8C4F32D
:1088B800074009F03FF8200E12E009F03BF8606825
:1088C800BDE8384009F0E7B8206809F0D5F86068D5
:1088D800BDE8384009F0D0B8054809F009F800208B
:1088E800BDE8384009F026B838BD00BF042D002087
:1088F800D2A501082DE9F04FB74BB84F1A888BB0B5
:108908000193002A40F0A380B7F8D207B44E42F290
:108918000103C21A50425041FFF7DCFEFFF7F4FD95
:108928003468492009F006F8AE4B2546186809F066
:10893800A3F855F8040B09F09FF8284607F0AAFC9D
:1089480004F1100007F0A6FC04F11C094FF0100810
:10895800A54D01232A6803FA08F3134203D0D9F876
:10896800000009F098F808F10108B8F1130F09F1AF
:108978000409EDD104F1280007F07CFCB7F8443174
:10898800B4F92E00C01A09F077F82B68DB0408D573
:10899800964BB4F864001B88181AC0F30D0009F050
:1089A8006BF82B68980403D5B4F8660009F064F8EE
:1089B8002B68590503D504F16C0007F05BFC2B68A4
:1089C8001A0502D5A06E09F066F82B681B0403D5BA
:1089D800B4F8720009F050F804F13000A04607F02E
:1089E80049FC04F1360007F045FCB7F8443138F982
:1089F8003C0FC01A09F040F801277D4B1B789F42B5
:108A080008DA38F9020FB4F93C30C01A09F043F813
:108A18000137F2E72B68980505D5B4F95E00A0F296
:108A2800DC5009F038F8326872487260B260121A85
:108A38009110714A4A43531C032293FBF2F202EB52
:108A480042029A1A742303FB02033360C9E16B4B99
:108A58006B4A1B6811688B4206D00AA9002041F8AE
:108A6800203D1360FFF7CCFE019B97F8D2171B88B7
:108A780097F8D3070B44013BB3FBF0F200FB12332A
:108A88008B4280F07981564C0120FFF723FEFFF7D7
:108A98003BFD50202668656808F04CFFA2682368F3
:108AA80010681B68626803441068A3EB400008F074
:108AB800F2FF6A6873689B1A0293AA68B3689B1AE4
:108AC8000393EA68F36802A89B1A049307F0E2FB91
:108AD8002A6933699B1A02936A6973699B1A03931B
:108AE800B369AA6902A89B1A049308F02BFF06F140
:108AF8001C0905F11C0B1027A0463B4801210368FF
:108B0800B9401942824606D0D9F80000DBF8003097
:108B1800C01A08F0C0FF0137132F09F104090BF13F
:108B2800040BEAD106F1260005F12601002331F9EC
:108B3800024F30F9022F121B02AC44F823200133F4
:108B4800042BF4D10322002702ABBF0053F82230D4
:108B5800FFB26BB103F108010F2902D847F00107F2
:108B680006E08033FF2B94BF47F0020747F0030766
:108B780012F1FF32E8D2384608F0DCFE00240DF18D
:108B88000809A34607F00302022A10D0032A17D0C7
:108B9800012A4AD1BBF1000F41D0D9F8000000F0FA
:108BA8000F00204308F0C6FE4FF0000B3DE0BBF17C
:108BB800000F0CD0D9F80000C0F3031020432CE0BC
:108BC800BBF1000F1ED199F8010008F0B3FE99F827
:108BD800000008F0AFFE28E0A02E00202C25002081
:108BE800282D00209C2E0020942E0020902E00205E
:108BF8006C180020342D002035C2724FA82E00209A
:108C0800A42E0020D9F80000C0F30330204308F058
:108C180091FED9F80000C0F3071008F08BFED9F8D0
:108C280000402401E4B24FF0010B09F1040906AB3E
:108C380099454FEA9707A5D1BBF1010F02D120460C
:108C480008F078FEDAF8003013F480541FBFB6F845
:108C58006420B5F86410521A029218BF01249904CE
:108C68000AD50AAA02EB8401B5F86600B6F86620B0
:108C7800121A41F8202C01345A0513D502AA02EB26
:108C8800840E06F16A0705F16A00002237F9021F0F
:108C980030F902CFCCEB01014EF822100132032A41
:108CA800F4D103341F0508D50AAA02EB8400A96E83
:108CB800B26E521A40F8202C013418040BD50AABB6
:108CC80003EB8402B5F87210B6F872305B1A42F8FA
:108CD800203C013400E0F4B1012C03D1029808F0E3
:108CE800DAFE18E0631E002002AA400052F8232092
:108CF800C0B20AB140F0010013F1FF33F4D208F01A
:108D080019FE002702AB53F8270008B108F0C3FE8C
:108D18000137A742F6DB30200321FFF773FC36202A
:108D28000321FFF76FFC314B3C201978FFF76AFCF1
:108D3800DAF80030990506D5B6F95E00B5F95E3067
:108D4800C01A08F0A8FED8F800202948D8F804303E
:108D5800C8F80420121A9110264AC8F808304A4365
:108D6800531C032293FBF2F202EB42029A1A742379
:108D780003FB0203C8F800301F4B1B681A0630D5E6
:108D88001E4C1F4D22682B689A420BD162686B6893
:108D98009A4207D1019B1B88102B11D1194B1B88B4
:108DA8005B060DD1482008F0C5FD206808F073FE69
:108DB800606808F070FE23682B6063686B600EE0E3
:108DC800114A0F4B11782A7C914208D10F4A9968B1
:108DD8001068884203D15268DB689A4201D0FFF7D5
:108DE80033FC08F077FD0BB0BDE8F08F6C1800205D
:108DF800342D002035C2724FCC240020D811002019
:108E0800142D0020A22E00207612002078120020B7
:108E18002DE9F84F0C9E3A4CC2EB030B0B9BF61A4C
:108E28006368002914BF4FF0060A4FF0040A0133A3
:108E38000546904613D1236853455ED2314A3248DD
:108E480052F82320032B98BF294608F061FD636878
:108E5800013363602D4B002205469A7113E000250B
:108E680011E02B4A1278954240DA0B9BE3B109FBDB
:108E780006F2995C01228A40264909680A4213D100
:108E8800636801336360D4F804900A9B1C4F9945CA
:108E9800E7DB2BD10A2008F04DFD3B6801333B602E
:108EA8004FF0FF337B6021E0184A917921B12C20E3
:108EB80008F040FD013501E001219171226809FBAC
:108EC8000BF308EB030752B958F8030008F010FD3C
:108ED80097F904104B1C0544D2D00F4802E03A44DD
:108EE8000E48117908F014FD0544C9E7206850457B
:108EF8002CBF00200120BDE8F88F0020BDE8F88FC6
:108F0800AC2E002010840108DDA501089016002071
:108F180008010020942E0020ECA5010820A70108D4
:108F280030B585B004AC002524F8025D0091ADF899
:108F3800060021461020FFF727FC9DF80600214671
:108F4800FFF722FC9DF807002146FFF71DFC9DF85E
:108F580000002146FFF718FC9DF801002146FFF7A5
:108F680013FC9DF802002146FFF70EFC9DF8030054
:108F78002146FFF709FC9DF80E00C043C0B2294600
:108F8800FFF702FC05B030BD10B5054C206803F0B2
:108F9800D0FF18B1206803F0C9FFF6E710BD00BF85
:108FA800F412002013B5044601A9006802F0BAF9CA
:108FB800132002F0F3F9BDF9040002F0DDF91B20DB
:108FC80002F0ECF9BDF9060002F0D6F9232002F010
:108FD800E5F92368002BB4BF53204E2002F0CCF9EA
:108FE80001A9606802F09EF9122002F0D7F9BDF9D4
:108FF800040002F0C1F91A2002F0D0F9BDF9060008
:1090080002F0BAF9222002F0C9F96368002BB4BF54
:109018005720452002F0B0F902B010BDF0B5012488
:10902800B0FBF4F58D4201D34C43F9E70026D4B1E7
:10903800B0FBF4F504FB1500B4FBF1F41EB9002DE8
:1090480001DC002CF3D1092D03F1010EEFB204DD90
:10905800002A14BF3725572500E030253D441D70F0
:1090680001367346E3E71C70F0BDF0B50124B0FB90
:10907800F4F58D4201D34C43F9E70026D4B1B0FB97
:10908800F4F504FB1500B4FBF1F41EB9002D01DC66
:10909800002CF3D1092D03F1010EEFB204DD002AF3
:1090A80014BF3725572500E030253D441D70013693
:1090B8007346E3E71C70F0BD03685A1C0260197020
:1090C80070472DE9F843089E002B0746884614464A
:1090D80014BF4FF030094FF02009334613F8012B25
:1090E8000AB9254603E0002CFBDD013CF6E7002D1C
:1090F80004DD38464946C047013DF8E724EAE474F0
:109108003546A01B284415F8011B11B13846C04745
:10911800F7E7BDE8F883024B186803F00DBF00BFFE
:109128005010002090ED017A07EE901AB5EE407AC3
:10913800F1EE10FA01BFF8EEE77A9FED0E7A67EECE
:10914800877AB7EE007A04BFC7EE277AC0ED017AB6
:1091580090ED017AD0ED007A30EE877A30EE670A2A
:10916800C0EE870AE0EE807AB0EE670AC0ED007ABA
:10917800704700BFDB0FC94010B50278202A0346AC
:1091880000F10100F9D0092AF7D02D2A03D10346AE
:10919800BFEE000A04E02B2A08BF0346B7EE000A18
:1091A800DFED387A1A46134612F8010BA0F13001A8
:1091B800CCB2092C0AD807EE101AB8EEC77AF2EE2C
:1091C800046AA7EEA67AF0EE477AECE72E2816D1C5
:1091D800F2EE046A1146B0EE666A0B4611F8012BEE
:1091E800303AD0B209280AD807EE102AB8EEC77A62
:1091F80087EE267A66EE866A77EE877AEDE71A7842
:1092080002F0DF02452A35D15A782D2A02D10233DD
:10921800012004E02B2A14BF013302330020013B54
:10922800002213F8011F3039CCB2092C03D80A24C4
:1092380004FB0212F5E7B2F59A7F28BF4FF49A7241
:109248001346B7EE007A072B05D9DFED0F6A083B06
:1092580027EE267AF7E702F007032BB1F2EE046A4D
:1092680027EE267A013BF8E7F0EE476A20B1C7EE11
:10927800877A03E0F7EE006A67EEA67A20EE270AFF
:1092880010BD00BF0000000020BCBE4C30B52DED65
:10929800028B87B0B0EE408A0C220021054603A855
:1092A8000CF0E1FBB5EEC08ADFED2A7AF1EE10FA98
:1092B800CCBF38EE278A38EE678ADFED277A28EEAA
:1092C800278A6946FDEEC87A17EE904A84EAE47068
:1092D800A0EBE47008F06AFE002CACBF20232D231D
:1092E80068468DF80C300CF002FC012807D13023B9
:1092F8008DF80D308DF80E308DF80F300CE0022807
:1093080005D130238DF80D308DF80E3004E0032898
:1093180004BF30238DF80D30694603A80CF0CAFB52
:1093280003A80CF0E4FB0338C4B2224603A928467C
:109338000CF00AFC00232B55284608490CF0BAFB10
:1093480003AB284619190CF0B5FB284607B0BDEC4D
:10935800028B30BD6F12033A00007A4410A6010850
:1093680070B5064615460846B6FBF2F414B1204619
:10937800FFF7F6FF05FB1464024B1B5D00F8013B89
:1093880070BD00BF12A601082DE9F04F814689B0D3
:109398008A4616461C4600253178002900F0DD80F3
:1093A800252902D00136484675E07278302A08BF70
:1093B800B278A2F1300319BFB71C4FF0000BF71CAD
:1093C8004FF0010B092B4FF0000819D8A2F1300318
:1093D800D9B2092905D80A2202FB083817F8012B47
:1093E800F4E7A2F16103052B02D8A2F1570305E0C7
:1093F800A2F14103052B03D8A2F137030A2BEADDBA
:109408006C2A31D13A78642A07F1010600F083808A
:109418000BD8252A3DD003D8002A00F09E80BBE750
:10942800582A0CD0632A19D0B6E7732A22D002D85A
:109438006E2A37D0B0E7752A5CD0782AACD1271DC0
:109448002068A2F1580462424FF01001624155E0D1
:109458002CD9582A32D0632A2AD13E464846217848
:10946800271DD04701350FE0642A64D00ED9732A2E
:1094780014D13E462368009348465146424600238D
:10948800FFF71FFE271D05443C4685E7252ADFD147
:109498003E4648462521D04701357DE70AD86E2A41
:1094A80006D13E46236804341D6075E7002A54D06F
:1094B8003E4671E7752A26D0782AF9D1A2F15803D9
:1094C80004F1040C5A422068CDF80CC04FF010018A
:1094D8005A4105ABFFF7A2FDDDF80CC03E466446D5
:1094E80005AB00934846514642465B46FFF7E9FD07
:1094F800054451E72068271D0A21002205ABFFF724
:10950800B4FD3C46ECE704F1040CCDF80CC020682F
:109518000A210022DDE72068002804F1040708DAA0
:109528002D238DF8143040420DF115030A21002235
:10953800E5E705ABFAE72068002804F1040C0ADA2D
:109548002D238DF8143040420DF11503CDF80CC0D1
:109558000A210022BEE705ABF8E7284609B0BDE8B6
:10956800F08F0EB40FB505AB019053F8042B0649E4
:10957800039301A8FFF708FF019B00221A7004B0AB
:109588005DF804EB03B07047C19000080FB413B541
:109598000B4904AB08680B4953F8042B096801937D
:1095A800FFF7F2FE0446084B186803F0B9FC0028E0
:1095B800F9D0204602B0BDE8104004B0704700BFA3
:1095C8007C010020780100205010002080EAE07320
:1095D800A3EBE0738B4206DB002801DD401A7047DD
:1095E80002D00844704700207047FDEEC07A17EE9D
:1095F800903A2033402B43D8DFED237AB4EEE70AC4
:10960800F1EE10FA04DDDFED217A30EE670AF3E7B8
:10961800DFED1F7AB4EEE70AF1EE10FA04D5DFEDBC
:109628001B7A30EE270AF3E7DFED1A7AB4EEE70A81
:10963800F1EE10FA04DD30EE670A37EEC00A0AE0F0
:109648009FED157AB4EEC70AF1EE10FA44BF30EE7A
:10965800270A37EE400A60EE007ADFED106A9FEDC8
:10966800107AA7EEA67ADFED0F6AE7EE876A9FED1C
:109678000E7AA7EEA67A20EE276AA6EE070A7047AA
:109688009FED0A0A704700BFDB0F4940DB0FC94056
:10969800DB0F49C0DB0FC93FDB0FC9BF9A7C2E36F1
:1096A800FAAF4FB93587083CA4AA2ABE00000000CB
:1096B800DFED027A30EE270A97E700BFDB0FC93FDC
:1096C80038B52DED068B90ED008AB0EE480A0C46B1
:1096D8000546FFF7EDFFB0EE40AAB0EE480AFFF7E7
:1096E80084FFD5ED018AB0EE409AB0EE680AFFF724
:1096F800DFFFB0EE408AB0EE680AFFF776FFD5EDDF
:1097080002AAF0EE408AB0EE6A0AFFF7D1FFF0EE47
:10971800409AB0EE6A0AFFF768FF60EE0A6A69EEDF
:10972800297AF0EE665AE7EEA85A29EE8A6A29EEF7
:10973800007A69EE889A29EE489A28EE400A28EEBF
:109748000A8AC4ED035AF0EE465AE7EE685AE6EE86
:10975800A87AA6EE687AC4ED009AC4ED028A84ED70
:10976800059A84ED088ABDEC068B84ED010AC4EDE8
:10977800045A84ED067AC4ED077A38BD10B52DED8C
:10978800048B8AB090ED009AD0ED028A90ED018AA0
:109798000446084601A9FFF793FFDDED047A9DED25
:1097A800017A68EE277AE9EE077A9DED077AE8EE06
:1097B800877A9DED027AC4ED007ADDED057A68EED0
:1097C800277AE9EE077A9DED087AE8EE877AC4ED04
:1097D800017ADDED067A28EE278ADDED037AA9EE17
:1097E800278ADDED097AA8EEA78A84ED028A0AB0F5
:1097F800BDEC048B10BD074B1A8822EA000090428A
:1098080010B518801C4602D0012003F0C3F9208847
:1098180010BD00BF34130020064B1A881043904235
:1098280010B518801C4602D0012003F0B3F9208837
:1098380010BD00BF34130020024A936823EA0000D9
:10984800906070472C25002008B5104B1A7800232B
:10985800D9B2914207D20E4951F823100968002065
:1098680008600133F4E7322003F0D3F9094B1B6891
:109878005A0309D5084B9B685B0305D440F2DC50BA
:10988800BDE8084003F0C5B908BD00BF6C1800204A
:109898003C180020CC2400202C250020454A6923B0
:1098A8002DE9F34113704FF4FB635380BE2313710A
:1098B800EF2382F8D537002382F8D63719461646A3
:1098C800F25C0133B3F5FB6F81EA0201F8D1394B41
:1098D80083F8D617384B1A69120604D5374A5A60E6
:1098E80002F188325A6004270020013F17F0FF0771
:1098F8004FD0314B3422DA60002444B1002356F8AB
:109908000480019306F040FD0428EED117E006F02C
:109918003BFD0428E9D1284D2B6943F002032B6154
:10992800274B6B612B6943F040032B6106F02CFD3C
:109938002B69042823F002032B61DFD0D5E71E4DE5
:109948002B6943F001032B6104F1006303F57E33B7
:109958001FFA88F21A8006F017FD042810D1194B57
:1099680023440193019B4FEA1848A3F8008006F0AE
:109978000BFD2B69042823F001032B6105D0B4E704
:109988002B6923F001032B61AFE70434B4F5FB6FB7
:10999800B3D1094A1369042843F08003136102D143
:1099A80007F0D8FC10B90A2003F078FA02B0BDE835
:1099B800F08100BF2C2500200020024023016745CC
:1099C80000F8030802F8030810B50E4C206803F0ED
:1099D80033F82068047A002202FB02F3193B634340
:1099E80003F6C4135343192193FBF1F3064921F8F5
:1099F80012300132072AEFD10449BDE8104002F0C5
:109A0800D1BF00BFD01100202010002070260020F8
:109A18002DE9F04107F09EFC10B90A2003F03EFA48
:109A2800A44CA549A54D4FF4FB6220460CF010F854
:109A380094F8AC37022B84BF002384F8AC3794F831
:109A4800AC274FF4CC7101FB02F3E018234400F576
:109A58003970286093F8380303F54C73022801FB2A
:109A6800024284BF0020187292F83833944A137067
:109A78000C2202FB0343934A03F2AE731360A368FC
:109A880046F209021A401AB98A4A43F4005393600D
:109A9800A368D80703D54FF40050FFF7CDFEA3689D
:109AA800590409D50820FFF7C7FE4FF40050FFF707
:109AB800C3FE0120FFF7C0FEA3681A0706D54FF4BE
:109AC8000050FFF7B9FE0120FFF7B6FEA3689B041C
:109AD80002D54020FFF7B0FE94F8DC21754B2AB17F
:109AE80093F8E02112B1002283F8E021764B774EFB
:109AF8001E604FF0000C674604EB0C03B3F8F4E16A
:109B08004FEA5E0101F077314FEA9E0303F03333E9
:109B1800C1EB0E00C11A4FEADE0303F01133CB1A72
:109B280003EB23131EF0010803F00F324FF0FF037D
:109B380092FBF3F3C3EB032318BF0137A2EB030334
:109B480018BFFFB2012B0ADD022B40F0B080B8F13C
:109B5800000F00F0AC801EF0BC0F00F0A8800CF1E4
:109B6800080CBCF1200FC7D1013F012F00F29F80E4
:109B7800FFF72AFF302200215548564F0BF073FF9C
:109B8800554BD5F800801F60544B002108F179002F
:109B9800C3F8008002F090FF514B80F0010018706C
:109BA800504B07F126021A604F4B07F1D0021A609A
:109BB80098F8000005F0FAFC28684C4B00F5C572CF
:109BC8001A60FDF759FD4A4BDFED4A6A07F1940226
:109BD8001A60494B00221A809A71484B07F12C02EF
:109BE8001A602B68464A93ED187A03F2191111602E
:109BF800444A03F289111160434A07F108011160D0
:109C0800424A1760424A07F19C011160414A07F134
:109C1800A60111604049536167EE266A0E60B6EEF0
:109C2800007AB4F8661187EE267A101D07EE901AAE
:109C3800B4F86811F8EE677AC2ED027A07EE901A66
:109C480093F85C10117193F87810517194F8DF1142
:109C58001174F8EE677AB3F81611C2ED037A07EEBD
:109C6800901A2E492E4A086003F1640111602D4AAA
:109C78002D4982ED007AF8EEE77A9FED2C7A2C4A8E
:109C88000B60C7EE277A2B499FED2B7A67EE877A10
:109C9800C2ED007A03F168020A60284903F2111341
:109CA8000B60274B1F60274B1A60BDE8F08106F058
:109CB8003FFB5DE72C25002000F80308AC110020CD
:109CC80078230020D01100208C2F0020B6260020F9
:109CD800540F002070260020880F00208C0F0020D1
:109CE800030000208C20002070060020980F002020
:109CF800480F0020DB0F4940940E0020E820002088
:109D0800C0170020C0090020381900203C19002085
:109D1800D408002098160020980900201C21002053
:109D28005421002050210020FC070020000061443D
:109D3800D0080020F00700204C3D0F44C008002048
:109D4800C8080020FC06002008B5FFF7A7FDFFF7AC
:109D58005FFE0120BDE8084002F01CBF08B50848B6
:109D68000BF0C5FEC0B209280246054B04DC0130E1
:109D78002021C0B29954F6E700221A5408BD00BF4A
:109D88004D17002008B507480BF0B1FEC0B21428E3
:109D9800044B04D8421C20211954D0B2F7E7002202
:109DA8001A5408BD4D1700202DE9F74FA74C02F0B3
:109DB80009FF26686568A768861BF643451BC71B0D
:109DC800ED43FF43F60F8046ED0FFF0F2EB93FB965
:109DD800002D00F08682B9462CE04FF0000929E0FA
:109DE800B14627E003EB8A0BBBF802301A050ED404
:109DF80013F4805F1DBF964A9BF801101268954ABC
:109E0800954B14BF52F82120126843F82A20BBF85A
:109E18000230D80516D499050AD5904B1B7813F053
:109E2800040F0CBF8E4A8F4A8B4B126843F82A20C6
:109E380009F10109207B8C495FFA89FA82450B6890
:109E4800D0D326E0894A5046594605F0D3FB884BC3
:109E58001B885A0603D550465946864A16E05807C5
:109E680003D550465946844A10E0190703D5504691
:109E78005946824A0AE09A0703D550465946804A0D
:109E880004E0DB07D4D57F4A5046594605F0B2FBBB
:109E9800CEE7DFF808E20093BEF906307822A3F592
:109EA8007A7353434FF47A7293FBF2F303F22B1352
:109EB80001930022F3465FFA82FE864517D2009B83
:109EC80003EB820EBEF802E01EF4806F0DD0DFF8BF
:109ED8008891019B39F822E040F2671A9E449EFB64
:109EE800FAFC0AFB1CEE29F822E00132E3E74DB345
:109EF80008F5C333A0336360637B544A13BB937381
:109F0800614B1B6813F0020F0AD0DFF894E19EF84A
:109F180000E0BEF1000F03D04FF0010E82F80EE012
:109F2800DA0506D5594B5B791BB1A37B43F00203D5
:109F3800A3734A4B1B7813F0050F02BFA37B43F0B2
:109F48000403A37394F80EE0BEF1000F03D13F4B56
:109F58005B7B002B4FD094F80DC01CF0010FACF1C7
:109F68000C031DD1BCF1030F07D8DFF8E8903C4A79
:109F78001EF0040F08BF4A4600E0364AACF1040C54
:109F8800BCF1070F05D8DFF81CC11EF0010F18BF80
:109F98006246DBB2032B0ED81EF0020F3C4B06E0E4
:109FA800DBB2032B06D82F4B2A4A1EF0020F18BF2C
:109FB8001A4600E0274A4FF0000C5FFA8CF3834200
:109FC8000DD20B6803EB8C035B881B0642BF224B48
:109FD800D2F8009043F82C900CF1010CEDE785B114
:109FE800BEF1000F08D0637B184A0133DBB2142B93
:109FF80006D1002304E025B1637B002BF3D100E0F8
:10A008005373002E52D0234AB2F90250B2F90020FD
:10A01800002DB8BF6D42002A4FF03203B8BF52423C
:10A0280095FBF3F592FBF3F2EDB2D3B2AB4238BF36
:10A038002B46194A13B192FBF3F300E0134643444D
:10A048002360E37B014A7BBB01232EE0B01600208E
:10A05800BC1700204CA101080A0E0020C22F0020C6
:10A0680084A0010874A00108B81F002028840108F2
:10A07800341300202E840108348401083A8401082E
:10A088004084010846840108CC240020940E002056
:10A098008CA0010850120020400D03000825002064
:10A0A800BC12002094A001080023D3738E4D8F4B5F
:10A0B8002D78E27BADB9002F00F00E818C4B267B0A
:10A0C8001A788C4B8C4D93F800C08C4BD3F800E079
:10A0D8000B6802F004020021D2B203EB86060F4699
:10A0E800B5E01AB9864A1A61002508E0854AFAE7F8
:10A0F8000A68AB00D6187688760604D40135EBB228
:10A108008342F5D3D7E7804EB6F90060192E25DDD6
:10A1180012F803E094F814C026690EF00F09E1451F
:10A128000CDCDFF8C8C19CF815C0BCEB1E1FDEBFF5
:10A13800DFF8D8E1D6F800C043F80EC012F803E003
:10A1480094F816C00EF00F09E14533DBDFF89CC127
:10A158009CF815C0BCEB1E1F2CDC26E0193629DA4A
:10A1680012F803E094F814C026690EF00F09E145CF
:10A178000CDCDFF878C19CF817C0BCEB1E1FA2BF2F
:10A18800DFF888E1D6F800C043F80EC012F803E003
:10A1980094F816C00EF00F09E1450BDBDFF84CC14F
:10A1A8009CF817C0BCEB1E1F04DBD6F800E0574E26
:10A1B80043F806E0544EB6F90260192E1BDD12F87A
:10A1C80003C094F814E026690CF00F09F1450CDC83
:10A1D800DFF8189199F81590B9EB1C1FDEBFDFF86E
:10A1E8002CC1D6F8009043F80C90D25C02F00F0C0A
:10A1F800F4451EDD82E7193680DA12F803C094F8B8
:10A2080016E026690CF00F09F1450CDBDFF8DC904D
:10A2180099F81590B9EB1C1FDEBFDFF8F0C0D6F82F
:10A22800009043F80C90D25C02F00F0CF445FFF656
:10A2380065AF94F817E0BEEB121FA2BF334A366829
:10A248009E505BE75888000504D404330435B342B4
:10A25800F8D122E04AB101EB0C0A06209AFBF0F98A
:10A2680000FB19A001280DDC01E057B9012793F87C
:10A2780001900EEB89003EF829A090F80290C07872
:10A2880003E01746002081468246013125F802ACDA
:10A2980085F800906870C9B2D7E7164A1378013B71
:10A2A80013F0FF0308BF06231370114B1B785B07DD
:10A2B80041BFBBF90630A3F57A7303EBC3034FF430
:10A2C8007A7243BF93FBF2F30133DBB20123104AE6
:10A2D80092FBF3F34344A36003B0BDE8F04FFAF7F1
:10A2E8005BBB03B0BDE8F08FC30E0020B0160020A2
:10A2F800C22F00203A0000200C0E0020BC170020BE
:10A3080090A001084CA10108501200200A0E00205C
:10A31800400D03002DE9F04F2DED0A8B89B08046E2
:10A32800059390F85030049102921BB1322BA8BFCC
:10A33800322300E0012307EE903AF8EEE7BADFEDAA
:10A34800A87AA84B9FEDA8CA1B88C7EEABBA002B0A
:10A3580008BF012307EE903AB8EEE7AAA34B039390
:10A368002AEE0CCA1A887BEE8CBA12F0020FCCEED9
:10A378002BBA27D09E4AB2F90030B2F9022083EAFC
:10A38800E37182EAE270A1EBE371A0EBE27088422C
:10A398000446B8BF0C46B4F5E17F16DA88429FED53
:10A3A80095BA05DD002AD8BF524207EE902A04E08C
:10A3B800002BD8BF5B4207EE903AF8EEE77A87EEBB
:10A3C8008BBA04E09FED8CBA01E0B7EE00BADFF873
:10A3D80058A2DFED899ACDF804800AF1080B0AF13A
:10A3E80010070AF11C090024F0EE69AA834931F923
:10A3F80014307F4909EE103AB8EEC99A31F9143091
:10A40800F5EE047A29EE279A08EE103A039BBDEE82
:10A41800C99A1988F8EEC97A9FED799A89074FEA9F
:10A42800440627EE899AB8EEC88A00F081807549FB
:10A4380031F9143007EE903AF8EEE77AB0EE007A88
:10A44800E8EE077A029B5842FDEEE77A17EE901A7B
:10A45800814203DB8B42A8BF0B4618466A49059B1D
:10A46800715E401A33F91410084407EE900AF8EEAA
:10A47800E78A07F085FF48B16449F2EE049A88EE4E
:10A48800A90A085D07F058FB60EE298A98F81C3085
:10A49800DFED5F6A0AEE903A98F8083007EE903AD6
:10A4A800F8EE677AF8EE6AAA68EEA77AB1EE047A4F
:10A4B80067EEA67A2AEE877AFDEEE77A17EE901A0B
:10A4C800F1EE477AFDEEE7AA1AEE903A994208DBD8
:10A4D800FDEEC7AA1AEE903A8B42A8BF0B460AEEC9
:10A4E800903AD9ED007AE8EE8C7ABBEE0E7AF4EE6B
:10A4F800C77AF1EE10FAF8EEEAAA09D4B3EE0E7AAA
:10A50800F4EE477AF1EE10FAC8BFF0EE477A01E0B0
:10A51800F0EE477AC9ED007A98F8123009EE903AD1
:10A52800F8EE699A67EEA97ADFED3A9A67EEA99A8A
:10A53800039B1988CA0779D43048305E0028B8BF11
:10A548004042B0F5206F02DD0020386026E0019B14
:10A558009FED317A5B7868EE077A07EE103AB8EE2D
:10A56800477A87EE877AD7ED007A37EE497AE7EEB1
:10A578000C7A9FED2A7AF4EEC77AF1EE10FA09D434
:10A588009FED277AF4EE477AF1EE10FAC8BFF0EEA5
:10A59800477A01E0F0EE477AC7ED007A019BD7EDE4
:10A5A800007ADB7A08EE903AF8EE688A8B0768EE54
:10A5B800A77ADFED1C8A67EEA88A3BD538EE6A8A4F
:10A5C800F0EE6A7AEBEE087A78EEE98AB0EE678AFE
:10A5D800F0EE697AEBEE287AF0EE678A2AE000BF9F
:10A5E80083F9223E64110020BD37863534130020DC
:10A5F800501200200000E1430000000090110020EC
:10A60800CDCC4C40BA2F0020C22400205C8D01081C
:10A618006F12033C0AD7A33D0000A043000040C3CB
:10A62800000040430AD7233CC8160020F0EE698A90
:10A63800B0EE6A8A89499FED8A7A635C98F851106E
:10A6480007EE903AF8EEE77A67EEC97AA7EE878ABE
:10A6580059B18448844DB0EE480A00EBC400D5EDEA
:10A66800000AFEF75FFDB0EE408A9AED007ADBED56
:10A67800007A7E49AAEC019A39EE477A635C7C4DF0
:10A6880087EE0C7A043709F1040909EE103A37EE1F
:10A69800677AB8EEC99AEBEE877A38EE280AEBECBF
:10A6A800017A67EE897A9FED739A27EE899A30EEE0
:10A6B800490A0BF0E7FBBDEEC88A6F49A85318EEAC
:10A6C800103AFDEEE88AB1EE499A18EE902A41F860
:10A6D8002430BDEEC99A694B694E43F8242019EE1F
:10A6E800102A46F82420019A069101320192079314
:10A6F8000CB901247AE6049A624B9479B3F90430D0
:10A70800640028345C43604BB3F9043000EE103A1F
:10A71800BAEECF0A0BF0B6FB6411201A002C07EE34
:10A72800900AB8BF6442322CF8EEE76A574A02DD55
:10A738000023936026E0BDEECAAA1AEE103A23F071
:10A74800030307EE903AB8EEE7AADFED517A98F8DE
:10A758000D30CAEE277A07EE103AB8EE477A9368BA
:10A7680026EE877A67EE277AFDEEE77A17EE901ADB
:10A778000B4448498B42A8BF0B4647498B42ACBFA4
:10A788009360916093685B13B3F5807FA8BF4FF423
:10A7980080736FF0FF029342B8BF134607EE903AFA
:10A7A800F8EEE78AFDEEE67A98F8032017EE903A7D
:10A7B80053439B1107EE903A384B1B78032BB8EEA6
:10A7C800E78A14D9B8F84E20B2F5FA7F0FD2FDEE19
:10A7D800C87A534217EE901A994204DB914217EE59
:10A7E800903AA8BF134607EE903AB8EEE78A98F871
:10A7F800511081B14B0803D09942A8BF194600E017
:10A808000121194B2648D3ED000AB0EE480AFEF79D
:10A8180089FCB0EE408A78EE287AFDEEE77ACDED35
:10A82800017ABDF80430AB801BB200EE103AB8EEE6
:10A83800C00A0BF027FB069BA880BDEEC88AFDEE78
:10A84800E88A83ED028A079BC3ED028A0023B3607E
:10A8580009B0BDEC0A8BBDE8F08F00BFEC160020F4
:10A86800A69B443BE41F0020FC1F0020EF1600209D
:10A8780048200020F7CC9238502000205C2000208F
:10A888006820002050120020901100200020002095
:10A8980000803B45FEFFFF0F020000F06C1800200F
:10A8A800F41F00202DE9F04F2DED028B87B0002614
:10A8B8000493C14B0391B3F90280B3F900300292BB
:10A8C800B8F1000FB8BFC8F10008002BB8BF5B4251
:10A8D8009845B8BF9846B8F5FA7F0746A8BF4FF421
:10A8E800FA780090B2460196B1463446B34D2B88AB
:10A8F800990757D0B04BB24A33F8143032F91420C4
:10A90800022013FB0022029B5B429A424FEA440159
:10A9180003DB029B9342A8BF1346AA4A31F902B04F
:10A92800049A32F91420CBEB030303EB020B07F074
:10A9380027FD88B107EE90BAA34BB8EEE70AB2EE4E
:10A94800048A185D80EE080A07F0F6F820EE080A77
:10A95800FDEEC07A17EE90BA3B7A642203FB0BF344
:10A9680093FBF2F33A7F6FF0040909FB02F94B45B8
:10A9780004DB02EB82099945A8BF9946934A52F82D
:10A9880024100BEB010342F210718B42A8BF0B4657
:10A998008F498B42B8BF0B4642F82430BA7C5343E8
:10A9A8001B1301932D8805F00303012B38D0824B2C
:10A9B800884933F914A0009B51F824E093F801C0AA
:10A9C800854B33F9140080EAE073A3EBE073B3F529
:10A9D800206F4FEA840616DC0AEB8A031A0192FB01
:10A9E800FCF3042290FBF2F0181A8644BEF57A5F55
:10A9F800A8BF4FF47A5E794B9E45ACBF41F824E07E
:10AA080041F8243002E0002341F824308B597D2698
:10AA180093FBF6F6009BDB7A7343402693FBF6F62E
:10AA2800AA0711D50198C8F5FA7208FB0AF308FBC2
:10AA380006F54FF4FA7102FB093302FB005593FB4C
:10AA4800F1F395FBF1F505E0EB074DBF019D3546A8
:10AA580053464B46604A32F91410042291FBF2F235
:10AA68005F49615C4A436FF04F0192FBF1F297F83E
:10AA7800511013444FEA440B08EE103A59B1594BA0
:10AA88005948D3ED000AB8EEC80A00EBC400FEF737
:10AA980049FBBDEEC08A504B544A3BF803003BF9D2
:10AAA80002302BF8020001B2101D0C32CB1A50F8FC
:10AAB80024E0042193FBF1F152F8243040F82410EB
:10AAC80073440B4497F8501042F824E04FEA840C82
:10AAD80000EE103A79B1434A4548D2ED000ACDF864
:10AAE80014C0B8EEC00A00EBC400FEF71BFBDDF88B
:10AAF80014C0BDEEC00A3F4A3F49125D3F4810EE00
:10AB0800103A5343202293FBF2F318EE102A2A44FA
:10AB1800D21A2BF8012018EE102A4CF80020384AD7
:10AB28004CF80250374D5B424CF80530009B01331E
:10AB380000930CB90124D9E61F4B97F80DE0B3F93F
:10AB48000440039B9B790F335B0063435B11224CEA
:10AB5800002B4FF00406B4F9044094FBF6F41D4EA4
:10AB6800A3EB0404B8BF5B42322BD6F808C00DDC57
:10AB7800254B0EFB04CE7345A8BF7346DFF890E063
:10AB88007345ACBFB360C6F808E001E00023B360CA
:10AB9800FB785C431D4B1B78032B4FEAA4143AD96E
:10ABA800B7F84E30B3F5FA7F35D25F42BC4231DB9D
:10ABB8009C42A8BF1C462EE05012002034130020EF
:10ABC800BA2F0020C22400205C8D0108F416002052
:10ABD800F0D8FFFF002000209011002080C1FFFF67
:10ABE800EC160020FC1F0020E41F0020FC160020AB
:10ABF80030200020EF1600204820002050200020A0
:10AC08005C20002068200020FEFFFF0F6C18002049
:10AC1800020000F03C46B368846043F34F33B3F559
:10AC2800807FA8BF4FF480736FF0FF06B342B8BFB0
:10AC38003346E618936000238E80AB6007B0BDEC06
:10AC4800028BBDE8F08F2DE9F04F2DED028B85B01A
:10AC580083460293B84B01911D88009205F00205C6
:10AC6800ADB295B1B54BB3F90250B3F90030002D30
:10AC7800B8BF6D42002BB8BF5B429D42B8BF1D46AE
:10AC8800B5F5007FA8BF4FF40075D9460026AB4B39
:10AC9800AB4C33F81610AB4B54F8267033F916301A
:10ACA80083EAE37EAEEBE37E08B2BEF5206F4FEA9F
:10ACB800460A4FEA40004FEA860812DC4FF0040EBD
:10ACC80093FBFEF3C31A1F44B7F57A5FA8BF4FF48E
:10ACD8007A579D4B9F42ACBF44F8267044F8263003
:10ACE80002E0002344F8263054F8087099F80B3035
:10ACF80099F80140FF115F438F4B1B8844439B0722
:10AD08004FEAA7174FEAA41456D0904B33F90A30EC
:10AD1800022011FB0031009B5B42994203DB009B40
:10AD28008B42A8BF0B468A493AF90110591A029B6F
:10AD380033F91630CB1808EE103A07F021FB68B14A
:10AD4800B8EEC80A834BB2EE048A80EE080A985D12
:10AD580006F0F2FE20EE080ABDEEC08A7E487F4962
:10AD680058F8003018EE102A42F2107E134473454A
:10AD7800A8BF73468B42B8BF0B4648F800309BF813
:10AD880008109BF81C00514300EB8000C911C0F16A
:10AD9800000E714503DB8142A8BF01468E469BF831
:10ADA80012104B431B13FF1ACEEB04046F436C4382
:10ADB80003EB67270EEB6424624B04213AF9030086
:10ADC80090FBF1F16648805D4143A4EBA1129BF82A
:10ADD800511008EE102A69B16248634C0393B8EE2B
:10ADE800C80A00EBC600D4ED000AFEF79BF9039BE6
:10ADF800BDEEC08A5D4933F80A303AF901002AF8F5
:10AE080001300FFA83FEC0EB0E0E04209EFBF0F01B
:10AE180001F1040E0C3158F80E4058F8013048F88A
:10AE2800014023449BF8501048F80E00034400EEFC
:10AE3800103A59B14C4B4E48D3ED000AB8EEC00A4F
:10AE480000EBC600FEF76EF9BDEEC00A49494A4854
:10AE5800895D4A4C10EE103A18EE102A4B435B11EC
:10AE6800D119C91A2AF8001048F804204449454A5B
:10AE780048F801705B4248F8023009F101090EB93F
:10AE8800012604E72D4B2E4EB3F90450019BD6F84A
:10AE980008E09B790F335B006B435B11294D002B56
:10AEA800B5F904504FF0040795FBF7F7A3EB070734
:10AEB800B8BF5B42322B9BF80D500BDC324B05FBC5
:10AEC80007E5AB42A8BF2B46304DAB42ACBFB360E1
:10AED800B56001E00023B3609BF8035005FB07F35E
:10AEE8002B4D2D78032D4FEAA3130CD9BBF84E50E8
:10AEF800B5F5FA7F07D26F42BB4203DBAB42A8BF6E
:10AF08002B4600E03B46B568A36045F34F35B5F5E1
:10AF1800807FA8BF4FF480756FF0FF06B542B8BFB9
:10AF280035465E19002386808D60936005B0BDECC0
:10AF3800028BBDE8F08F00BF3413002050120020B0
:10AF4800002000209011002080C1FFFFBA2F0020B0
:10AF5800C22400205C8D0108F4160020F0D8FFFF01
:10AF6800EC160020E41F0020FC1F00201017002012
:10AF780030200020EF16002048200020502000201C
:10AF88005C20002068200020FEFFFF0F020000F078
:10AF98006C1800202DE9F04F2DED028B87B00026AC
:10AFA8000493B24B0392B3F90270B3F900300190E5
:10AFB800002FB8BF7F42002BB8BF5B429F42B8BF8B
:10AFC8001F46B7F5FA7F8146A8BF4FF4FA77B04617
:10AFD8000296B3463446A64D2B8899075BD0022CBF
:10AFE80059D0A24BA34A33F8143032F91420022066
:10AFF80013FB0022039B5B429A424FEA440103DBA6
:10B00800039B9342A8BF13469B4A31F902A0049AB6
:10B0180032F91420CAEB030303EB020A07F0B0F974
:10B0280088B107EE90AA954BB8EEE70AB2EE048A0B
:10B03800185D80EE080A06F07FFD20EE080AFDEE96
:10B04800C07A17EE90AA99F80830642203FB0AF335
:10B0580093FBF2F399F81C206FF0040B0BFB02FB37
:10B068005B4504DB02EB820B9B45A8BF9B46844AE9
:10B0780052F8243042F2107153448B42A8BF0B4659
:10B0880080498B42B8BF0B4642F8243099F8122009
:10B0980053431B1302932B8803F00302012A01D1A7
:10B0A800022C3FD17848714A30F9140032F91480E3
:10B0B8007649019A51F824E0567880EAE075A5EBC4
:10B0C800E075B5F5206F4FEA84021EDC022C16D01D
:10B0D80008EB8801090191FBF6F6042190FBF1F0D9
:10B0E800361AB644BEF57A5F68496948A8BF4FF476
:10B0F8007A5E8645ACBF42F801E0505007E088EA26
:10B10800E875A5EBE875642DE2DD002088505F49FD
:10B118007D26525892FBF6F6019AD27A724340265F
:10B1280092FBF6F69A0713D5022C11D00298C7F5B0
:10B13800FA7307FB06F507FB08F203FB0B224FF433
:10B14800FA7103FB005392FBF1F293FBF1F508E06F
:10B15800DB0704D5022C02D0029D5A4601E0354691
:10B168004246494B33F91410042391FBF3F3494940
:10B17800615C4B436FF04F0193FBF1F399F8511069
:10B18800D3184FEA440A08EE103AB1B1022CB8EECF
:10B19800C80A414B08D14A0803D09142A8BF1146BA
:10B1A80000E001213D4802E03D4800EBC400D3ED3A
:10B1B800000AFDF7B7FFBDEEC08A334B394A3AF8AB
:10B1C80003003AF902302AF8020001B202F108003D
:10B1D8001432CB1A50F824E0042193FBF1F152F811
:10B1E800243040F8241073440B4499F8501042F866
:10B1F80024E04FEA840C00EE103A79B1264B2A4835
:10B20800D3ED000ACDF814C0B8EEC00A00EBC400B4
:10B21800FDF788FFDDF814C0BDEEC00A234A2449B3
:10B22800125D10EE103A5343202293FBF2F318EE0E
:10B23800102A2A44D21A2AF801201E4A18EE101A97
:10B248004CF802101C4A4CF802501C4A5B424CF85D
:10B258000230019B01340133032C01937FF4BBAE10
:10B2680007B0BDEC028BBDE8F08F00BF5012002084
:10B2780034130020BA2F0020C22400205C8D01085E
:10B28800F4160020F0D8FFFF9011002000200020C5
:10B2980080C1FFFFEC160020FC1F0020F41F0020D7
:10B2A800E41F00202417002030200020EF16002083
:10B2B80048200020502000205C200020682000202A
:10B2C800022803D0431E584258417047064B1B685A
:10B2D8001B7823B1054B1868C0F3C0407047044B76
:10B2E8001878C0F3800070477006002070110020A5
:10B2F800C22F002010B50A4C5E280146206805D1EF
:10B308005D2101F019FE20683E2105E05D2903D189
:10B3180001F012FE20683D21BDE8104001F00CBE8E
:10B328004417002030B50028104C114AB8BF4042DD
:10B338003C2590FBF2F304FB030068430D4D90FBA2
:10B34800F2F22D682D7B25B903EB830303EB83030E
:10B3580001E0C3EB031302EB83030B8004FB02023F
:10B368004FF47A7392FBF3F24A8030BD806967FF2D
:10B37800809698006012002010B50446C0B2FFF70E
:10B38800B9FFC4F30720BDE81040B3E7024B5E21C4
:10B39800186801F0D1BD00BF4417002038B5064C2D
:10B3A80005465E21206801F0C7FD20682946BDE8F2
:10B3B800384001F0C1BD00BF44170020674B73B58A
:10B3C8001878674DFFF77CFF2B788342044620D01E
:10B3D800C8B1644B1B68E3B193F9000002230093E2
:10B3E800614B1B685B78003318BF0123019304216C
:10B3F8004FF41653002201F016FC5C4B186040B164
:10B4080001232B7005E0594E306802F06AFF346062
:10B418002C70574B574D1878FFF752FF2B78834203
:10B42800044618D088B1544B1B68A3B100220124EC
:10B4380093F9000000944FF496430192082101F01B
:10B44800F2FB4E4B186028B905E04C4E306802F00C
:10B4580048FF34602C704A4B4A4D1878FFF730FF8C
:10B468002B78834204462E4642D0002837D0464BDC
:10B478001A68002A3CD0D37992F90000434C002B7B
:10B4880008BF022302220092002254F823300192BE
:10B49800102101F0C8FB3E4B0546186040B33D4CF7
:10B4A80094F84A30022B0BD094F89620022A01D146
:10B4B8004C3405E023B1002A04F14C0418BF0024E1
:10B4C800354B1C6044B1204600214C220AF0CBFACF
:10B4D8000223256084F84A300123337008E02C4E9B
:10B4E800306805F01BF9306802F0FBFE34602C7000
:10B4F8002A4B2B4D1878FFF7E3FE2B78834204463E
:10B5080029D000B3274B1B682BB3274A93F90000B7
:10B5180012685278002A0CBF0822092203230093DC
:10B5280001924FF461432021002201F07CFB1F4B64
:10B53800186080B11E4A012313702B701D4B1A68C6
:10B548001D4B1A6007E0194E306802F0CAFE184B0E
:10B5580034601C702C7002B070BD00BF78060020EB
:10B5680030120020740600206012002044170020CA
:10B57800790600208012002004130020F412002015
:10B58800840600200A13002080060020608D010830
:10B598000C130020A0220020101300209006002089
:10B5A800201300208C060020880600202413002089
:10B5B80028130020F02400202C130020642928BF21
:10B5C8006421F8B510FB01F56424064695FBF4F4F4
:10B5D8000027E4B2FBB2A34204D29F2005F0F7FC97
:10B5E8000137F7E7B4420BD2C4EB84101421C4EB43
:10B5F800800095FBF1F5663D2844C0B205F0E7FCF4
:10B608000134E4B2B44201D29A20F7E7F8BD2DE93B
:10B61800F743934C01F0D6FA6368C31A002BC0F2C3
:10B62800678300F5433303F5A07363608D4B1D7882
:10B63800237AC5F38005EB1A18BF012325724DB193
:10B64800002B00F05583884B5A789A7001225A7063
:10B658001A702BE0844A2BB1D37843F00203D370DD
:10B6680093785370D67806F0020101F0FF0339B9D8
:10B678007D498968411A002903DB06F0010300E0CF
:10B68800012303F00107784917707BB1F2070DD544
:10B698000A790132D2B20523B2FBF3F303EB830339
:10B6A800D31ADBB2714A0B71D35C4B706E4EDFF864
:10B6B800088233787BB3F37823F00203F3706C4B82
:10B6C8000344AE20B36005F0A6FC08B105F0A8FC61
:10B6D80088F80000002800F00B83B02005F09BFCE0
:10B6E800402005F098FC002005F095FC102005F09E
:10B6F80092FC4FF48067013F0020BFB205F062FC66
:10B70800002FF8D1384605F0FAFC7278594B53F8F7
:10B71800220005F077FC98F80030002B00F0E88252
:10B728007378062B00F2B382DFE813F00700B1024A
:10B73800180078006C018901EE014F494F4A504BBF
:10B748005048FDF70EFF012005F0D9FC4D4805F0E3
:10B7580059FC022005F0D3FC4B48AEE14B4F3B6847
:10B768009B0735D5DFF85481DFF85491B8F80010FD
:10B7780044480A23B1FBF3F203FB121399F80010B3
:10B78800009192B242499BB2FDF7EBFEFEF7FAFA3E
:10B79800012005F0B4FC3B4805F034FC3D4B99F81A
:10B7A80000201868B8F80030067906FB12316423C7
:10B7B8004B43C1788E1B56430220B3FBF6F6F6B214
:10B7C80005F09DFC31461520FFF7F8FE032600E042
:10B7D80001263B681F0540F15A822F4B2F491F68ED
:10B7E8000968009164232E4997FBF3F2254803FB6F
:10B7F8001273FDF7B6FEFEF7C5FA304605F07FFC7A
:10B80800204805F0FFFBFCF727FE0746701C05F0F3
:10B8180076FC15203946FFF7D1FE38E20120214F8A
:10B8280005F06DFC204805F0EDFB3B68980749D50D
:10B838001E4A1448B2F90210B2F900300091B2F968
:10B8480004201B4901921B4AFDF78BFEFEF79AFA6A
:10B85800022005F054FC0B4805F0D4FB032632E027
:10B8680044170020C22F00207C17002037A60108AB
:10B87800404B4C004C8401083CA6010845A6010831
:10B8880085A101084D1700204CA60108CC240020F2
:10B8980053A60108581200206412002068120020E4
:10B8A8006BA601086C12002080A601083A1200203D
:10B8B80096A60108A5A60108E90200205C1200204E
:10B8C800FC00002002263B68D9071AD57C4A7D482F
:10B8D800B2F90210B2F900300091B2F904207A49A5
:10B8E80001927A4AFDF73DFEFEF74CFA304605F024
:10B8F80006FC744806F1010805F084FB5FFA88F835
:10B9080046463B681A0718D5714A6E48B2F90210C4
:10B91800B2F900300091B2F904206B4901926D4AE6
:10B92800FDF71FFEFEF72EFA304605F0E8FB6548E6
:10B93800771C05F067FBFFB23E46674A6249B2F9D9
:10B948000030B2F902200092644A5E48B2F9002041
:10B958000192634A634FFDF704FEFEF713FA30467F
:10B9680005F0CDFB574805F04DFB97ED000A55480B
:10B97800FDF78CFC53480AF0BAF806F101085FFAA3
:10B9880088F8C0B2B946092809D8431C2044DBB25C
:10B9980020224272E218002191721846F3E7494FBB
:10B9A80099ED010A3844FDF771FCFEF7EBF94046C2
:10B9B80005F0A5FB384605F025FB99ED020A384647
:10B9C800FDF764FC38460AF092F80236F6B2C0B2C7
:10B9D800092809D82318421CD2B220215972A31869
:10B9E800002199721046F3E73F4AB2F9003000EEA1
:10B9F800103A3844B8EEC00AFDF748FCFEF7C2F921
:10BA0800304657E00026394F3B78B34240F23F8139
:10BA18000E2E00F03C817008013005F070FB3046B6
:10BA280006F09EFA3B78B34206D9202005F0CFFAFB
:10BA3800701CC0B206F094FA0236F6B2E3E72C4E58
:10BA48002C4996F8AC271F48FDF78BFD012005F01F
:10BA580056FB1C4805F0D6FA274B28491F78194889
:10BA68003A46FDF77EFD022005F049FB154805F032
:10BA7800C9FA0C2303FB0766214996F8AF2796F805
:10BA8800AE371048FDF76DFDFEF77CF9032005F091
:10BA980036FB0C4805F0B6FA96F8B41796F8B227B4
:10BAA80096F8B337074800911649FDF75AFDFEF797
:10BAB80069F9042005F023FB024805F0A3FAE6E043
:10BAC800901100204D17002096A60108A9A601088C
:10BAD8009611002050BC0108C22400204812002002
:10BAE800ADA601082C210020382100203C2300208D
:10BAF8002C250020B1A6010878230020BDA6010846
:10BB0800CEA60108DFA601087B4B1B681B0640F187
:10BB1800BA80236A616A794A8B421FBF536292F8DE
:10BB28002830013303F003034FF001014FF0000008
:10BB380018BF82F8283005F0EEFA94F82830704AD9
:10BB4800D05C05F044FA0220012105F0E4FA002651
:10BB58006C4B9B5D3620C3EBC30393FBF0F0C0B284
:10BB6800062828BF06206038C0B2013605F02FFA33
:10BB7800102EEDD1644B65491B78654813F0020F10
:10BB8800644B1A7814BF59234E23FDF7EAFCFEF7DD
:10BB9800F9F8022005F0B3FA5D4805F033FA5E497A
:10BBA8005E4B4E680A685A4892FBF3F25C4996FB72
:10BBB800F3F3FDF7D6FCFEF7E5F8032005F09FFA4E
:10BBC8005348584E05F01EFA574B58491A885048A2
:10BBD800FDF7C7FCFEF7C2F8042005F090FA4C48C0
:10BBE80005F010FA524B53491A884948FDF7B9FC39
:10BBF800FEF7B4F804210A2005F08DFA444805F050
:10BC080001FA4D49E26A4248FDF7ABFCFEF7A6F897
:10BC1800052005F074FA3E4805F0F4F97268B36837
:10BC280046493B48FDF79DFCFEF798F805210A2098
:10BC380005F071FA364805F0E5F93369F2684049CC
:10BC48003348D21AFDF78DFCFEF788F8062005F078
:10BC580056FA2F4805F0D6F9B2683A492C48FDF74C
:10BC680080FCFEF77BF806210A2005F054FA2848E4
:10BC780005F0C8F934492648152209F065FFFEF792
:10BC88006DF8072016E7F37843F00203F370002DF0
:10BC98002ED12E4B9B79032B9BBF2D4A9B183F25FA
:10BCA8001D7F0021122005F036FA284605F08FF98D
:10BCB8001320002105F02FFA264B1B78002B264B6A
:10BCC8001B7814BF72202120002B18BF522005F0CA
:10BCD8007EF91420002105F01EFA94F83050084B24
:10BCE800585D013505F0030505F071F984F8305009
:10BCF80003B0BDE8F08300BFCC2400204417002027
:10BD0800F1A601081D12002070120020F6A60108F5
:10BD18004D17002076120020781200208096980097
:10BD280007A70108000800207212002014A70108C4
:10BD3800D41100201CA7010823A701082AA701087D
:10BD480033A701083AA7010830030020940E002009
:10BD58004C840108C30E0020280F002038B50024A9
:10BD68000B4D6059254404F0CDFD696811B10948AF
:10BD7800FDF70CFCA96811B10748FDF707FC074857
:10BD8800103404F0BFFDB4F5D87FE9D138BD00BF49
:10BD98006C84010873A7010879A701083AB1010862
:10BDA800F0B585B0044609F0A2FE082826D1621E27
:10BDB800E01D1F4912F8013F09681944497801F04C
:10BDC8000301022908BF203B82421370F1D12546A6
:10BDD80004F1080715F8016B1648314609F079FE99
:10BDE80020B12846314609F074FE10B101F00EFE6C
:10BDF8001CE0BD42EED1204604F0D8FA0E4804F00B
:10BE080081FD00230D4A1A4404A992F88A210A44A4
:10BE18000849595C02F80C1C0133082BF2D10023A5
:10BE280007488DF80C3001A9FDF7B0FB05B0F0BD4F
:10BE38000C0100205DBC01087FA701082C2500200B
:10BE48007CB001082A4B2B4C1E68206880B502F094
:10BE58003DFA304602F03AFA206841798D0704D459
:10BE6800036841F002015B699847234B234D102278
:10BE78009A6120229A612B689A0341BF0623637155
:10BE8800E37923F0010344BF43F00203E371206820
:10BE980001F04FF890B1184F10233B85154B1868E7
:10BEA80001F044F88046FBF733F808B103F06CFC66
:10BEB8003046414601F040F81023BB61304601F09E
:10BEC80038F878B10C4FD4F800904FF02008A7F854
:10BED8002880304601F02AF80146484601F02CF83F
:10BEE800C7F818802B689B03D1D5FFF790FBCEE7E6
:10BEF800942300207817002000040048CC24002058
:10BF08002DE9F047054609F0F2FD314E0446D6F812
:10BF1800088090B92F4804F0F5FC2F4B53F82410F3
:10BF280049B10123A34013EA080F02D02B48FDF7BB
:10BF38002DFB0134F1E72A4822E028462949224608
:10BF480009F0DEFD58B92848284C04F0DBFC54F809
:10BF5800041F0029EFD02148FDF718FBF7E72B78DD
:10BF68002D2B03BF013504F1FF344FF0010A4FF0C8
:10BF7800000A4FF00009184B53F8297027B91C48DC
:10BF8800BDE8F04704F0BEBC28463946224609F011
:10BF9800B7FDC8B9012000FA09F0830501D5154895
:10BFA800EEE7BAF1000F03D0FDF746FC124803E0B4
:10BFB80040EA0800B060114804F0A4FC3946104873
:10BFC800BDE8F047FDF7E2BA09F10109D3E700BF80
:10BFD8002C25002085A701081C8601088FA70108C9
:10BFE8003AB1010893A7010898A701081886010823
:10BFF800A4A70108B3A70108C1A70108CAA7010897
:10C008007BB0010810B5084804F07CFC074B0024FD
:10C018001C741C64064B1C7001F010F904F056FEE9
:10C02800044B1C6010BD00BFD2A701087817002080
:10C03800C32F00209423002070B5064600240B4B24
:10C04800E518AA8816420AD0E1580948FDF79EFA71
:10C058002846002104F0E3FB064804F053FC14349E
:10C0680040F694439C42EAD170BD00BFC08F0108DE
:10C07800FEA701083AB10108F0B504788BB005466F
:10C088000CB1002436E04A4B19680E2303FB041157
:10C0980001F58C70B1F91D51B1F91921B1F91B31B4
:10C0A800009591F82051019591F82151029590F948
:10C0B8000700039001F590713E4891F90210049130
:10C0C80021460134FDF762FA082CDCD16DE02D2BF6
:10C0D80014D1072C1BDC284609F060FD0AAB661C4E
:10C0E80003EB440424F8100C15F8013F303B092BEE
:10C0F800FAD934462B78002BE9D104E0A3F13002B9
:10C10800092A09D8E5E7082CBDF8182009D00BB092
:10C11800BDE8F04001F07ABC202BF8D10135264665
:10C12800E7E7072AF3D8BDF81A00214BA0F2EE2161
:10C1380089B240F2DC55A9421B68E8D8BDF81C104A
:10C14800A1F2EE24A4B2AC42E1D8BDF81E7004B24C
:10C158003EB2A642DBDB0DB2AE42D8DCA542D6DB4E
:10C16800BDF92440642CD2D1BDF8266034B2112C1C
:10C17800CDDCBDF82050B42DC9D8BDF82240B42C70
:10C18800C5D812B24FF00E0E0EFB0233A3F81B11E6
:10C198006421A3F81901A3F81D7183F8205183F8CD
:10C1A800214183F81F1183F822610BB0F0BD00BF55
:10C1B800AC11002008A80108F0B504468FB020464D
:10C1C80009F095FCC5B225BBAC48AD4C04F09AFB10
:10C1D80094F8D61009B9AB4854E049B294F8D42081
:10C1E80094F8D530009194F8D710019194F9D810AB
:10C1F800029194F9D910039194F8DA100491A248A5
:10C2080029460135FDF7C2F9102D04F10704DFD1E5
:10C21800E1E720469D49052209F072FC0546B8B9B8
:10C2280029469B48702209F01EFC9A4B196828463B
:10C238000E2303FB001301300022082883F8232172
:10C2480083F8242183F8252183F82621F0D113E1EE
:10C2580020469149042209F053FC05462046002D4A
:10C268004AD1202109F035FC002800F00581461C40
:10C27800304609F03CFC2C460746884B53F82450BE
:10C288002DB987480FB0BDE8F040FDF77FB93046BB
:10C298002946FAB209F034FC01340028EDD1784A75
:10C2A80002F170011646002382F8DA3082F8D6309F
:10C2B80082F8D53082F8D43007328A42F3D17949EE
:10C2C80001EBC40191F80822934210DAD1F80C72FC
:10C2D800C3EBC302B0183A4400F1D4011768C0F8A0
:10C2E800D4709088888092798A710133E7E729466B
:10C2F8006D48FDF74BF990E06C49072209F000FC06
:10C3080005462046002D4AD1202109F0E2FB0646C9
:10C3180009F0EDFBC4B274BB6548FDF737F9214657
:10C3280064480134FDF732F90E2CF8D15548FDF771
:10C338002DF9002460482146FDF728F90025554AC3
:10C348005E4811680E2202FB04120123D2F8232151
:10C358005B49AB4013425B4B05F1010508BF194629
:10C36800FDF714F90E2DEAD146480134FDF70EF910
:10C37800082CDFD180E03046534909F013FC2C46E5
:10C3880000284CD0022C4FD009F008FC06AB4E49CF
:10C3980043F82400002009F005FC0134F0E74A497D
:10C3A80009F000FC002460B1082C38D009F0F6FB35
:10C3B80006AB454943F82400002009F0F3FB01349B
:10C3C800F1E7082C2BD1069B0F2B28D8DDF81CE0B1
:10C3D800BEF1070F23D8089F0D2F20D8099E06F11C
:10C3E8006402C82A1BD80A9DFF2D18D80B98642808
:10C3F80015D80C99642912D8884210DA0D9C032CA0
:10C408000DD8324AC3EBC303134483F804E05F71C9
:10C418009E71DD71187259729C722D4CCFE60FB067
:10C42800BDE8F04001F0F2BA069B072B20D8079927
:10C438000D291DD80278722A0DD06E2A18D1154AF6
:10C4480012680E2000FB032301228A40D3F823112F
:10C4580021EA020209E00F4A12680E2000FB0323BA
:10C4680001228A40D3F823110A43C3F8232101E0AB
:10C4780001F0CCFA0D4CA2E60FB0F0BD30A80108CF
:10C488002C2500203AB101085BA8010877A801080B
:10C4980000260020AC1100207DA80108549C01084A
:10C4A800A4A701086C84010882A8010828A801082B
:10C4B8007DA701088EA8010820A7010893A80108F4
:10C4C80095B401084FB5010897A80108FC2500207C
:10C4D8009EA401082DE9F743047805468CB9324D2E
:10C4E80095F8A712B5F8A42295F8A6322F4800911E
:10C4F80021460134FDF74AF8102C05F10405EFD167
:10C508004EE009F04BFB0F28044636DC2846202174
:10C5180009F0DFFA264EE4B2D6F84480451CA400A0
:10C528000027284609F03AFB5FFA87F9B9F1010FAD
:10C5380083B208D0B9F1020F0BD0B3F5B47F24D27F
:10C54800726C13530AE0FF2B1FD8736C2344987046
:10C5580004E0FF2B19D8736C2344D87028462C218B
:10C5680009F0B7FA054608B1013502E0B9F1020F42
:10C578000BD10137032FD4D112E00E4800210F222E
:10C5880003B0BDE8F04301F0BEB908EB0400002198
:10C59800042209F068FA03B0BDE8F04301F036BAA6
:10C5A80003B0BDE8F08300BF2C25002099A801083E
:10C5B80078170020ADA801082DE9F0412DED048B76
:10C5C800B2498AB0044609F057FAB1490028204612
:10C5D8000CBF0126072609F04FFAAE49002820466D
:10C5E80008BF022609F048FA002808BF0426F10708
:10C5F80040F10581A848A94C04F084F9002003F013
:10C608008DFFA74804F07EF9A64804F07BF963790A
:10C61800A54AA648013B254652F82310FCF7B6FF69
:10C62800A348FCF7B3FF4FF00008274695ED058AAD
:10C63800B5EE408AF1EE10FA04D19E48FCF7A6FF49
:10C64800002570E09C48D5ED069A95ED079AD5ED42
:10C65800088A4146FCF79AFFB5EEC08AF1EE10FA57
:10C6680002D5202004F046F9B0EE480A06A8FCF7E7
:10C678000DFE01469148FCF789FFF5EEC09AF1EEF0
:10C6880010FA02D5202004F035F9B0EE690A06A8A0
:10C69800FCF7FCFD01468948FCF778FFB5EEC09A27
:10C6A800F1EE10FA02D5202004F024F9B0EE490A80
:10C6B80006A8FCF7EBFD01468048FCF767FFF5EE9E
:10C6C800C08AF1EE10FA02D5202004F013F9B0EE7A
:10C6D800680A06A8FCF7DAFD08F10108014678485F
:10C6E800FCF754FFB8F10C0F05F110059ED1A4E733
:10C6F80049B294F8D42094F8D530009194F8D71022
:10C70800019194F9D810029194F9D910039194F8F1
:10C71800DA1004916B4829460135FCF737FF102DD4
:10C7280004F1070403D094F8D6100029E0D10025BD
:10C738004FF00E0808FB05F80024634A926C424447
:10C748000123D2F80A20A340134240F09480013418
:10C758000E2CF2D10135082DEAD15C485C4C04F06E
:10C76800D1F8D7F8088054F8041F19B15948FCF7D4
:10C778000DFFF8E70D46584B53F8254054B10123F7
:10C78800AB4013EA080F03D054482146FCF7FEFEDD
:10C798000135F0E7524804F0B5F821467B180AAA9B
:10C7A80093F88A3113444F4A8A5C03F8102C0131FC
:10C7B8000829F3D1002306A94B488DF82030FCF74F
:10C7C800E5FE4A4804F09EF8494801F055FC4948FE
:10C7D80004F098F8464801F01FF9474804F092F829
:10C7E8004348FFF777FE4548FCF7D0FE4020FFF7A7
:10C7F80023FC434804F086F83D4801F0DFFCB2070B
:10C8080026D5404804F07EF83F4804F07BF83848C5
:10C8180003F0C4FE3D4804F075F8354801F080F88F
:10C828003B4804F06FF8324801F078FB3948FCF7D0
:10C83800ADFE2F4801F0FCF9374804F063F82C48A6
:10C84800FFF71AFC2D48FCF7A1FE8020FFF7F4FB48
:10C85800730716D5314804F055F8314804F052F8FA
:10C86800234803F075FE2548FCF790FE4FF48070CE
:10C87800FFF7E2FB05E0294622462A48FCF786FE38
:10C8880065E70AB0BDEC048BBDE8F081B3A80108E8
:10C89800BFAC0108BAA80108C0A801082C250020CF
:10C8A800CEA80108E0A80108549C0108ECA80108DA
:10C8B800F7A8010804A9010811A901087CA7010823
:10C8C8007CB0010819A901087817002038A90108C7
:10C8D8001886010848A901081C86010856A90108FC
:10C8E80063A901085DBC01086FA9010878A90108BE
:10C8F8009EA4010887A9010893A901083AB1010873
:10C90800A1A90108AEA90108C1A90108CFA9010878
:10C91800D9A90108E8A90108F6A9010802AA01088D
:10C9280013AA010825AA010810B5084B19680022A6
:10C9380001EBC20393F90240844201D1981C10BD57
:10C948000132042AF4D1002010BD00BF4423002086
:10C9580038B1438811EA030003D08B420CBF012091
:10C968000220704730B50A4B0A491C680A78032A26
:10C978000AD8134604EBC303551CEAB29D88284223
:10C98800F5D00A70981C30BD0A70002030BD00BF79
:10C9980044230020C4170020014B00221A70E1E74D
:10C9A800C41700202DE9F047877890F803C0214D7F
:10C9B800BBB2C7F1640E03EB83065C42C3F1780097
:10C9C8005FFA8EFE7600CCF16408A4B280B2A3B2FE
:10C9D8000FFA83F9B9F1000F05DC002B14BFBA4632
:10C9E8004FF0010A00E0F24613FB03F303FB0CF2DD
:10C9F8001AFB0AF392FBF3F3434403FB09F30A22FD
:10CA080093FBF2F333449BB225F8023FB1F8009050
:10CA18004A880A34C9EB020AA4B21AB202FB0AF223
:10CA28004FF47A73844292FBF3F34B442B80CED1BC
:10CA3800BDE8F087C417002010B5447800780022BC
:10CA480002FB02F3193B634303F6C413534340F656
:10CA5800C411434393FBF1F3034921F81230013227
:10CA6800072AEDD110BD00BFDE1700200430114B9E
:10CA780033F91000B0F5617F10B506DB40F63303DB
:10CA880098420246A8BF1A4601E04FF461720C783A
:10CA9800192340F2833013FB0404944207DA4978DF
:10CAA80013FB01039342B4BF0020012010BD0020F6
:10CAB80010BD00BF0825002010B500F15003027812
:10CAC8008A4203D18478C278944204D304309842CD
:10CAD800F5D1002010BD012010BD1FB5084B1B6803
:10CAE8001B030AD58DF8040001230D2001A98DED43
:10CAF800030A8DF80530FBF783FE05B05DF804FBEB
:10CB0800CC2400201FB5084B1B681B0309D58DF8E2
:10CB18000400029100230D2001A98DF80530FBF7D0
:10CB28006FFE05B05DF804FBCC24002010B5064B61
:10CB380000241C7005F02CFF044B83F82840DC62AD
:10CB48001C865C6310BD00BF902F0020C417002016
:10CB580010B510B9BDE81040E8E700230C225A438D
:10CB68000A4C1119125D824203D00133102BF5D102
:10CB780010BD074B586B18B14A784078824203D2EF
:10CB8800002259631A86DA6210BD00BF208E0108A0
:10CB9800C417002010B540001428A8BF1420002393
:10CBA800074A022199540B4499181424834201F826
:10CBB800014CF5DBFF21D1540F20BDE81040C7E739
:10CBC800A423002010B50A4A0A4B11689B6800BFCD
:10CBD80012689142F7D1084A946B4FF47A7000FBBF
:10CBE80004F2D31AB3FBF4F300FB013010BD00BF0D
:10CBF800F024002010E000E0C417002038B50446F7
:10CC0800FFF7E0FF0546FFF7DDFF401BA042FAD320
:10CC180038BD10B504462CB14FF47A70FFF7EEFF1B
:10CC2800013CF8E710BD2DE9F04F87B088469DF824
:10CC3800444011461A469DF84030814600250C2094
:10CC48006843814E87198057484505D197F808A051
:10CC5800BAF1000F04D0F3E00135042DEFD1EFE075
:10CC6800B9F1010F00F0DA8006DCB9F1000F40F0ED
:10CC7800E78000947548D6E0B9F1020F00F0D18042
:10CC8800B9F1140F40F0DC80714FBB6943F0010328
:10CC9800BB617B694FF0904443F400337B6101260C
:10CCA80003224FF4805B04A94FF090408DF81520C3
:10CCB8000392CDF810B08DF814608DF816608DF8D9
:10CCC80017A0FBF7F1FAA4F828B0C820FFF7A1FFD6
:10CCD800C4F818B07B69039A43F400337B6120469B
:10CCE8004FF4C0534FF0020B04A904938DF815209C
:10CCF8008DF814B08DF816A08DF817A0FBF7D4FAAC
:10CD0800636A23F470436362636A43F46043636253
:10CD1800636A23F470236362636A43F46023636283
:10CD28004C4B4D4C4FF480221A6002F18042A2F520
:10CD38003F321223E366082384F87130136884F8BD
:10CD4800726023F480231360536823F480235360B4
:10CD580094F8703003F1804303F582331A6842F483
:10CD680080221A60E26E3D4B22F01F0002F01F0283
:10CD7800C15806FA02F221EA0202C250E26E3849AC
:10CD880022F01F0002F01F0250F801E006FA02F23A
:10CD98002EEA02024250E26E22F01F0102F01F0248
:10CDA800C85806FA02F20243CA502E4B2E4AC3F85C
:10CDB80000A0FB6943F40003FB612C4B04A8DA6074
:10CDC8008DF810908DF811B08DF812A08DF81360C1
:10CDD80004F068FE2A238DF810309DF813308DF882
:10CDE80011608DF812A01BB104A804F05BFE04E0EA
:10CDF8001F4B4FF48062C3F884201E4A1E4B1360F9
:10CE080002221A721D4A1E4B13601E4A1E491B68D5
:10CE1800116098471D4BE3631D4807E000941D48C7
:10CE280001E01D48009400F027FB48B1064B80F84C
:10CE380004900C2202FB053585F80880686000E044
:10CE4800002007B0BDE8F08F4823002000380140DB
:10CE58000010024014040140C417002008040140D7
:10CE68000C040140D80042420005FA0500ED00E03C
:10CE780000E100E03422002038220020C81F0020F2
:10CE8800A8000020C41F00203C00002004880108DE
:10CE980000180020004400400048004038B5134BFB
:10CEA800202240F2DB151A85684310229A61851EFC
:10CEB8000B24013C14F0FF0411D00C4A938A9BB256
:10CEC80083F020039382938A9BB283F01003284651
:10CED8009382FFF79EFE1920FFF79BFEE9E7044BBC
:10CEE800044A1A60044B054ADA6038BD0004004859
:10CEF800FC9F0020EFBEADDE00ED00E00400FA0567
:10CF0800024A136801331360704700BFF024002001
:10CF1800024B5B6F03B11847704700BFC41700206E
:10CF280003681B6918470368DB68184703689B6830
:10CF3800184703685B68184703681B6818472DE99A
:10CF4800F84FB0F90230934218BF00232DED028B41
:10CF580018BF0370057804460E469146002D40F030
:10CF68008B8007EE902A9FED770AF8EEE77AB6EE07
:10CF7800008A27EE800ADFED747A20EE270AA046A1
:10CF880020EE080A08F0F4FFDFED706A60EE266A0A
:10CF9800B7EE006AB0EE667AA0EE007A40F2DC5393
:10CFA8006365D0EE006A1023A4F8523037EE067A93
:10CFB80076EE866AC6EE077A1823A4F8503027461C
:10CFC80084ED046A27EE807A27EE007A77EE075A16
:10CFD80084ED017AC4ED025A70EE005A84ED037AAA
:10CFE800B8EE007AA5EE807A27EE877A67EEA67A01
:10CFF80084ED057AC4ED067ADFED557A98ED047A6A
:10D0080027EE277AF0EE678AB5EEC07AF1EE10FACD
:10D018004CBF77EE487A77EE087A013517EE900A1A
:10D0280005F012FDD8ED017A67EEA87AC7E90E017E
:10D03800F5EEC07AF1EE10FA4CBF77EEC87A77EECB
:10D04800887A08F1040817EE900A05F0FDFC032D14
:10D05800C7E9080107F10807CED1A6F2DC531B0483
:10D068002367E3676367C4F88030A367C4F8843034
:10D078000123A4F802902370D4F85490B4F9528094
:10D08800636A276A206FE26FD4F840C0D4F8801032
:10D09800C4F88020C9EB060606FA08F64FEAE67BD4
:10D0A800734307FB0B332667A7FB06671F44636CB4
:10D0B800656F60674FEAE27B53430CFB0B3EACFBAA
:10D0C80002237344B61A67EB0307E36AA26AC4F83B
:10D0D80084104FEAE07B434302FB0B3EA2FB002394
:10D0E8007344B6185F41E36CA06CB4F95020A5678F
:10D0F8004FEAE17B4B4300FB0B33A0FB01011944D2
:10D10800636B361A206B4FEAE57B05FB03F300FBE4
:10D118000B3367EB0107A0FB05011944801979411E
:10D1280005F068FC08F1FF3201239340E067C0185E
:10D1380041EBE371424605F05DFCBDEC028B4844CF
:10D14800BDE8F88F6F12833ADB0F4940F404B53F0E
:10D158000000804B2DE9F8430024234B93F8A86086
:10D16800E0B2B0420CD203EB8003204A9B6F32F846
:10D1780010101BB10B2801D8DB6898470134ECE785
:10D188001B4B1B685B032DD500242346E2B2B24239
:10D1980028D2DFF8549009F178074FEA840857F845
:10D1A800242055689D4215D0284604F045F8EFF331
:10D1B8001283502282F3128828216A6A01FB0090A8
:10D1C8000132C0F8D0206A6942F001026A61DBB21C
:10D1D80083F3118857F808301B6800221A6001345D
:10D1E8002B46D3E7BDE8F883C4170020B011002010
:10D1F800CC24002008B50E4B1B6813F4805F0D4B40
:10D2080014BFD3F87421D3F8782193F8A810928822
:10D218000023D8B2884204D2074820F813200133EB
:10D22800F7E7FFF797FF3220BDE80840F1E400BFB9
:10D23800CC240020C4170020B01100200A4B1A6823
:10D248000A4B30B502F48052D3F87441D3F87851C0
:10D2580000230AB1A18800E0A988054820F8131026
:10D2680001330C2BF5D130BDCC240020C41700208D
:10D278007A23002070B5124D0024214605F27D1056
:10D28800702285F87C4108F0EEFB2146D5F8F03194
:10D298000B4A0B4493F9020080B102F27D141E6818
:10D2A8000E5108199C8884809B79837192F87C318F
:10D2B80007310133702982F87C31E7D170BD00BF96
:10D2C800C4170020094B1A680E2303FB0020437A79
:10D2D800FF2B07D0064A12789A4203D9054A32F83A
:10D2E800130000E0808800B2704700BFC01700201C
:10D2F8003C23002008250020026BC168034610B5B6
:10D30800406942B11A6C8C1A013A005D08BF0A469E
:10D31800C0B21A6410BD1A6A805C01328A4228BF02
:10D328000022C0B21A6210BD436B13B190F84400DA
:10D338007047836A406A1B1A584258417047036B0A
:10D3480013B15B68016C01E0C369016A8B423CBFA1
:10D35800C2689B18581AC0B27047836A8169426BC9
:10D368001944D160416A99429DBF0169CB1A536043
:10D37800CB1A96BF0023536083624FF0000380F8F6
:10D388004430136888BF816243F00103136070471B
:10D39800436A8269D154436A02690133934228BFC0
:10D3A80000234362436B1BB11B68DB0705D4D4E73A
:10D3B800026D136843F08003136070474171F7F7FB
:10D3C80089B98160F7F786B9026D036B70B50446B9
:10D3D800D5699BB9A90611D5C36A1BB1908C80B2D7
:10D3E80098470BE0E169928C40694E1CD2B2E66125
:10D3F8004254E169E268914228BFE361616BA1B9D7
:10D408002A0612D5636AA26A9A42236D09D0501C73
:10D41800A669A062B25C1A852369984205D3A16205
:10D4280003E01A6822F080021A602B0742BF236DBE
:10D4380008221A6270BD0D4B0D484FF400525A6015
:10D448000C4A11684FF6FE730B401360426B11686B
:10D458004FF6FE730B401360426A836A9A4200D00B
:10D468007BE7012380F84430704700BF000002408A
:10D4780068240020440002402DE9F0471E46A14BD5
:10D488008CB09842894690469DF850507ED19E4B6C
:10D498009E4A1A609E4A5A6102F580729A614FF458
:10D4A8008072DA601A619B4A1A63143A5A63A2F5C9
:10D4B8004842203ADA6404329A64C3F8088018654E
:10D4C800954B9A6942F480429A615A6942F0010286
:10D4D8005A6102238DF80830032315F0010A8DF8EC
:10D4E80009304FF000038DF80A3014BF02230123DE
:10D4F8002C078DF80B3017D5884C402701978AF0F8
:10D5080001038DF80A30236A23F070632362236ACB
:10D5180043F0E0632362204601A9FAF7C5FEBAF199
:10D52800000F23D1A76121E0B0070ED50CA9402335
:10D5380041F82C3D7948036A23F070630362036A5B
:10D5480043F0E0630362FAF7AFFEF1070ED50CA9CA
:10D55800802341F82C3D7148036A23F0704303622D
:10D56800036A43F0E0430362FAF79EFE0E238DF848
:10D5780000300022012368468DF801308DF8022022
:10D588008DF80330604C04F08DFA08E1644B984242
:10D5980074D1644B5D4A1A604FF48072DA601A6184
:10D5A800614A5A6102F580729A615B4AC3F8088041
:10D5B8001865D36943F40033D36102238DF808302A
:10D5C800032315F0010A8DF809304FF000038DF898
:10D5D8000A3014BF022301232A078DF80B3019D50E
:10D5E8004FF09044042701978AF001038DF80A3020
:10D5F800236A23F470632362236A43F4E06323629B
:10D6080020460DEB0701FAF74FFEBAF1000F25D1BE
:10D61800A76123E0B3070FD50CA9042341F82C3DDB
:10D628004FF09040036A23F470630362036A43F483
:10D63800E0630362FAF738FEF7070FD50CA9082351
:10D6480041F82C3D4FF09040036A23F47043036285
:10D65800036A43F4E0430362FAF726FE26238DF8B3
:10D6680000300022012368468DF801308DF8022031
:10D678008DF803302B4C04F015FA90E02B4B9842B0
:10D6880040F00E812A4B214A1A604FF48072DA600A
:10D698001A61284A5A6102F580729A611E4AC3F8D3
:10D6A80008801865D36943F48023D36102238DF879
:10D6B8000830032315F0010A8DF809304FF00003F4
:10D6C8008DF80A3014BF022301232C078DF80B3084
:10D6D80032D5124C4FF4806701978AF001038DF818
:10D6E8000A30636A23F470636362636A43F4E06335
:10D6F8006362204601A9FAF7D7FDBAF1000F3FD1BE
:10D70800A7613DE000380140682400201C8801081A
:10D71800B8190020580002400010024000040048D8
:10D728000044004014240020B81B0020004800409A
:10D73800C0230020B81D0020B0070FD50CA94FF456
:10D74800806341F82C3D5848436A23F47063436270
:10D75800436A43F4E0634362FAF7A6FDF1070FD585
:10D768000CA94FF4006341F82C3D4F48436A23F459
:10D7780070434362436A43F4E0434362FAF794FD1B
:10D7880027238DF800300022012368468DF80130E8
:10D798008DF802208DF8033004F084F9434CC4F866
:10D7A8002C900027012384F844302762E761A762A0
:10D7B80067626671C4F80880A5712046F6F78AFF8B
:10D7C800F20734D5236B002B2AD001A8FAF708FBFF
:10D7D800E36C01934FF480530A9380230693E36824
:10D7E800ADF8103020230993206B636902930B97DF
:10D7F8000597079708970397FAF71DFB01A9206B70
:10D80800FAF7FBFA236B216D1A6842F001021A60DD
:10D818008A6842F040028A605B689BB2236406E033
:10D82800236D20221A621A6842F020021A60B30798
:10D838002FD5636B43B301A8FAF7D2FAA36C01930F
:10D848004FF480530A93802306932369ADF8103070
:10D8580000251023606B03930B9505950795089594
:10D868000995FAF7E8FA606B01A9FAF7C6FA636B4B
:10D878001A6842F002021A60226D5D605D6093686A
:10D8880043F08003936004E0226D136843F0800343
:10D898001360226D136843F001031360204600E013
:10D8A80000200CB0BDE8F08700040048C023002029
:10D8B800F8B504460E46174600252046202108F0F4
:10D8C80008F90446D0B10134204608F067F9B0F5EC
:10D8D800617F05DB40F634039842A8BF184601E093
:10D8E8004FF46170A0F56170192390FBF3F00DB946
:10D8F800307000E070703B7801333B700DB9012542
:10D90800DBE72046F8BD30B505460C4613462946E8
:10D9180022460248BDE83040FBF738BE00AF010898
:10D928007FB504780646E4B9354B1B6803EB8403DE
:10D93800192193F87B0093F87C6093F8792093F889
:10D948007A304FF4617511FB005011FB06510090BD
:10D9580001912C4821460134FBF718FE142CE3D121
:10D968004BE008F01BF91328054641DC244B701CDA
:10D978001C68202100238DF80F3008F0AAF81E3506
:10D98800064670B10136304608F008F919289FBFDD
:10D9980004EB850358709DF80F30013398BF8DF85C
:10D9A8000F303046202108F094F8064670B1013651
:10D9B800304608F0F3F80D289FBF04EB85039870F4
:10D9C8009DF80F30013398BF8DF80F3004EB8504B4
:10D9D8003046E11C0DF10F02FFF76AFF9DF80F308A
:10D9E800042B0AD0601C0021042208F03CF804E053
:10D9F800054800211322FFF786FF04B070BD00BF61
:10DA0800AC1100201FAF0108ADA80108014802F0C1
:10DA180079BF00BF34AF01082DE9F04304788FB017
:10DA28000546002C59D17B4B0021142209A807AECA
:10DA3800D3F8008008F017F807223046002108F0D4
:10DA480012F805A80023A700059308EB07058380B3
:10DA58001A467149B5F802E031F813C01CEA0E0FF6
:10DA68000AD00DF1380C0E3102F1010E6244595CF6
:10DA780002F81C1C5FFA8EF20133072BE9D1002152
:10DA88000B46664AB5F802E011F802C01CEA0E0F10
:10DA98000AD00DF1380C063203F1010E63448A5C9A
:10DAA80003F8242C5FFA8EF301310629E9D118F81E
:10DAB80007305B498DE841006A78029209A81A0983
:10DAC80003F00F03FBF74DFD2146564809AA013420
:10DAD800FBF75CFD202CA6D198E008F05FF81F2822
:10DAE800044600F3868028462021E4B207F0F1FFBF
:10DAF8001F2C02D9FFF78AFF88E0464B1B6803EB0F
:10DB08008404451C00212046042207F0ACFF0027AE
:10DB1800454B09AE304600210A2217F803905FFAF8
:10DB280087F807F0A0FF002315F8012B32B10A2B64
:10DB380004D04A4502D0F2540133F5E74A455ED194
:10DB480008F1FF33032B09D8DFE803F01005023F83
:10DB58000DF1230134E00DF123011EE0304608F0F9
:10DB68001DF82378C0B243EA001006E0304608F0FA
:10DB780015F8237800F00F001843207031E00133C6
:10DB8800062B0AD0244800F11B069E5D9642F6D16A
:10DB980003445A7D63881343638011F8012F02B34D
:10DBA8000023EFE70133072B0AD01B4800F10E06CC
:10DBB8009E5D9642F6D130F8132063881343638044
:10DBC80011F8012F6AB10023EFE7304607F0E6FFAE
:10DBD8000F2804DC304607F0E1FF607001E0002305
:10DBE80063700137052F93D1012401F073FD6CB9DF
:10DBF80080E70E4800211F22FFF785FE06E0204639
:10DC08000021042207F02FFF0024EEE70FB0BDE843
:10DC1800F08300BFB81F0020348801084988010834
:10DC280042AF010851AF010855880108ADA80108A5
:10DC3800F8B50478064674B9304DB5F8C621B5F87C
:10DC4800C8312F4821460134FBF7A0FC042C05F10C
:10DC58000405F2D1F8BD2B4907F00EFFA8B9274BF0
:10DC68004FF47A714FF4FA62A3F8C611A3F8C821E9
:10DC7800A3F8CA11A3F8CC21A3F8CE11A3F8D02198
:10DC8800A3F8D211A3F8D421F8BD304607F086FFD7
:10DC9800032805462BD83046202107F01AFF0446F2
:10DCA80030B10134204607F079FF0126074600E02D
:10DCB80006462046202107F00CFF10B9BDE8F840C1
:10DCC800A4E6013007F06AFF012EF7D1A7F2EE2291
:10DCD80040F2DC539A42F1D8A0F2EE229A42EDD8F3
:10DCE800064B703503EB8503DF801881F8BD0648C5
:10DCF80000210322BDE8F84005E600BF2C250020DE
:10DD08005DAF010877A8010862B301082DE9FF415A
:10DD180004780546002C39D17348744D02F0F2FDA1
:10DD2800D5ED057AF5EE407AF1EE10FA00F0D880DC
:10DD380021466F48FBF72AFC95ED050A6846FBF774
:10DD4800A5FA01466B48FBF721FC95ED060A6846E3
:10DD5800FBF79CFA01466748FBF718FC95ED070AA4
:10DD68006846FBF793FA01466248FBF70FFC95ED0E
:10DD7800080A6846FBF78AFA013401465E48FBF751
:10DD880005FC0C2C05F11005CAD1A9E05B49052258
:10DD980007F0B6FE40B9554B03F1C00200215961A6
:10DDA80010339342FAD19BE028465549042207F0E4
:10DDB800A7FE04462846002C40D1202107F089FE02
:10DDC800002800F08D80451C284607F090FE074685
:10DDD8004C4B53F824601EB94B4802F093FD7FE08A
:10DDE80028463146FAB207F08BFE01340028EFD1FD
:10DDF8003E4B03F1C0029E46002159611033934205
:10DE0800FAD1424B03EBC4029846D2F804C0BCF1E5
:10DE1800000F04D131463E48FBF7B8FB57E0002716
:10DE280018F834309F42F5DA3B010EEB03056344E2
:10DE38000FCB143585E80F000137F1E707F0AEFE88
:10DE48000B28064647DC2846202107F042FE0546F7
:10DE580050B101352846FBF78FF9244B03EB061325
:10DE680083ED050A012400E004462846202107F036
:10DE780030FE054648B101352846FBF77DF91B4BB6
:10DE880003EB061383ED060A01342846202107F028
:10DE980020FE054648B101352846FBF76DF9134BBE
:10DEA80003EB061383ED070A01342846202107F007
:10DEB80010FE10B9FFF7AAFD12E00130FBF75CF97C
:10DEC8000A4B032C03EB061686ED080AF2D111481B
:10DED800FFF71CFF04E0104801210C22FFF713FD97
:10DEE80004B0BDE8F08100BF70AF01082C25002008
:10DEF8008BAF010891AF01087CB0010877A8010831
:10DF08007DA80108549C0108A4A7010830AE0108A7
:10DF180082A801089EA40108ADA80108F0B50478FC
:10DF280087B006461CBB514B1968062303FB041136
:10DF3800192091F8CA5091F8CB7091F8CE2091F839
:10DF4800C9304FF4617610FB056510FB076000953A
:10DF5800019091F8CC000290C83145484979039165
:10DF680021460134FBF712FB0C2CDCD17CE007F0D6
:10DF780015FE0B28044672DC3C4B701C1D682021E2
:10DF880000238DF8173007F0A4FD064680B101364E
:10DF9800304607F003FE03289FBF062303FB045304
:10DFA80083F8CE009DF817309CBF01338DF81730E9
:10DFB8003046202107F08DFD074680B101373846ED
:10DFC80007F0ECFD0D289FBF062303FB045383F8DD
:10DFD800C9009DF817309CBF01338DF8173006260D
:10DFE8006643A9193846CA310DF11702FFF760FCDC
:10DFF800202107F06EFD074670B10137384607F05B
:10E00800CDFD14289FBF9DF817307619013386F887
:10E01800CC0098BF8DF817303846202107F059FDFD
:10E0280078B1013007F0BAFD0D289FBF062303FB26
:10E03800045383F8CD009DF817309CBF01338DF849
:10E0480017309DF81730062B0ED0062202FB04501D
:10E058000021C93007F007FDFFF7D8FC04E00548A8
:10E0680000210B22FFF74FFC07B0F0BDAC110020D8
:10E0780095AF0108ADA80108F0B5027887B08AB954
:10E088004A4C04F1200694F8F221002348495956D5
:10E0980050B281426DD00C33302BF7D10834B442E2
:10E0A800F1D180E0002204920592451C07F076FD2C
:10E0B800C4B260B2FEF738FC074618B18DF81040BC
:10E0C800012400E004462846202107F002FD054609
:10E0D80038B10135284607F061FD0134ADF812006A
:10E0E800E4B200262846202107F0F3FCB0B3451C13
:10E0F800284607F053FD00222E4951F8223083426A
:10E108005FFA82FE04D00132082AF5D1002300E02C
:10E11800734651F82320824220D1022E0FD0032EBD
:10E1280012D05A1E012ED2B204D0042A13D88DF868
:10E1380014300EE0042A0ED88DF8153009E0052BAE
:10E1480009D88DF8173004E09A1E052A03D88DF8EF
:10E1580016300134E4B20136042EC3D1052C03D89D
:10E1680007B0BDE8F04051E404AB03CB38607960F8
:10E1780019E094F8F7010F4B94F8F65153F8200082
:10E18800B4F8F421009094F8F90153F820000190B4
:10E1980094F8F80153F82000029053F82530064807
:10E1A800FBF7F4F97AE707B0F0BD00BF2C25002093
:10E1B80048230020608D0108B5AF01082DE9F3411F
:10E1C800047880464CB9204601A903F0EFFE0134DB
:10E1D800FFF7F4FF122CF6D16BE007F0DFFCC6B2B4
:10E1E800112E61D8344C06F1D00704EB470308F12F
:10E1F800010020219D7807F06CFC18B9AA1E554231
:10E20800554139E04378682B06D0732B07D0612B32
:10E2180013D14FF0000804E04FF0010801E04FF07F
:10E228000208A8F102035D4200F101004FF020014D
:10E238005D4107F04EFCD8B115B9FFF7E7FB38E0B0
:10E24800013007F0ABFC40F2ED2380B2984205DDC7
:10E2580040F6CA039842A8BF184601E040F2EE20F3
:10E2680004EB4703A0F2EE20192290FBF2F0D870DD
:10E2780004EB470383F8028004EB47040F4AA378B2
:10E28800134493F8262055B1E3780D4840F2EE2464
:10E298001925314605FB0343FBF778F909E03146B8
:10E2A8000848FBF773F904E0074800211122FFF73B
:10E2B8002AFB02B0BDE8F0812C2500203488010833
:10E2C800D4AF0108E6AF010862B3010810B50446EF
:10E2D8002046FEF725FE18B90A20FEF79AFCF7E754
:10E2E80010BD002207490C2303FB02135968814221
:10E2F80004D10022C2621A725A6070470132042A9D
:10E30800F0D1704748230020704708B50B4B002018
:10E3180093F82C10F9F7B0FC094B1B68187A0828F9
:10E3280001BF084B4FF480521A80102208BF5A8050
:10E33800A0F109035842584108BD00BFA8000020B9
:10E3480034220020BC1F0020024B4FF480221A60A8
:10E35800704700BF14040140704770477047FEE7DC
:10E36800FEE7FEE7704730B50024E3B293420DD2D2
:10E37800030F092B94BF3033373301F8143001EB06
:10E388004403002500015D700134EEE730BD30B56F
:10E39800002202F1805303F5B8539B0042F4004475
:10E3A8001D6840F60F7144F0800429400132214372
:10E3B800042A1960EDD1024B40F08000186030BD8E
:10E3C8004C5C00402DE9F347884D894C2B68894EF9
:10E3D8009BB2A380A28831880A40970507D54FF6DB
:10E3E800FF53854A2B6013780133DBB21370A3887F
:10E3F8000B40180440F100830023ADF802302B686D
:10E408007B4F9AB21804A28040F1F682BB8803F0D1
:10E418000F03BB71002B40F0C182784A13689BB28E
:10E428003B803B8803F030037B803B8803F44053F8
:10E438003B8011684BF6BF730B4083F4005383F0A5
:10E44800200343F4004343F080031360BB88D906DC
:10E4580021D4116848F60F730B40694913600B68A3
:10E468001A7A022A884601D0042A02D1F9F790FBC9
:10E478005AE2062A40F06B825A78052A08D11A789F
:10E48800520605D1D878FFF782FFBB681B6A984708
:10E49800E3689B685AE213689BB2ADF80230BDF896
:10E4A80002301F0540F1D0811168554F40F68F7337
:10E4B8000B40544913600A68534B92B213445B00F3
:10E4C80088461A683B68187A092817D092B2520011
:10E4D80002F1804202F5C0421178197051785970E2
:10E4E8009188C8B2090A41EA002159801189C8B245
:10E4F800090A41EA002199809289DA8001221A7278
:10E50800DA8893F80190002A40F0DC801A7812F03B
:10E518007F024AD1B9F1090F0FD1DA78012A00F246
:10E52800B8809978002940F0B4809988002940F093
:10E53800B0809A72A3685B68A9E0B9F1050F10D1A1
:10E5480093F90320002A01DA0823B9E09A78002A0F
:10E55800FAD19A88002AF7D19B7A002B00F0A28082
:10E56800F2E7B9F1030F0ED1DA78012A40F0918071
:10E578009A88002A40F08D805A7A42F020025A7216
:10E58800A368DB6983E0B9F1010F40F08280DA7893
:10E59800012A7ED19A88002A7BD15B7A980678D5A1
:10E5A800F9F78CFB00287DD073E0012A2ED1B9F150
:10E5B8000B0F6ED1E26858799269D97890473B6819
:10E5C8009A7A002A65D0002863D11A79002A60D186
:10E5D8009B78002B5DD1064B9B68DB689847084BFE
:10E5E8001B685A79DA72DA781A735BE0445C004087
:10E5F800BC1F00209C220020C52F0020005C00408A
:10E6080034220020505C004004300020022A40D10F
:10E61800B9F1010FC4D0B9F1030F3AD1587920F0FC
:10E62800800E4FEA8E0202F1804101F5B84110F0E8
:10E63800800F096814BF01F0300101F44051BEF1A8
:10E64800030F26D8B3F802E0BEF1000F21D101B3C1
:10E658009B7AF3B102F1804202F5B84201061368D1
:10E668004BBF23F4E04323F4804323F0400323F01B
:10E6780070034BBF9BB29BB283F0100383F48053AB
:10E6880043F4004343F080031360A3689B699847F1
:10E6980008E0E36848465B69984703280FD00028DC
:10E6A8007FF452AFD8F80020A14B92B213445B001C
:10E6B8001A6800221A6030236380062300E00923C9
:10E6C8003A6847E1B9F1060F12D11A78520678D1A3
:10E6D8009B78012B02D1E368DB6967E0022B02D14A
:10E6E800E3681B6A62E0032B6BD1E3685B6A5DE059
:10E6F800B9F1000F38D15988002962D15A6822F43B
:10E708007F42B2F5003F5CD11A7812F07F0204D143
:10E718009B88002B00F0D58153E0012A08D1E268DC
:10E7280058799269904700284BD13B689B7A17E04B
:10E73800022A46D15A7902F00F010BB29B0003F16D
:10E74800804303F5B84312F0800F1B6814BF03F031
:10E75800300303F44053032933D812F0700F30D13B
:10E76800002B40F0AE812CE0B9F1080F04D11B78E2
:10E778005B0600F0A88124E0B9F10A0F21D11A78CC
:10E7880002F07F02012A1CD19A7AD2B15988C1B904
:10E798005A6822F47F42B2F5803F12D1E268587974
:10E7A80092699047002800F090810AE04BB13A68DE
:10E7B8004FF00008A2F812809361404698474046FF
:10E7C8000BE0E3683A681B6950789847032804D13E
:10E7D800584B1B6809221A72BDE03A68138A4FF633
:10E7E800FF718B4201D10923B4E0022800D00BB994
:10E7F8000823AFE092F9001000291FDAD1880191AF
:10E808000198834202D9019B138210E08B420ED2F9
:10E81800E16891F82C00834201D2002105E093FBC6
:10E82800F0F100FB113313B90121434B1970E36870
:10E8380093F82C309382F9F7ABF98CE00323137229
:10E848004FF44053238086E0BDF802301BB2002B02
:10E85800BFF6D5AD116840F68F730B401360354A8B
:10E8680017683B7A022B904671D0042B6FD0032B8C
:10E8780001D0052B66D1BB693A8A8BB9398A002940
:10E888003BD04FF4405323802C4B1A68284B92B24C
:10E8980013445B001A6800221A60302363802CE05E
:10E8A800002AEBD0B7F81490914528BF91461FFA7B
:10E8B80089FA504698473B8ACAEB03033B827B8A16
:10E8C80053447B821D4B1A681D4B92B213445B0064
:10E8D80009F101021B689BB203F1005303F5405391
:10E8E80052105B004FF0000E9645C7D053F82E101B
:10E8F80020F81E100EF1010EF6E7BB8A8B42D8F8FD
:10E90800003001D8032201E011B105221A720BE090
:10E9180006221A72094B1A68054B92B213445B001F
:10E928001A68196030236380D8F800301B7A0FE02A
:10E938000230002034220020C42F0020505C004008
:10E9480004300020072B02D1E368DB6898470823CE
:10E95800D8F800201372FFF7D8FC5E4B1A684BF604
:10E96800BF7313402288D704228848BF83F480539A
:10E978009004628848BF83F40053D106628848BF78
:10E9880083F01003920648BF83F0200343F400434A
:10E9980043F080034F4A9BB213602DE09A0002F1C6
:10E9A800804202F5B842116889B2ADF80210BDF88C
:10E9B800021009B2002909DA106840F68F71014087
:10E9C8001160013B444A52F823309847BDF80230A1
:10E9D8001F067FF514ADA1798B0003F1804303F581
:10E9E800B84348F60F72186802401A603A4B03EBB6
:10E9F80081039B69984702E5A2883388134059052B
:10EA080005D54FF6FF332B60344B5B689847A288D7
:10EA180031880A40920444BF4DF6FF732B60A388E7
:10EA28002F4A0B40DB0452D54EF6FF732B600023B0
:10EA38001374137C052B41D8DFE803F0030D141879
:10EA4800222D6369264D1BB901F04CFD062300E019
:10EA580005232B743BE001F045FD042323740123B7
:10EA6800636134E002236374032328E0637C013B81
:10EA7800DBB26374637C53BB194B04221A7426E01F
:10EA8800184A13689BB243F01003136005232374DC
:10EA98000A2363741BE0637C114A013BDBB2637495
:10EAA800637C03F0FF0093B90E490C684FF6EF73CF
:10EAB80023400B6006231374506108E00623237477
:10EAC80005E0094B73E6094B71E6094B6FE602B0A6
:10EAD800BDE8F087005C0040208D0108A8000020F8
:10EAE800BC1F0020405C004041780008F97800080D
:10EAF800D578000838B5294C2DED048B94ED008AA3
:10EB0800B0EE480A0546FAF7D3FDF0EE408AB0EEBB
:10EB1800480AFAF76AFD94ED019AB0EE408AB0EE21
:10EB2800490AFAF7C5FDF0EE409AB0EE490AFAF73D
:10EB38005CFD95ED017AD5ED027A95ED006A68EEF7
:10EB4800676A27EE088AE7EE286A68EE000A67EE29
:10EB5800807AE6EE290AB0EE660AE7EEA80A07F020
:10EB680093FADFED0F7A20EE270ADFED0E7A80EEBA
:10EB7800270AD4ED027A30EE270AF2EE047A80EE04
:10EB8800270A07F07FF9BDEC048B83B21A0444BF4F
:10EB980000F5B47083B218B238BD00BFD41F00208E
:10EBA8000000E144DB0F49402DE9F04F2DED028BC9
:10EBB80085B007460293A14B1B889807934636D524
:10EBC800109B9F48DC89B0F900301B1B03F2F3153A
:10EBD80040F2E632954203D8002BB8BF5B4201E011
:10EBE8004FF4FA73B0F90220121B02F2F31440F248
:10EBF800E630844203D8002AB8BF524201E04FF4FD
:10EC0800FA729342B8BF1346C3F5FA73052293FB11
:10EC1800F2F30A22643B53433A7FD21053436422EF
:10EC280093FBF2F3134423EAE373DBB200E06423BB
:10EC38000093CB1C0193B8460024019BDFF828A25F
:10EC480013F8016F0193022C4FEA440905D1BAF970
:10EC580004301B365E43761146E07A493AF81420B0
:10EC680031F91410022012FB0011CBF1000291427D
:10EC780003DB59450A46A8BF5A467349029B31F936
:10EC88000950551B33F91420154403F079FB88B15A
:10EC980007EE905A6D4AB8EEE70AB2EE048A105DA4
:10ECA80080EE080A02F048FF20EE080AFDEEC07A5E
:10ECB80017EE905A614A1288D10712D43AF90930EE
:10ECC8001B365E4393074FEA26160DD5BB7C5D4382
:10ECD8009DF900305D43642395FBF3F506EB25169B
:10ECE80002E03E7A75432E11594B042533F9093059
:10ECF80093FBF5F5574B03F10C02751BA25C92468A
:10ED080098F8012051466A434A43642192FBF1F284
:10ED180097F85110D21108EE102AB1B1022CB8EEB2
:10ED2800C80A08D14A0803D09142A8BF114600E09A
:10ED38000121494803E003F1100000EBC400D3EDC2
:10ED48000A0AFAF7EFF9BDEEC08ADFF808E1434B8B
:10ED580098F80B6018880EF12C0300FB05F253F8A5
:10ED68002410D21206FB0216B6F5001F3C4AA8BFB3
:10ED78004FF400169642B8BF16460EF1380243F813
:10ED8800246052F8243042F82450EB1A0EF1440162
:10ED98004FF6FF720009B2FBF0F043430EF150004A
:10EDA80051F8245050F8242040F824509B112A444C
:10EDB80041F8243097F850101A444FEA840C76131F
:10EDC80000EE102A79B10EF15C00B8EEC00A00EB33
:10EDD800C400DEED0A0ACDF80CC0FAF7A3F9DDF895
:10EDE8000CC0BDEEC00A98F8153010EE102A18EEC7
:10EDF800101A5A43534653431A463144642392FB2C
:10EE0800F3F3184A1B12194422F8091018EE100AD5
:10EE180002F1080101344CF8010002F1140120321A
:10EE2800032C4CF801604CF8023008F101087FF41B
:10EE380004AF05B0BDEC028BBDE8F08F34130020A1
:10EE480008250020BA2F0020C22400205C8D01086C
:10EE580090110020D41F0020F41F0020641100200E
:10EE68000000E0FF48200020501200202DE9F04F5C
:10EE78002DED048B944CDFF85482D4F8A4308DB077
:10EE8800064692489847914894F8B4200146F9F705
:10EE980047FA8F4B1988994604F58272002973D076
:10EEA800D4F8B8301B7808EE103A04F1BC0A04F123
:10EEB800C8054FF0000BB9F8007038F91B00B7F51A
:10EEC8007A7F02BF0023CAF800302B61DAF80030DD
:10EED8000344CAF800302B6907EE900A0133012B6E
:10EEE8004FEA4B01F8EEE77A2B6106D10023C5ED16
:10EEF800017AC5ED007AAB601BE0D5ED006A07EE3C
:10EF0800103A37EEE66AB8EEC77A86EE077A36EE3A
:10EF1800877AD5ED026A85ED017A77EEC77A85EDB5
:10EF2800007AE6EE276AF0EE667AC5ED036AC5ED6B
:10EF3800026A0023012F28F8013053522FD12B6980
:10EF4800012BC3BF03F1FF3300EE103AD5ED037A6E
:10EF58009FED600AC8BFB8EEC00A8DE80600C8BFBA
:10EF680087EE800A07F034FA9DE8060018EE103A9A
:10EF780063B1F8EEC87AB4EEE70AF1EE10FA05DDEF
:10EF88004FF47A73A9F8003000231CE0DAF8003057
:10EF98004FF47A7003F5FA7393FBF0F353520BF1C5
:10EFA800010BBBF1030F0AF1040A05F1140582D124
:10EFB800012F04D138460092FDF7CAFD009A013F9F
:10EFC800A9F80070E0E738F8131032F813003E4D46
:10EFD800091A28F813100133032BF4D13E4F3B686C
:10EFE80013F0020300F0C8823C4B05F585705B689E
:10EFF80098473B4B05F585701A780146F9F790F963
:10F00800B5F8103105F58579002B41D0D5F81401F4
:10F018000023B4F81021334939F913E02A4DB2F529
:10F02800C87F04BF002241F823204FEA830C51F81F
:10F038000C20724441F80C20002129F8131020F804
:10F0480013100133032BE4D1B5F81031012B1AD179
:10F05800D5F818314FF4C87EC83393FBFEF303800C
:10F06800D5F81C21C83292FBFEF242801E4AD5F820
:10F0780020311288C83393FBFEF39B1A83803180BA
:10F088007180FAF761FEB4F81031013BA4F8103131
:10F09800164B1B68590740F18D80B4F824210A4BA0
:10F0A800322A25D1D3F814211188A3F826115188C2
:10F0B8009288A3F82A213288A3F82C217288A3F811
:10F0C8002811A3F82E2115E0D41F0020901100204C
:10F0D800BE2F0020000000006C12002098230020A2
:10F0E800C62F0020EC20002004000020CC240020A3
:10F0F800002A3ED0D4F814A10023B4F82421AA4948
:10F1080039F91300A94D322A04BF002241F82320FF
:10F118004FEA830E51F80E20024441F80E200022D7
:10F1280029F813202AF813200133032BE5D1B5F869
:10F138002431012B18D10C2085F83D3185F83C216C
:10F14800FDF706FDB5F82631AAF80030B5F82831E4
:10F15800AAF80230B5F82A31AAF80430B5F82C31EB
:10F168003380B5F82E317380B4F82431013BA4F80C
:10F17800243194F83E318D4AE3B1D2F81451D2F8D3
:10F188003001002182F83E114FF0320E90FBFEF064
:10F198002880D2F8340190FBFEF06880D2F838312C
:10F1A800834A93FBFEF312889B1AAB8031807180EF
:10F1B800FAF7CAFDD4F81421B4F80A3111885B1A99
:10F1C800A4F80A315188B4F80C315B1AA4F80C3150
:10F1D8009288B4F80E319B1AA4F80E31FDF7F2FCB0
:10F1E800D4F8403194ED516AD4F84861C4F840012C
:10F1F800C3EB000A07EE90AAB8EE678A002528EE4E
:10F20800066A96F800C06B486B490DF10C0E2A4649
:10F2180038F9123007EE903AF8EEE77A67EE867A18
:10F22800EEEC017ABCF1000F1CD007EE90CAF8EEA4
:10F23800E76AB7EE007AC7EE266A39F9123007EEA8
:10F24800903AF8EEE77A37EE667A67EEA67AD1ED6D
:10F25800006AE6EE877AC1ED007AFDEEE77A17EEEE
:10F26800903A01E039F81230438030F8023F013219
:10F27800032A13FB035501F10401C9D1DFF83081DA
:10F288004E4864236B43B8F800506D4393FBF5F583
:10F29800493D03A9ADB2FAF771FA3B2DD6ED016AE3
:10F2A80011D9B4F96431D4ED580A07EE903AF8EE62
:10F2B800E77A434BF4EEE70AF1EE10FA1EDD1A780E
:10F2C80042F008021DE0F7EE007A36EEA77A3B4AD4
:10F2D80087EE877A00233B4931F913100133032B5A
:10F2E80007EE901A92ED006AF8EEE77AE6EE267AD3
:10F2F80067EE877AE2EC017AEDD1D2E71A7822F04C
:10F30800080294ED570A1A7006F0BEFEB0EE409A55
:10F3180084ED000A94ED580AD4ED577AD4ED568A54
:10F32800DFED299A294D20EE000AF1EE688AA7EE52
:10F33800A70A07F04DF8F0EE400AB0EE680A06F0AA
:10F34800A3FEF0EE408A84ED010A29EE290A06F0B0
:10F3580099FD28EEA90A288006F094FD3B6868808C
:10F368001A0739D51A4803A9FAF708FAD6ED026A36
:10F37800174AF7EE007A36EEA77A002387EE877AE7
:10F38800144931F913100133032B07EE901A92ED4B
:10F39800006AF8EEE77AE6EE267A67EE877AE2EC1C
:10F3A800017AEDD10A4842E004210020D41F002050
:10F3B8000400002038120020202100202C210020E9
:10F3C800701200203A1200204C3D0F44C224002045
:10F3D8003C210020961100206D4D03A92846FAF71C
:10F3E800CDF995ED010A95ED007AD5ED027A20EE7A
:10F3F800000AA7EE070AA7EEA70A06F0E9FFB5EE8E
:10F40800400AF1EE10FA11D0D5ED007AC7EE807AF5
:10F41800C5ED007AD5ED017AC7EE807AC5ED017A9F
:10F42800D5ED027A87EE800A85ED020A5848FFF783
:10F4380061FB584BDFED587A1880564B9FED577A91
:10F44800B3F9003028EE278A07EE903A544BF8EECD
:10F45800E77AB3F9002067EEC77AB1EE499ACDEDA5
:10F46800087A07EE902AB3F90220B3F904308DED3B
:10F47800069AF8EEE77AF1EE688ACDED097A07EE9A
:10F48800902AF8EEE77A09A8CDED0A7A07EE903AC5
:10F49800F8EEE77A06A9CDED078ACDED0B7AFAF7F3
:10F4A8006DF973789DED0B7A012B19D13D4B1B78C3
:10F4B8005B070FD4D4F87431402293FBF2F29B1A05
:10F4C80007EE903AF8EEE77A77EE877AFDEEE77A7C
:10F4D800C4ED5D7AD4F87431402293FBF2F301E075
:10F4E800B8F800309DED090A07EE903AF8EEE77A91
:10F4F80037EE677AD4ED5E7A8DED0B7A94ED5F7A0C
:10F5080038EE077A88EE078A9DED0B7A37EE677A30
:10F51800E8EE077AB0EE678AC4ED5E7A06F0B2FCD0
:10F52800D4F880512978FAF751F8D4F884319DED50
:10F538000A0A1844C4F8840106F0A4FC2978FAF7EA
:10F5480045F8D4F88831B0EE480A1844C4F8880160
:10F5580006F098FC6978FAF739F8D4F88C31124A31
:10F5680018441368C4F88C0153441360D4F89031DC
:10F578000133C4F8903105E0A5F80A31A5F80C313B
:10F58800A5F80E310DB0BDEC048BBDE8F08F00BFBF
:10F598006000002048120020BD37863535FA8E3CC1
:10F5A8003A120020C22F0020A42F002001380A4B55
:10F5B800042804D8DFE800F00507090B0D00074A06
:10F5C80008E0074A06E0074A04E0074A02E0074A5B
:10F5D80000E0074A1A607047000100209DAF00084C
:10F5E800B1EB0008AD2301084FAC0008ADA8000836
:10F5F8001DA3000810B54B88DC0641BF2F4B1479BA
:10F608001B6853F8244044BF2D4B43F820404B88D7
:10F618009B0641BF294B54791B6853F8244044BFCB
:10F62800274B43F820404B881C070ED5254B0C78F8
:10F638001B78B3EB141FA1BF204BD4781B6853F879
:10F648002440A4BF1E4B43F820404B889B070ED58F
:10F658001D4B0C781B78B3EB141FDFBF174B547886
:10F668001B6853F82440DCBF154B43F820404B88F7
:10F67800DC070FD5154C0B78247803F00F03A34251
:10F68800DFBF0E4B14781B6853F82440DCBF0C4BCB
:10F6980043F820404B885B070FD50B780C49097855
:10F6A80003F00F038B42A1BF044B92781B6853F8F9
:10F6B8002220A4BF024B43F8202010BDBC17002015
:10F6C8000A0E0020C7160020C5160020C416002008
:10F6D800C6160020254A264826490023F0B5156895
:10F6E80003700B701C461A462E1976884EB92F5D8A
:10F6F8003FB9037000230A704B7007781C461A46FE
:10F708000CE0360548BF013204F1040403F101039B
:10F7180048BFD2B2802CDBB2E6D1EAE7E0B2B84209
:10F728000CD215F8240006099E4200F00F00A8BF6D
:10F73800731C9042A8BF421C0134EFE78A704B70DB
:10F74800C2F3470102F001020A444C1E0A490B4861
:10F758000A70C3F3470203F0010313440470084915
:10F76800501E084A08701370F0BD00BFB81F002073
:10F77800BC16002068210020C6160020C4160020F0
:10F78800C7160020C51600202DE9F04FC24BDA68D5
:10F798002DED028B1A61C14A1168D960C0490B6806
:10F7A80043F020030B60BF4B1978012990460CBF2A
:10F7B800002201221A70BC4B1A78910789B040F1D7
:10F7C8003D83BA490978042940F23883B849097851
:10F7D80001F0040101F0FF0011B922F001021A70D2
:10F7E8001B78DB0702D408B1F7F7A8FFB149CA783C
:10F7F800531C052293FBF2F202EB82029A1AAE4BDB
:10F80800CA701B78039392000023AC4CDFF8CCC27B
:10F81800DFF8D8925CF8231091FBF9F504F10800A1
:10F8280004F1100640F82350A54844F8231000FBC3
:10F83800051142F2107091FBF0F080B226F8130027
:10F848004FF0140E04F1140604F13C0A0EFB036E8B
:10F858005AF823605EF802704EF80210F61B314425
:10F8680044344AF82310052691FBF6F109FB0511EB
:10F8780044F82310039C012C4FEA830BE24605D180
:10F888000238B0F5797F98BF4BF80C100BB90123FB
:10F89800BBE7884CD8F80030226D9FED8A7A8A4EF3
:10F8A8008A4D9B1A07EE903AF8EE677AD8F800303E
:10F8B8002365C7EE877A7C4B1B78B7EE008AF4EE97
:10F8C800C87AF1EE10FA58BFF0EE487A13F0010347
:10F8D800C4ED157A12D005AA00927D4B06AA0192B2
:10F8E8000CCB9AE80300F7F727FE6421059A069BDC
:10F8F800B2FBF1F293FBF1F3328000E033802B800E
:10F9080094F858306B48002B3BD0D0ED157AC26D77
:10F91800DAF80030C8EE276A9B1A026E022507EE55
:10F92800103AB8EEC77ADAF8043027EE267A9B1A2E
:10F93800FDEEC77AB0F9662017EE901A07EE903AF6
:10F94800644BB8EEE77AD3ED007A67EE277A67EE74
:10F95800A67AFDEEE77A17EE903A02FA83F3B0F949
:10F96800642093FBF5F302FA81F29BB292FBF5F265
:10F9780092B2A0F86A30A0F86820A0F86630A0F823
:10F988006420012384F85830534BDAF804101B889C
:10F99800DAF80000474D514E216603F03003E06568
:10F9A800002B00F04B8205F17403009305F17803F6
:10F9B8000193EA6E2B6FF7F7BFFD72682B6F9B1AE6
:10F9C80007EE903A434B326893ED007AEB6EF8EE0F
:10F9D800E77A9B1AEB67384B67EE877A1B78FDEE60
:10F9E800E77A012BC5ED207A03D0022B00F0DF80E7
:10F9F80024E2D5ED287A3A4BD5ED215A95ED255AD2
:10FA080095ED156A95ED264AD5ED274A35491D68C5
:10FA1800B1EE677ABDEEC77AFDEEE77A17EE10EA27
:10FA280017EE90CA0020304A91ED007A52F8207003
:10FA380007EE907AF8EEE77AA2F1140367EEA57A5A
:10FA480033F81060FDEEE77A283217EE903A9B1BE8
:10FA58009BB222F810301BB207EE903AF8EEE77A24
:10FA68003B4467EE857A4400FDEEE77ACDED037AF4
:10FA780007EE903AF8EEE77ABDF80C8067EE847AE4
:10FA8800A7EE867AFDEEC77A17EE902A724531DB2B
:10FA98006245A8BF62462EE000080020F02400203E
:10FAA8006C120020D611002070120020761200205F
:10FAB800C22F002068210020940F00206C21002014
:10FAC800806967FF00007A44EA120020EC120020E7
:10FAD800D81100206C000020341300207812002078
:10FAE800980F0020C80F0020E4210020809698007D
:10FAF800DB0FC940724607EE902AF8EEE77A5FED11
:10FB0800046AC1ED007AFDEEE77A313617EE903AD5
:10FB180043449AB2AB78D1ED027A07EE103AB8EEC8
:10FB2800477A4B684F6027EE267AFB1A88EE077AE9
:10FB3800B6B2622E06EE903AF8EEE66A37EE067A2C
:10FB4800C6EE866A86EE077A76EEE76AE7EE267AEA
:10FB5800C1ED047AC1ED027A0FD964EEA77ABA4EE4
:10FB6800FDEEE77A17EE903AB3F5FA6FA8BF4FF4B7
:10FB7800FA63B342B8BF334600E0002313441BB214
:10FB880040F6B8329342A8BF1346B04A9342B8BF72
:10FB98001346AF4AA352AF4A142303FB002351F87C
:10FBA800142B1A60002840F0498101203BE7AA4B3A
:10FBB800D5F874801F68D4F878903E89DFEDA78A5D
:10FBC8004FEA58039E4228BF1E46B5F8A8301AB21D
:10FBD8009642C3BFD5ED157A9FEDA17A67EE877A75
:10FBE800B6B2C1BFFDEEE77A17EE906AF618B6B264
:10FBF800C8BFA5F8A860D4F8AC50C5EB09052846DD
:10FC0800F7F7DEFC0028D8BF404241F29312904239
:10FC1800CCBF0020012088B307EE905AB8EEE70A5F
:10FC280020EE280AF9F7E1FC07EE908AF8EE677AE9
:10FC380040F6B83320EE270AFDEEC07ACDED037A00
:10FC4800BDF80C20A4F8B02012B29A42A8BF1A46F8
:10FC58007E4B9A42ACBF09EB02034B4448F6A042E4
:10FC6800934203DDA3F50C43A03B04E0002BBCBF8B
:10FC780003F50C43A033C4F8B43001E0C4F8B490E1
:10FC8800D4F8B450C5F50C53283307EE903AF8EE83
:10FC9800E77A67EEA88AB0EE680AF9F709FD8DEDF4
:10FCA800070AB0EE680AF9F7A0FCD4ED317AD4ED72
:10FCB8002E4AD4ED155A94ED2F4A94ED305A6549E1
:10FCC8008DED060AB1EE677ABDEEC77AFDEEE77AEA
:10FCD8000DF1180E17EE10AA17EE90BA0020614A1F
:10FCE800FEEC016A32F91030DFF88C9107EE903A99
:10FCF80007EE106AF8EEE77AB8EEC77A3C32D6EE2D
:10FD0800877A4FEA400CFDEEE77ACDED037ABDF92C
:10FD18000C30B3F57A7FA8BF4FF47A734B45B8BF60
:10FD28004B461FFA83F922F810900FFA89F207EE72
:10FD3800902AF8EEE77A27EEA47ABDEEC77A8DED21
:10FD4800037A27EE847AD1ED007ABDF80C90E7EEBD
:10FD5800257AFDEEE77A17EE902A524503DB5A45DD
:10FD6800A8BF5A4600E0524607EE902AF8EEE77A16
:10FD78009FED3D6AC1ED007ABA7891ED027A06EE00
:10FD8800902AF8EE666A4A684B6066EE866A9A1AA6
:10FD9800C8EE266A143106EE102AB8EEC66A76EE68
:10FDA800A56A86EE256AC5EEA66A36EE476AA6EE0D
:10FDB800867A01ED017A01ED037A25EE077ABDEE28
:10FDC800C77A17EE103ABDEEE77A4B4417EE102AC1
:10FDD80013441BB240F6B8329342A8BF13461B4ADD
:10FDE8009342B8BF13461A4A2CF802301F4A14230C
:10FDF80003FB0023C3ED007A08B901206FE73B79C4
:10FE080023B1642395FBF3F5194B1D803B88984576
:10FE18000DD9D4F8AC30A06FC01AF7F7D1FB80EA3F
:10FE2800E072A2EBE07242F210739A4206DD114BC7
:10FE380001221A700E4BB4F8C8201A8009B0BDEC24
:10FE4800028BBDE8F08F00BF30F8FFFF48F4FFFFDA
:10FE58001C100020F00F0020980F0020D302373923
:10FE68000000C842D0210020DB0FC940C80F002085
:10FE7800900F0020940F002018FCFFFF20B9034BBF
:10FE88001B6808221A8270470148704734220020F4
:10FE98007000002020B9034B1B6808221A827047A3
:10FEA80001487047342200207000002021B9012841
:10FEB8008CBF0220002070470220704710B5094B04
:10FEC8001A68D378042B0BD8074C518ADB002344DB
:10FED80018B99B895B1A138210BD9B68581810BD0E
:10FEE800002010BD3422002070000020054B196846
:10FEF800054B4A8A18B99B8D9B1A0B827047986AE2
:10FF0800104470473422002070000020054B196807
:10FF1800054B4A8A18B99B8E9B1A0B827047186B3F
:10FF2800104470473422002070000020074B1B68E3
:10FF38001B7803F07F03212B06D100F0DF00022895
:10FF480014BF02200020704702207047342200208E
:10FF5800212810B508D1114B1B681B7803F07F03CB
:10FF6800212B10D0022010BD2028FBD10B4B0C4AAE
:10FF78001B6810701B7803F07F03212B094B18BFF7
:10FF880000230BB9EEE7084B044A1268002493617A
:10FF9800548220469847204610BD00BF34220020D6
:10FFA800C72F002085FE00089DFE00087047034B00
:10FFB8001A78202A04BF00221A707047C72F002021
:10FFC800014B04221A607047A82F0020034B9B7B2B
:10FFD80013B1034B05221A60704700BF342200207A
:10FFE800A82F00200D4B0E491A680E4B92B21344ED
:08FFF8005B000D4A1B68C3F316
:020000040801F1
:10000000090310B51362136A9BB201335B1000221F
:100010009A4206D0074851F8044B20F812400132AA
:10002000F6E710BD505C0040206200401E3000200A
:100030003422002058220020014B00225A667047CB
:10004000342200202DE9F843664B674E1B68DFF829
:10005000B881664A00254FF0C0099D7283F8099067
:10006000DD723560D8F8003023F4EC4323F07003E0
:1000700043F400739BB2C8F80030D8F8003023F482
:10008000E04323F040039BB248F2800483F0100366
:100090002343C8F80030336812FA83F35B0040272B
:1000A0001A681F6033689BB203F1005303F5405395
:1000B0005B0028461A6880221A60D8F8003023F4C2
:1000C000F8731B051B0D2343C8F80030484B93F809
:1000D0006410F7F7D5FDD8F80030464A464923F4B6
:1000E000804323F070039BB283F440532343C8F84A
:1000F0000030136823F4EC4323F070039BB21360C9
:10010000336811FA83F35B0003201968C3F8009089
:1001100013683A4923F4E04323F040039BB283F091
:10012000200323431360136823F4804323F07003F8
:1001300023439BB21360536823F4EC4323F0700312
:1001400043F4C0639BB25360336811FA83F35B00DE
:1001500019684FF480711960536823F4804323F0C9
:10016000700323439BB25360536823F4E04323F0AE
:1001700040039BB283F0200323435360D8F80C3034
:100180001F4A23F4EC4323F070039BB2C8F80C30F1
:10019000336812FA83F35B0039461A684FF48872A9
:1001A0001A60F7F76DFDD8F80C3023F4804323F084
:1001B00070039BB283F440532343C8F80C30D8F843
:1001C0000C3023F4E04323F040031C43A4B2C8F8EE
:1001D0000C402846FEF7DFF80A4B01221A60BDE802
:1001E000F88300BF34220020505C0040043000201F
:1001F00070000020045C0040083000201030002017
:100200001C300020A82F0020005C0040134A144B33
:1002100050681B68181810B5146808D011490822D6
:10022000FEF7A5F8204610490422FEF7A0F80F4873
:100230000268002393720E4A012111600D49136078
:100240004FF4E0540B6014600B604FF43641A0F89B
:1002500068101160084A136010BD00BFB0F7FF1F9F
:10026000ACF7FF1FDA000020EA0000203422002053
:10027000405C0040445C0040A82F002010B50446BC
:10028000B0F9000001F00BFCB4F9020001F007FC2A
:10029000B4F90400BDE8104001F001BC10B50446FB
:1002A000006801F0FCFB606801F0F9FBA068BDE8A4
:1002B000104001F0F4BB2DE9F74F0120FCF770FB73
:1002C000002488B3012C2FD8194E4FF04C0909FB9C
:1002D00004FA06EB0A0808F1B407BD7815B1013439
:1002E000E4B2EEE790F9003090F804E01846114BC4
:1002F00003228DE8240001212A4653F82E30FCF712
:1003000096FC834660B106F16C00504429464A468B
:1003100005F0ADFB01231C44C8F86CB0BB70E4B21F
:100320000120FCF723FBCCE703B0BDE8F08F00BF52
:1003300034220020608D01080021222210B51148CE
:1003400005F095FB104B0022194610480424105C60
:1003500083F8F2010132052083F8F741042A4FF0B7
:10036000000483F8F60183F8F94183F8F80103F1FA
:100370000803EAD10123A1F8F431522381F8F031C6
:1003800010BD00BF1C2700202C25002007B001084D
:1003900010B5F7F7CDFD4FF43024012806D11CB17C
:1003A000F7F7C6FD013CF8E7052010BD002C08BF9B
:1003B000052010BD70B50646441E14F8011F89B112
:1003C000094D284605F089FB0028F6D005F1080301
:1003D00098423FBF054B401BC018A31B38BF80F895
:1003E0008A31EAE770BD00BF5DBC01082C25002002
:1003F00007B51D4B03F58472C3F804211B4A92F81C
:1004000092215AB1012A14D1032183F80A1107213C
:1004100083F80C2183F80B110C2208E0022183F8E9
:100420000A11032183F80C2183F80B11072283F8AA
:1004300008210F4B0F4AC3F884204020FCF7B0FA84
:1004400070B10122002390F9000040218DE80C00DA
:10045000094A4FF4E133FCF7EAFB003018BF0120F2
:1004600003B05DF804FB00BF342200202C250020DF
:1004700070000020D5790008017B000801200021D0
:1004800000F09EB9F0B5184A92F80D31D2F810710B
:100490001546032B11D807EBC3025E1C941CF6B261
:1004A00009D013469288D10705D5104203D008E041
:1004B0000131042908D13346EBE785F80D310020DE
:1004C000F0BD93F802E00021074C0C2204F58A7C71
:1004D00002FB01F31CF803209645E9D1234484F87C
:1004E0000D61D3F81801F0BD342200200A4B10B57D
:1004F00019684FF6FB720A401A60084A927B1C4644
:10050000074B0AB1052200E001221A6001F098F9B8
:100510004FF43643236010BD405C0040342200207D
:10052000A82F002007B5064B0093064B0193064900
:10053000064A074B0748F9F72DF803B05DF804FBAE
:10054000B0A1010885A101084CA6010845A6010833
:10055000A4A101080BB0010808B5037833B90C4B0E
:100560000C481978BDE80840F9F714B805F01AFBF3
:1005700002280CD8064B1870074B0C2202FB0030E7
:10058000064B06301860F9F723FA0548E5E708BD81
:10059000782300202BB00108D42C0020D01100209B
:1005A0009EA4010808B503783BB90B4B0B4893F8A0
:1005B000AC17BDE80840F8F7EDBF05F0F3FA0228E4
:1005C00008D8054B83F8AC07F9F76CF9F9F724FA6A
:1005D0000348E8E708BD00BF2C2500202FB0010824
:1005E0009EA4010838B5037803BB214B1B68013377
:1005F0000F2B07D81F490C2202FB03121C469568DB
:100600002DBB00E01C4601340F2C01DD002400E06E
:1006100005D818490C2202FB04129568BDB99C420A
:10062000F1D11548BDE83840F8F7B4BF05F0BAFA83
:100630000F28044605D80F4A0C2303FB00239D68AE
:100640002DB921460D48BDE83840F8F7A3BF084B47
:100650001C60FCF76FFA21462A460948F8F79AFF12
:100660000C235C43034B185DBDE83840FCF774BABB
:10067000F8000020208E01083CB0010852B00108AB
:100680006AB0010873B5037813B9FDF7C3F93DE00B
:100690001F4901AA05F0E7FA00240146264625462F
:1006A00099B134B1012C08D1084605F07BFA064611
:1006B00003E0084605F076FA05461549002001AA30
:1006C00005F0D1FA01340146EAE70B2D02D91148B1
:1006D0000C220BE0022C10D1A6F57A73B3F57A7FC9
:1006E00007D90D484FF47A714FF4FA62FDF70FF90C
:1006F0000CE00A4B03EB45035E80084B084803EB14
:1007000045032946B3F90220F8F744FF02B070BD53
:1007100097A80108ADA80108E1AB010878230020E3
:1007200081B0010838B50D4C23688342054606D1D7
:10073000FDF7DBFD204600214C2205F098F9E36C23
:10074000AB4209D12846FDF7D0FD054800214C22D7
:10075000BDE8384005F08BB938BD00BFA0220020AD
:10076000EC220020034B1A68D379591C1344D17131
:10077000187A70471413002010B5FFF7F3FF84B206
:10078000FFF7F0FF04EB002080B210BD10B5FFF7BB
:10079000F3FF0446FFF7F0FF04EB004010BD064BEB
:1007A00010B5044621461868FCF7CAFB034B1B68CA
:1007B00098796040987110BD181300201413002020
:1007C00038B5044624200D46FFF7E9FF4D20FFF71A
:1007D000E6FF002C084C14BF21203E20FFF7DFFF6E
:1007E0002368002228469A71FFF7D9FF236893F8FF
:1007F0004900BDE83840D2E714130020014600202C
:10080000DEE710B50446C0B2FFF7C9FF200ABDE815
:100810001040C4E710B5044680B2FFF7F2FF200C89
:10082000BDE81040EDE737B58288836804461006BE
:100830000D4641BF2B4991F8AC174FF4CC7000FB2B
:100840000133D10544BF2849097802F03F0244BF73
:1008500001EB410103EB8103042A12D006D8012ADF
:100860000DD0022A32D193F9001030E0102A0AD0BC
:10087000202A0AD0082A29D1B3F9001027E01978D4
:1008800025E0198823E0196821E093ED000A684605
:10089000F8F700FD01461548F8F77CFE05B3D4EDE6
:1008A000037A6846B8EEE70AF8F7F4FC0146104808
:1008B000F8F770FE94ED040A6846B8EEC00AF8F73F
:1008C000E9FC01460A48F8F765FE09E000210948FD
:1008D000F8F760FE25B10848E1682269F8F75AFE8A
:1008E00003B030BD2C250020782300207CA7010810
:1008F00075A7010820A7010890B00108024B014626
:10090000D869FCF71DBB00BF7823002010B5441E3A
:1009100014F8011F21B1034BD869FCF711FBF7E76D
:1009200010BD00BF78230020F7B52B492B4B08786A
:100930002B4D1C682B4B05EB80001A882A4BD0F8F6
:10094000C0101B78294800914FF47A71B4FBF1F183
:10095000F8F720FE26484821F8F71CFE254B1F68B3
:100960000026F3B205EB8302D2F8D010E9B10124DE
:100970009C403C4217D0220715D01F4AD25C0B2066
:1009800000FB0323164A1D4802EB8303D3F8F02033
:10099000F8F700FE022C06D1194B93F8281011B17C
:1009A0001848F8F7F7FD0136DBE71748FFF7AEFF09
:1009B000164B17481A68174B9A420CBF164B174B29
:1009C0001A88174B198892B24FF4FB6303B0BDE845
:1009D000F040F8F7DFBD00BFBC120020F02400207B
:1009E000208E01085C120020FC00002097B0010856
:1009F000DAB001086C12002004010020EAB00108FE
:100A000078230020F2B001083AB1010868110020F3
:100A1000F6B00108005400406C1100206E11002057
:100A2000641100202DE9F0410024804625460F4E38
:100A3000A7594146384605F09DF858B139460C484B
:100A4000F8F7A8FD30190021FFF7EDFE0948FFF780
:100A50005DFF0135143440F694439C42E7D11DB943
:100A60000548BDE8F04151E7BDE8F081C08F0108BD
:100A700002A801083AB10108A4A701082DE9F04F26
:100A80002DED028B83B0054605F035F8064620B102
:100A9000012818D12B782A2B15D15C48FFF736FF97
:100AA00000245B4D5B486159F8F774FD2819314605
:100AB000FFF7B9FE5848FFF729FF143440F6944376
:100AC0009C42EED19CE028463D2105F006F8002826
:100AD00000F08F800346994613F8012D202AFAD0A2
:100AE000441C204605F05EF880462046F8F748FB97
:100AF000C5EB0909B0EE408A0026DFF834A11422C4
:100B000002FB06F40AF5D07B54F80B70384604F06B
:100B1000F2FF03461A4628463946019304F0F4FFD3
:100B2000019B00285BD15FFA89F29A4257D10AEB08
:100B30000402D2ED6B7AF8EEE77A0BEB0405B4EE23
:100B4000E78AF1EE10FA48DBD2ED6C7AF8EEE77A3C
:100B5000B4EEE78AF1EE10FA3FD8B2F8A431D2F839
:100B6000A82113F0200F08BF08EE108A1C0641BF11
:100B70002A4991F8AC174FF4CC7404FB0122D90533
:100B800044BF2749097803F03F0344BF01EB41010B
:100B900002EB8102042B18EE100A0BD004D8013BA3
:100BA000012B0ED810700CE0102B05D0202B06D096
:100BB000082B06D1108004E082ED008A01E082ED6E
:100BC000008A39461748F8F7E5FC2846002103B0AB
:100BD000BDEC028BBDE8F04F25E6134803E001367B
:100BE000A12E8AD1114803B0BDEC028BBDE8F04FB5
:100BF0008CE6284603B0BDEC028BBDE8F04F11E750
:100C000003B0BDEC028BBDE8F08F00BF28B1010836
:100C1000C08F010802A801083AB101082C25002064
:100C2000782300203DB1010848B10108A4A70108BC
:100C3000208E010870B50546284604F05CFF064684
:100C400058B9194B19485A79194B03EB8203BDE87F
:100C50007040D3F8301EF8F79DBC2846154932463F
:100C600004F052FF60B91448144CFFF74FFE54F8DB
:100C7000041F19B11248F8F78DFCF8E7114805E098
:100C80000024114B53F8241019B91048BDE87040E6
:100C90003CE62846324604F037FF01340028F0D104
:100CA000014B0B4D5C71C7E72C25002068B1010892
:100CB000208E010893A7010874B10108509C010817
:100CC0008FA701083AB10108549C0108A4A70108A4
:100CD0009EA4010808B50748FFF718FE064BD8691F
:100CE000FDF7F8FAFCF78AFAF8F7B2FD034B044A6D
:100CF000DA6008BD87B101087823002000ED00E02C
:100D00000400FA0508B50548FFF700FE00F048FBAF
:100D1000F8F7C8FDBDE80840DCE700BF93B1010863
:100D200008B50448FFF7F2FDF8F7BCFDBDE8084040
:100D3000D0E700BFA9B10108772048210122F4F7CC
:100D40009FB8772058210122F4F79AB807B50021FF
:100D500001AB03227720F4F717F89DF805309DF8D2
:100D600004001B0243EA00439DF80600184303B049
:100D70005DF804FB08B5FFF7E9FF014B186008BDFB
:100D80004413002008B5FFF7E1FF014B186008BDD0
:100D90004013002013B506220446432168206B4609
:100DA000F3F7F2FFA0B19DF800209DF8013043EA6F
:100DB000022323809DF802209DF8033043EA02239A
:100DC00063809DF804209DF8053043EA0223A38048
:100DD00002B010BD13B5062204463B2168206B46C5
:100DE000F3F7D2FFA0B19DF800209DF8013043EA4F
:100DF000022323809DF802209DF8033043EA02235A
:100E000063809DF804209DF8053043EA0223A38007
:100E100002B010BD13B501220DF107033A210446BB
:100E20006820F3F7B1FF0520FBF7ECFE9DF80730D3
:100E300003B10123237002B010BD0F4B1A7813B514
:100E40001C46BAB90D4B1B68A3B11A681AB10C49FC
:100E5000486902434A619A88ADF8042002228DF85D
:100E600007209868002201A98DF80620F3F776FE86
:100E70000123237002B010BDBC230020F00200202B
:100E80000010024008B5FFF7D8FF6B2180226820D0
:100E9000F3F7F6FF6420FBF7C0FE6B210322682006
:100EA000F3F7EEFF0F20FBF7B8FE104B19211A786D
:100EB0006820F3F7E5FF0F20FBF7AFFE0C4B1A217C
:100EC0001A786820F3F7DCFF1B2118226820F3F75B
:100ED000D7FF1C2110226820F3F7D2FF68203721AA
:100EE0000222BDE80840F3F7CBBF00BF2403002077
:100EF0000000002008B5FFF7A0FF074B1B7813B1D7
:100F0000012B03D008BD4FF4006201E04FF4805282
:100F1000024B1A8008BD00BFF4020020040000202C
:100F20002DE9F0410369C76805460E461F40002FB2
:100F300035D0B7FA87F24FF00043D340DB432B6143
:100F40001F40A2F11B03042BF1D8DFE803F0221F9E
:100F50001C190300746A24B1013C0023A4B273621B
:100F600001E0EC6AA4B2D6F82080B8F1000FDED020
:100F7000D8F80030404621469847D8F80480F4E776
:100F80003068696B07E07068A96B04E0B068E96BD2
:100F900001E0F068296C036889B29847C7E7BDE8AB
:100FA000F08107B52320FBF738FE68207521012268
:100FB0000DF10703F3F7E8FE28B19DF80700A0F153
:100FC00068035842584103B05DF804FB02464021D3
:100FD0003C20F3F755BF70B500EB8000094CA0F141
:100FE000A1059C3825440444074B15F8010F1E78D1
:100FF0007040FFF7EBFFA542F6D13046BDE87040E8
:10100000E4E700BF1C9D0108C82F002010B5441E56
:1010100014F8010F10B1FFF7DEFFF9E710BD02462B
:1010200080213C20F3F72CBF10B5D420FFF7F7FF49
:101030008020FFF7F4FFA820FFF7F1FF3F20FFF724
:10104000EEFFD320FFF7EBFF0020FFF7E8FF402083
:10105000FFF7E5FF8D20FFF7E2FF1420FFF7DFFF2A
:10106000A120FFF7DCFFC820FFF7D9FFDA20FFF748
:10107000D6FF1220FFF7D3FF8120FFF7D0FFCF204C
:10108000FFF7CDFFD920FFF7CAFFF120FFF7C7FF19
:10109000DB20FFF7C4FF4020FFF7C1FFA420FFF7CC
:1010A000BEFFA620FFF7BBFFAF20FFF7B8FFA620CB
:1010B000FFF7B5FFAE20FFF7B2FF2020FFF7AFFF2D
:1010C0000020FFF7ACFFB020FFF7A9FF4020FFF79B
:1010D000A6FF0020FFF7A3FF1020FFF7A0FF4FF4AB
:1010E0008064013C0020A4B2FFF770FF002CF8D10F
:1010F0008120FFF794FFC820FFF791FFAF20FFF793
:101100008EFF012010BD08B55038C0B2FFF787FF31
:101110000020FFF784FF1020BDE808407FE750392A
:1011200010B50446C8B2FFF77AFF04EB4400400054
:1011300004EB440400F00E00FFF771FFC4F3C3009A
:101140001030BDE810406AE701480249E8E600BFF8
:10115000004801401019002001480249E0E600BFA4
:1011600000400140E818002001480249D8E600BFCD
:1011700000040040C01800204FF080400049CFE636
:101180009818002001480249CAE600BF002C01401F
:101190007018002001480249C2E600BF002C01403F
:1011A00070180020224B10B5224C5A43224BB3FB3F
:1011B000F2F203880139013AA04289B292B29BB29D
:1011C0000ED004F50064A0420AD0B0F1804F07D0E1
:1011D000A4F59834A04203D004F58064A04202D163
:1011E00023F070039BB2154CA04206D004F5806436
:1011F000A0421CBF23F440739BB203800D4BC1621D
:10120000984202850FD003F5006398420BD003F596
:101210004063984207D003F58063984203D003F5FA
:101220008063984201D1002303860123436110BDEE
:1012300040420F00002C014000A24A040010004070
:101240000E4B800A984216D007D8B0F5801F0CD0FC
:101250004A3B98420DD102207047094B984206D074
:101260000233984205D104207047012070470320C3
:101270007047FE2070470020704700BF4B001000F1
:1012800050001000F8B50468064620460F46154683
:10129000FFF7D6FF04284BD8B27A910847B902234A
:1012A0008B40D4F80CE0DB439BB203EA0E03E3600F
:1012B0000A23204A03FB001342F82370043342F848
:1012C000235015463FB1B17AE268890802238B406A
:1012D0009BB21343E360282202FB00522032EFF35B
:1012E0001286502383F3128803B203EB8303DB00DF
:1012F00003F10C011C3329442B4451F8047F17B12E
:1013000017600A6804329942F7D100231360F3B2E0
:1013100083F31188282303FB0050036A1BB1E368A1
:1013200043F0010303E0E2684FF6FE731340E3600D
:10133000F8BD00BF701800200148FCF749B800BF95
:10134000C02300200148FCF743B800BF142400204C
:101350000148FCF73DB800BF682400200E4B1A7806
:10136000692A16D15A88B2F5FB6F12D11A79BE2AB2
:101370000FD193F8D527EF2A4FF000000BD113F8C7
:10138000012B5040054A9342F9D1B0FA80F0400950
:10139000704700207047704700F80308D8FF030823
:1013A0002DE9F04FEF4C00214FF4FB6285B0204651
:1013B00004F05DFBEC4B04F539721A60EB4B002234
:1013C0001A70EB4B04F2AE7119606923237003238A
:1013D000637140F20113A3604FF41673A4F86631F1
:1013E000FA23A4F86831BC23A4F864314FF4FA73EB
:1013F0002021A4F86E31012384F8623184F86A1147
:1014000084F87E316E2184F88631052384F87C11BE
:1014100084F823320A2140F2DC5384F87D11A4F8C9
:1014200098312B2140F24C4384F87F11A4F89A3173
:10143000212140F26C7384F88011A4F89C3123219F
:1014400040F2753384F88111A4F89E314FF4C871CD
:1014500040F64303A4F8A031A4F88211234699185A
:10146000023200254FF01E09242ABE4C81F8A251F9
:1014700081F8A391F3D14FF4FA6340F27E4040F239
:101480007E57DFF8E4B2A4F8C831A4F8CC31A4F850
:10149000D031A4F8D431A4F84401052340F23A70C5
:1014A000A4F84C7140F2EA5701264FF47A78C8222A
:1014B00019214FF0320A84F8DE31A4F846014FF4C6
:1014C000C87340F2DC50A4F84E7140F2B457A4F84F
:1014D000E221039284F8959184F8DD6184F8DF11AC
:1014E000019184F8E06184F8E16184F8E461A4F892
:1014F000E63184F8EA61A4F84A010290A4F8507138
:10150000A4F8543184F8ED61A4F8C681A4F8CA8126
:10151000A4F8CE81A4F8D281A4F84881A4F852A1FD
:10152000A4F856A1FEF708FFDBF8003026744FF050
:10153000170E83F815E083F816E04FF0550EE673AA
:10154000A573A58183F803E04FF00F0E83F805E043
:101550000199D9714FF0220E83F806E021214FF056
:101560000E0E83F80B9083F80C9083F810E05974FA
:101570004FF0350E53214FF0640928274FF02D0C02
:1015800083F81AE0D9764FF05A0E0A2183F81C909E
:101590004FF0780983F80DC083F808E0997483F858
:1015A0000A901D705F709F70DD7583F804A09D73B5
:1015B0001D76DD735D765F7283F814C04FF4FA7C9C
:1015C000A3F84EC0DFF8C0C1C3F838C0C3F83CC0B0
:1015D000DFF8B8C1C3F828C04FF07E5CC3F834C050
:1015E000F7EE087ADFF8A891DFF8A8C1C3ED087A12
:1015F000C3F82C90C3ED097AC3F83090C3F848C003
:10160000F1EE047A02989E774FF04B0C4FF00009F0
:1016100083F8501083F8525083F85170C3F840900B
:10162000C3ED117A83F84CC084F8AEE7A4F8B8078C
:101630004FF0410E042084F8AFE784F8B0A784F897
:10164000B15784F8B55784F8B65784F8B25784F880
:10165000B35784F8B45783F85C0015200191A3F8C0
:101660005850A3F85A50A3F85650C3ED187A83F88F
:1016700068004048D866404818674048586783F873
:1016800078603F4883F8647083F86570FEF792FED7
:10169000DBF800300199039A83F814614FF4487025
:1016A00083F8115183F8125183F8137183F818519C
:1016B000A3F816015E4684F8D81184F8D921A4F85D
:1016C000DA8119460E2202FB05326FF0170082F80C
:1016D0001901032082F81A016FF02F0082F81B0114
:1016E000072082F81C016FF0230082F81D010520FD
:1016F00082F81E0101355A2081F8200181F821016C
:101700006422FF20082D81F81F2181F8220101F1B8
:101710000E01D7D1002183F88911C821A3F88A11BD
:10172000142183F88C11A3F890211E214FF4967296
:1017300083F88D11A3F8922101212822A3F8942186
:1017400083F88E11074B03F1C0021F46C3F81490B3
:1017500010339342FAD10B480021402204F087F95C
:101760001AE000BF2C250020AC11002078230020B7
:10177000D01100209A99193FF6287C3F3D0A773F07
:1017800054BC0108D02700208FC2F53C0000204047
:10179000CDCCCC3E000040400023264D264C59596C
:1017A000FA1804330868C2F8A402382BF5D104F5FE
:1017B00009700021802204F05AF905F138017022E5
:1017C00004F5097004F048F9FDF788FF3668002336
:1017D0000125314604F27C404FF4CC7284F8D437B2
:1017E00084F8D25784F8D35704F036F904F2146021
:1017F00031464FF4CC7204F02FF9104B1B681A6875
:10180000C4F8BA275A68C4F8BE279A68C4F8C22731
:101810001A68C4F8C6275A68C4F8CA279A68C4F870
:10182000CE27022384F8D05484F8683605B0BDE88A
:10183000F08F00BFC09F01082C250020D011002090
:101840001549D1F8883043F47003C1F88830134B40
:101850001A6842F001021A605868114A02405A6040
:101860001A6822F0847222F480321A601A6822F414
:1018700080221A605A6822F4FE025A60DA6A22F064
:101880000F02DA62186B074A02401A6300229A605C
:101890004FF000638B60704700ED00E000100240E5
:1018A0000CC07FF8CCFC00FF38B5094B93F8D45737
:1018B00065B9084C2068FCF718FD074B25601B78BC
:1018C000022B03D1BDE83840FEF7F5BC38BD00BFA0
:1018D0002C250020102D00200C2D0020044B93F807
:1018E000D4371BB9034B1868FBF71EBB00207047A9
:1018F0002C250020102D002038B505460446204632
:1019000014F8011B21B1034B1868FBF719FBF6E72C
:10191000401B38BD102D00200FB407B504AB06499D
:1019200053F8042B01930020F7F732FD03B05DF864
:1019300004EB04B0704700BFA71A0108024B014630
:101940001868FBF7FDBA00BF102D0020F8B5011F85
:1019500006460023083051F8042F02F120043F2CE2
:101960003AD802F108040F2C06D80232032A04D90F
:10197000002B08BF012300E002238142EBD1012BA1
:1019800030680ED0022B1AD0736803F003039B005B
:1019900000F0030043EA0010B36803F003031843A8
:1019A00017E000F00F0040F04000FFF7C7FFB068FD
:1019B000736800F00F0040EA0310C0B209E000F0C5
:1019C0003F0040F08000FFF7B9FF3079FFF7B6FF26
:1019D000307ABDE8F840B1E706F10C0734463A46E4
:1019E000002552F8043D03F18001FF294FEA8505E7
:1019F00010D903F50041B1F5803F02D245F0010551
:101A000008E003F50003B3F1807F34BF45F0020521
:101A100045F00305B242E4D165F03F00C0B2FFF7E4
:101A20008DFF05F00303022B207807D0032B0CD089
:101A3000012B13D1FFF782FF60780FE0FFF77EFFE5
:101A40006078FFF77BFFA07808E0FFF777FF60780A
:101A5000FFF774FFA078FFF771FFE0780434FFF719
:101A60006DFFBC424FEAA505DBD1F8BD10B50446B9
:101A7000C0B2FFF763FFC4F30720BDE810405DE785
:101A800010B504467F2C06D964F07F00C0B2FFF782
:101A900055FFE409F6E7E0B2BDE810404EE7430029
:101AA00083EAE070ECE7084648E700BF0C4B0D49BD
:101AB000DA684378D243C2F30222C2F104029340AF
:101AC00002781B010A44DBB282F80033037801225A
:101AD000580903F01F0302FA03F341F8203070475E
:101AE00000ED00E000E100E073B50546002100686C
:101AF0000122FFF757FB2A6813889BB243F00103CA
:101B00001380EB7A8DF804300124002601A88DF8AB
:101B100005408DF806608DF80740FFF7C7FFEB7AA8
:101B20001B2B0BD1192301A88DF804308DF805402B
:101B30008DF806608DF80740FFF7B8FF02B070BD62
:101B4000F0B5BE4C23782DED028B013B012B85B007
:101B500000F26F816578854240F06B81A378022B9B
:101B600000F06781B64B5B5DE37023796D00F2EEA8
:101B7000048A1BB16319B3F9063009E06319D4ED87
:101B8000037AB3F90630F1EE677AC4ED037A5B426B
:101B900008EE103A2369A94EB8EEC88A1A0388EEF7
:101BA000288A35D5D6ED037AFDEEE77A28EE280AA5
:101BB00017EE903AD6ED057A8DF80A30FDEEE77A09
:101BC00017EE903A8DF80B3004F0A6F9FCEEC07ACF
:101BD00096ED060A17EE903A20EE280AADF8083086
:101BE00004F09AF9FCEEC07A96ED070A17EE903AE7
:101BF00020EE280AADF80C3004F08EF9FCEEC07A25
